:020000040000FA
:1000000031EF65F08B94000C63EF00F0000000000E
:100010000000000000000000056ED8CF06F0E0CF21
:1000200007F00001E9CF0DF0EACF08F0E1CF09F0C9
:10003000E2CF0AF0D9CF0BF0DACF0CF0F3CF14F007
:10004000F4CF15F0FACF16F000C00FF001C010F099
:1000500002C011F003C012F004C013F09DAA34EFE7
:1000600000F09EBA2BEF54F09DA03AEF00F09EB046
:1000700046EF56F09DA240EF00F09EB29DEF57F084
:100080000FC000F010C001F011C002F012C003F068
:1000900013C004F00E8E0DC0E9FF08C0EAFF09C0CE
:1000A000E1FF0AC0E2FF0BC0D9FF0CC0DAFF14C0A9
:1000B000F3FF15C0F4FF16C0FAFF055007C0E0FFBC
:1000C00006C0D8FF1000196ED8CF1AF0E0CF1BF091
:1000D0000001E9CF21F0EACF1CF0E1CF1DF0E2CF23
:1000E0001EF0D9CF1FF0DACF20F0F3CF28F0F4CFF5
:1000F00029F0FACF2AF000C023F001C024F002C09A
:1001000025F003C026F004C027F0A0A28BEF00F07A
:10011000A1B23CEF5DF023C000F024C001F025C087
:1001200002F026C003F027C004F0228E21C0E9FFB0
:100130001CC0EAFF1DC0E1FF1EC0E2FF1FC0D9FFC7
:1001400020C0DAFF28C0F3FF29C0F4FF2AC0FAFF5D
:1001500019501BC0E0FF1AC0D8FF10009EAA06D09D
:10016000ABB204D0AECF1CF19EBAFCD7000C01019B
:100170001F2B00001F510E0802E2010E1E6F00012E
:10018000000C010121512219206F2351201B201F37
:10019000000129EF01F09D9001015A6B216BFF0EC8
:1001A0001C6F0001DBDF01011CB704D01C5302E00F
:1001B000ABA202D053D002D01CC121F11F6B1E6B29
:1001C000226B1C6B0001CADF1CC122F1D0DF0101D0
:1001D0001E2D01D002D0ABA201D040D022A7F1D772
:1001E0002253EFE01F6B1E6B236B1C6B0001B6DF0D
:1001F0001CC123F1BCDF01011E2D01D002D0ABA236
:1002000001D02CD023A7F1D72353EFE02251480887
:100210000CE12351F90809E10001BB2D01D002D006
:10022000010103D0020EBB6F01011F6B1E6B246B1B
:100230001C6B000193DF1CC124F199DF01011E2D0D
:1002400001D002D0ABA201D009D024A7F1D7000180
:1002500098D701012051245D01E102D0010E5A6FAF
:100260001E6B00012DEF54F0C3C1B7F1C4C1B8F14A
:10027000C5C1B9F1C6C1BAF1C7C1BBF1C8C1BCF1B2
:10028000000CC9C1BDF1CAC1BEF1CBC1BFF1CCC127
:10029000C0F1CDC1C1F1CEC1C2F1000CA80EC36F37
:1002A000010EC46F000C546A536A526A516AC00E40
:1002B000B7170F0EB817F2DF000C786A776A766A04
:1002C000756A3F0EB717B86BE9DF000C0101666B6A
:1002D000656B000E82BA010E3D0E006E002EFED739
:1002E000662B663D03D0020E656F12D082AAF1D74D
:1002F000666B000E82BA010E663D03D0010E656F7B
:1003000007D03D0E006E002EFED7662B82BAF1D7C5
:10031000666B0001000C01017D6B010E7C6F7D514D
:100320007F5D0DE303E17C517E5D09E3390E006ED4
:10033000002EFED700D07C2BD8B47D2BF0D7000147
:10034000000C01012C2D6BD03853D8A468D030B2EA
:1003500066D0186AF2BC188CF29CF2BE188EF29E1F
:100360000001B4DF18BCF28C18BEF28E4750320880
:1003700005E101017F6B500E7E6F04D001017F6BA0
:10038000440E7E6F0001C7DF8098818A0101666B91
:10039000656B000E82BA010E663D02D0010E656FDC
:1003A0003D0E006E002EFED7662B82BA02D065533A
:1003B000F0E0819A655333E17F6B140E7E6F00018C
:1003C000AADF80884750320805E101017F6B3C0EAF
:1003D0007E6F04D001017F6B2B0E7E6F00019BDFCF
:1003E0008098818A0101666B656B000E82BA010EEE
:1003F000663D02D0010E656F3D0E006E002EFED7E9
:10040000662B82AA02D06553F0E0819A7F6B190EA9
:100410007E6F000180DF01016553D8B48088000140
:10042000000C0101F451F603F3CF01F0F4CF00F01A
:10043000F703F3500026F551F603F3500020026E47
:100440000001000C9D9A9D90E56BD06B1E0E006E16
:10045000002EFED70000E52BE53D01D09ED082BAEC
:10046000F5D7E56B1E0E006E002EFED70000E52BC3
:10047000E53D01D092D082AAF5D7E56BCF6BCE6B6C
:1004800001017F6B010E7E6F000145DF8A7CCE2B60
:10049000D8B4CF2BCF5303E1CE516308D8A064D09A
:1004A00082BAEED701017F6B010E7E6F000133DF50
:1004B0008A7CCE2BD8B4CF2BCF5303E1CE51DB08AF
:1004C000D8A052D082AAEED78A9CCF5303E1CE5156
:1004D000A20810E2CF530EE1CE51AB080BE3320E6F
:1004E000476E8390090E01017F6FC40E7E6F00017D
:1004F00012DF8380CF5303E1CE51870810E2CF5340
:100500000EE1CE518F080BE33C0E476E8290090E30
:1005100001017F6FC40E7E6F0001FDDE8280CF532C
:1005200003E1CE51870805E2CF5303E1CE518F0896
:100530000BE2CF5303E1CE51A20805E2CF5303E112
:10054000CE51AB0801E210D0CFC0F5F1CEC0F4F12E
:10055000010E0101F76F2E0EF66F000162DF02C07F
:10056000CFF001C0CEF019D0D02BD051040801E358
:100570006DD7CF6BCE6B83928286190E476E8C72CD
:100580008B76030E01017F6FE80E7E6F0001C3DEE4
:1005900047064752F4E1838282860000000C8B8478
:1005A000000C016A026A006A036A0101F75102E164
:1005B000F65118E0100EF86FD890F437F537003682
:1005C0000336F751035C02E1F651005C07E3F65194
:1005D000005ED8A00306F751035ED88001360236CC
:1005E000F82FEAD70001000C01017D6B010E7C6F32
:1005F0007D517F5D0DE303E17C517E5D09E3390EA2
:10060000006E002EFED700007C2BD8B47D2BF0D7D7
:100610000001000C0101716B666B656B7F6B050E51
:100620007E6F000178DE0101712B662B82BA666B4A
:100630007151F90803E366513C0808E2010E376F77
:1006400066513C0802E2020E656F03D084A4E6D72F
:10065000376B716B0001000C51520CE152520AE1F0
:10066000535208E1545206E1586A576A566A010E1D
:10067000556E04D0586A576A566A556A75520CE12D
:1006800076520AE1775208E1785206E17C6A7B6A89
:100690007A6A010E796E04D07C6A7B6A7A6A796A1A
:1006A000000CEF510408D8B05ED201013C53D8A42D
:1006B00002D0000158D27553D8B402D0000153D2F1
:1006C0005453D8B402D000014ED230A002D0000161
:1006D0004AD230A202D0000146D23153D8A443D22C
:1006E0003653D8A440D22E53D8A42BD26551020839
:1006F000D8B427D2010E486E9D90A0928198819A1D
:100700008380396B2F2D01D082802C50CA0824E1C0
:10071000355322E13A5320E13B531EE13C5102089C
:100720001BE1375319E10001C853D8B402D00101CD
:1007300013D001015C51F1080FE15E2D0DD00001D5
:10074000CD53D8B402D0010107D001012B2D01D027
:100750008186010E2E6FF5D12C50CA0805E12F536A
:1007600003E10001EEDD0101656B84B4818684B292
:10077000808883808280376B000144DC01017F6BBD
:100780001E0E7E6F0001C7DD838C010E01017F6F9D
:100790002C0E7E6F0001BFDD55DE98DD0101655135
:1007A000000801E289D1452D01D006D0455102084B
:1007B00003E04551030825E184B410D0838E7F6B9C
:1007C000C80E7E6F0001A7DD2C50CA0805E10101AB
:1007D0002F5303E10001B5DD010112D0452D10D0EA
:1007E00081967F6BFA0E7E6F000195DD8188270E62
:1007F00001017F6F100E7E6F00018DDD8198010178
:1008000086D02C50CA0802E13A5306E00001CE53CC
:1008100017E1CF5315E1010184B40FD081967F6BAE
:10082000FA0E7E6F000177DD838E010E01017F6F6E
:100830002C0E7E6F00016FDD010181860AD100015F
:1008400084A410D0819601017F6BFA0E7E6F0001A7
:1008500062DD8188270E01017F6F100E7E6F00011F
:100860005ADD10D0819601017F6BFA0E7E6F000178
:1008700052DD8188838E010E01017F6F2C0E7E6F09
:10088000000149DD8CDE0101F36B8196CFC0F5F1EB
:10089000CEC0F4F1090EF76FD90EF66F000181DEBC
:1008A00002C07FF101C07EF136DD8188CFC0F5F155
:1008B000CEC0F4F1020E0101F76F300EF66F0001A9
:1008C00070DE02C07FF101C07EF14750320802E1C4
:1008D00022DD01D089DE8198F9DC01016551000833
:1008E00001E2EAD081867F6B370E7E6F000113DD57
:1008F0000101F32B4750320803E1F3512708C5E209
:1009000047503C0803E1F3512F08BFE2A2D0000199
:10091000DDDC01016551000801E2CED08186030EC5
:100920007F6FE80E7E6F0001F6DC39DE2C50CA08BE
:1009300017E101013A53D8B402D0000111D03C5163
:100940000208D8B402D000010BD05E2D01D002D035
:10095000000106D00001CD5303E101017AD000016E
:10096000CE5305E1CF5303E1010173D00001AEDCAA
:1009700001016551000801E29FD0CFC0F5F1CEC062
:10098000F4F1F76B570EF66F00010BDE02C07FF13A
:1009900001C07EF14750320802E1BDDC01D024DE07
:1009A0000101F36B819681887F6B0A0E7E6F0001D7
:1009B000B2DC81988BDC01016551000801E27CD03A
:1009C0008188CFC0F5F1CEC0F4F1010EF76F180E9B
:1009D000F66F0001E6DD02C07FF101C07EF19BDC15
:1009E000819801017F6B140E7E6F000194DC81867B
:1009F000CFC0F5F1CEC0F4F10101F76B870EF66FB1
:100A00000001CFDD02C07FF101C07EF14750320806
:100A100002E181DC01D0E8DD0101F32BF32D01D0EF
:100A2000C1D7F3510308BEE0CFC0F5F1CEC0F4F159
:100A3000F76B7E0EF66F0001B4DD02C07FF101C0DE
:100A40007EF169DCD1DDD0DDCFDD0101F35102089B
:100A5000A9E0030E7F6FE80E7E6F00015CDC2C5076
:100A6000CA0805E101012F5303E100016ADC01011D
:100A7000070E7F6FD00E7E6F00014DDC2C50CA0830
:100A800005E101012F5303E100015BDC0101030ECD
:100A90007F6FE80E7E6F00013EDC0101655303E1CC
:100AA0000001B8DD0101862D02D0050E5B6F372DE8
:100AB00015D00001C86B010181967F6B640E7E6FBB
:100AC000000129DC839E01017F6BC80E7E6F00014F
:100AD00022DC839201012F53D8B45B6B2C50CA08DF
:100AE00008E12C50CA080EE13A2D01D002D03B2D6E
:100AF00009D0839C7F6BFA0E7E6F00010CDC81961F
:100B000080980101375308E1010E2E6F0001CE538A
:100B100003E1CF5301E18390000141DD2C50CA086D
:100B20000FE101012C2D01D002D0000109D0385372
:100B3000D8B402D0000104D000018EDD010EC56FD3
:100B40000101496B4B6B396B416B4C6B2E2D0AD0FD
:100B50002F2D01D005D0382D01D002D0762D02D016
:100B6000010E306F486A0001000C01012B2D70D07E
:100B70003753D8A46DD030B06BD0186AF2BC188C43
:100B8000F29CF2BE188EF29E000166EC01F018BCD9
:100B9000F28C18BEF28E4750320805E101017F6BDE
:100BA000500E7E6F04D001017F6B440E7E6F0001FA
:100BB0008BEC01F0819681880101666B656B000EFC
:100BC00082BA010E663D02D0010E656F3D0E006EC9
:100BD000002EFED7662B82BA02D06553F0E08198D2
:100BE000655336E17F6B140E7E6F00018BEC01F0D4
:100BF00081864750320805E101017F6B3C0E7E6F14
:100C000004D001017F6B2B0E7E6F00018BEC01F095
:100C1000819681880101666B656B000E82BA010EB8
:100C2000663D02D0010E656F3D0E006E002EFED7B0
:100C3000662B82AA02D06553F0E081987F6B190E73
:100C40007E6F00018BEC01F001016553D8B4818601
:100C50000001000C0101726B666B7F6B050E7E6FED
:100C600000018BEC01F00101722B662B82BA666BDE
:100C70007251F90803E366513C0808E2010E386F2F
:100C800066513C0802E2020E656F03D084A2E5D7EC
:100C9000386B726B0001000CEF510408D8B08DD294
:100CA00001013D53D8A402D0000187D27653D8B4B5
:100CB00002D0000182D25553D8B402D000017DD2B7
:100CC00030A002D0000179D230A202D0000175D24A
:100CD0003253D8A472D23653D8A46FD22F53D8A48B
:100CE0005AD265510208D8B456D2010E486E9D9072
:100CF000A0928198819A8280396B2E2D01D08380B9
:100D00002C50CA0824E1355322E13A5320E13B53E9
:100D10001EE13D5102081BE1385319E10001C9539E
:100D2000D8B402D0010113D001015C51F1080FE1E8
:100D30005E2D0DD00001CD53D8B402D0010107D0F3
:100D400001012C2D01D08088010E2F6F24D22C5050
:100D5000CA0805E12E5303E1000107DF0101656BBD
:100D600084B4818684B2808883808280386B00015D
:100D700002EC00F001017F6B1E0E7E6F00018BEC18
:100D800001F0838C010E01017F6F2C0E7E6F00013C
:100D90008BEC01F022EC02F066EC01F001016551F0
:100DA000000801E2AED1452D01D006D04551020820
:100DB00003E04551030828E184B211D081807F6BA4
:100DC000C80E7E6F00018BEC01F02C50CA0805E1C3
:100DD00001012E5303E10001C8DE010114D0452DAD
:100DE00012D080987F6BFA0E7E6F00018BEC01F0C1
:100DF000818A270E01017F6F100E7E6F00018BEC40
:100E000001F0819A010194D02C50CA0802E13A53B2
:100E100006E00001CE5319E1CF5317E1010184B27E
:100E200011D080987F6BFA0E7E6F00018BEC01F081
:100E30008180010E01017F6F2C0E7E6F00018BEC13
:100E400001F0010180882AD1000184A212D080988B
:100E500001017F6BFA0E7E6F00018BEC01F0818A3D
:100E6000270E01017F6F100E7E6F00018BEC01F0E9
:100E700012D0809801017F6BFA0E7E6F00018BEC1F
:100E800001F0818A8180010E01017F6F2C0E7E6F3F
:100E900000018BEC01F0CFEC02F00101F36B8098C4
:100EA000CFC0F5F1CEC0F4F1090EF76FD90EF66F91
:100EB0000001D1EC02F002C07FF101C07EF18BECA9
:100EC00001F0818ACFC0F5F1CEC0F4F1020E01012C
:100ED000F76F300EF66F0001D1EC02F002C07FF127
:100EE00001C07EF14750320803E18BEC01F002D0E3
:100EF000F4EC02F0819A66EC01F001016551000802
:100F000001E2FFD080887F6B370E7E6F00018BEC93
:100F100001F00101F32B4750320803E1F351270898
:100F2000BEE247503C0803E1F3512F08B8E2B6D0C7
:100F3000000166EC01F001016551000801E2E1D019
:100F40008088030E7F6FE80E7E6F00018BEC01F04E
:100F5000CFEC02F02C50CA0817E101013A53D8B483
:100F600002D0000111D03D510208D8B402D00001D6
:100F70000BD05E2D01D002D0000106D00001CD5370
:100F800003E101018BD00001CE5305E1CF5303E112
:100F9000010184D0000166EC01F0010165510008F7
:100FA00001E2AFD0CFC0F5F1CEC0F4F1F76B570E30
:100FB000F66F0001D1EC02F002C07FF101C07EF1BA
:100FC0004750320803E18BEC01F002D0F4EC02F060
:100FD0000101F36B8098818A7F6B0A0E7E6F00019E
:100FE0008BEC01F0819A66EC01F00101655100087B
:100FF00001E287D0818ACFC0F5F1CEC0F4F1010EB5
:10100000F76F180EF66F0001D1EC02F002C07FF10D
:1010100001C07EF18BEC01F0819A01017F6B140E0F
:101020007E6F00018BEC01F08088CFC0F5F1CEC05F
:10103000F4F10101F76B870EF66F0001D1EC02F0BD
:1010400002C07FF101C07EF14750320803E18BEC12
:1010500001F002D0F4EC02F00101F32BF32D01D0EA
:10106000B9D7F3510308B6E0CFC0F5F1CEC0F4F123
:10107000F76B7E0EF66F0001D1EC02F002C07FF13B
:1010800001C07EF18BEC01F0F4EC02F0F4EC02F024
:10109000F4EC02F00101F35102089CE0030E7F6FB3
:1010A000E80E7E6F00018BEC01F02C50CA0805E1C0
:1010B00001012E5303E1000158DD0101070E7F6F8E
:1010C000D00E7E6F00018BEC01F02C50CA0805E1B8
:1010D00001012E5303E1000148DD0101030E7F6F82
:1010E000E80E7E6F00018BEC01F00101655303E116
:1010F0000001B0DD0101872D02D0050E5B6F382D98
:1011000014D080987F6B640E7E6F00018BEC01F031
:10111000819001017F6BC80E7E6F00018BEC01F0A6
:10112000829601012E53D8B45B6B2C50CA0808E19B
:101130002C50CA080FE13A2D01D002D03B2D0AD025
:10114000839C7F6BC80E7E6F00018BEC01F0819653
:1011500080980101385308E1010E2F6F0001CE5332
:1011600003E1CF5301E182900001CFEC02F02C505B
:10117000CA0810E101012B2D01D002D000010AD0D4
:101180003753D8B402D0000105D000012CEC03F095
:10119000010EC56F0101496B4B6B396B426B4D6B97
:1011A0002F2D0AD02E2D01D005D0372D01D002D001
:1011B000752D02D0010E306F486A0001000C01014C
:1011C0003353D8B4346B2C50CA0823E13A2D01D0E4
:1011D00002D03B2D1ED03A2D03D03B2D01D0BED1E5
:1011E0003A2D0AD03B5308E1000156DD01012F6B77
:1011F000306B010E2C6FB2D13A530BE13B2D09D06D
:10120000000151EC03F001012E6B306B010E2B6FCE
:10121000A5D10001EF510408D8B0A1D10101545368
:1012200005E05553D8B402D0000199D130A002D0C6
:10123000000195D130A202D0000191D1755303E095
:101240007653D8A48BD13C51020804E03D510208EA
:10125000D8A484D13153D8A481D13253D8A47ED11B
:101260002D53D8A47BD165510208D8B477D1656BD2
:10127000060E5D6F2E2D03D02F2D01D004D02B2D07
:101280002AD02C2D28D0545309E1755307E1372D6E
:1012900005D0376B00010AEC03F00101555308E15A
:1012A000765306E1382D04D0386B0001D3DC010100
:1012B000545306E1755304E1375302E1010E2B6FDD
:1012C000555306E1765304E1385302E1010E2C6FC9
:1012D000010E2D6F43D1010E486EA0928198819A24
:1012E000545304E1755302E184B48186555304E1FB
:1012F000765302E184B2808854530AE1755308E1C1
:101300003C51020805E1372D03D03553D8B4376B73
:1013100055530AE1765308E13D51020805E1382DA5
:1013200003D03553D8B4386B000102EC00F0010152
:101330007F6B1E0E7E6F00018BEC01F0838C010E23
:1013400001017F6F2C0E7E6F00018BEC01F001011B
:1013500054530DE175530BE13C51020802E190A595
:1013600005D08A2D04D03C510208D8B4838E555341
:101370000DE176530BE13D51020802E190A905D041
:101380008B2D04D03D510208D8B48180010E7F6FAF
:101390002C0E7E6F00018BEC01F066EC01F0010178
:1013A0006551000801E254D054530DE175530BE12F
:1013B0003C51020802E190A505D08A2D04D03C5191
:1013C0000208D8B4818655530DE176530BE13D51A7
:1013D000020802E190A905D08B2D04D03D510208EE
:1013E000D8B480880F0E7F6FA00E7E6F00018BEC4B
:1013F00001F0CFEC02F00101545312E1755310E1FA
:101400003C51020802E190A505D08A2D09D03C513B
:10141000020806E1655304E100010AEC03F0010152
:10142000555311E176530FE13D51020802E190A9B5
:1014300005D08B2D08D03D51020805E1655303E12D
:10144000000108DC0101372D01D002D0382D43D036
:101450003C51020802E190A505D08A2D06D03C51EE
:10146000020803E1372D01D081963D51020802E1C7
:1014700090A905D08B2D06D03D51020803E1382DEF
:1014800001D080987F6B640E7E6F00018BEC01F0C1
:1014900001013C51020802E190A505D08A2D0AD035
:1014A0003C51020807E1372D05D0839E65510208A3
:1014B00001E083923D51020802E190A905D08B2DF5
:1014C0000AD03D51020807E1382D05D081906551C1
:1014D000020801E082962C50CA080AE0839C7F6BC8
:1014E000C80E7E6F00018BEC01F08098819601019F
:1014F0003C51020802E190A505D08A2D0DD03C5147
:1015000002080AE1375308E1545306E1755304E138
:10151000655302E1010E2B6F3D51020802E190A9D3
:1015200005D08B2D0DD03D5102080AE1385308E15A
:10153000555306E1765304E1655302E1010E2C6F29
:10154000010E2D6F2C50CA0808E1000166EC01F075
:101550002CEC03F0010EC56F0101486A0001010186
:101560007F6B0A0E7E6F00018BEC01F0000CEF51D7
:101570000408D8B07CEF0EF001013C5306E13D5366
:10158000D8A403D000017CEF0EF030A003D00001FE
:101590007CEF0EF030A203D000017CEF0EF031534F
:1015A000D8A47DEF0EF03253D8A47DEF0EF0335364
:1015B000D8A47DEF0EF065510208D8B47DEF0EF08F
:1015C000545304E05553D8A465EF0EF0755304E06E
:1015D0007653D8A465EF0EF09D90010E486EA09250
:1015E0008198819A83808280080E5D6F2E5308E176
:1015F0002F2D06D0000151EC03F026EF0EF0010173
:101600002F5308E12E2D06D000014CEC06F026EFFA
:101610000EF00101302D04D0000126EF0EF0010183
:101620002C50CA084AE13A5348E13B5346E13C5149
:10163000020802E12B5305E03D51020805E12C535D
:1016400003E10001BCDD01013C531AE02B2D14D055
:101650003C51020811E137530FE15E2D0DD000011E
:10166000CD53D8B402D0010107D001012B2D01D0F8
:101670008186010E2E6F04D0000151EC03F00101B0
:101680003D531AE02C2D14D03D51020811E138537E
:101690000FE15E2D0DD00001CD53D8B402D0010171
:1016A00007D001012C2D01D08088010E2F6F04D0AE
:1016B00000014CEC06F0010158D2656B2E5303E09B
:1016C0002F53D8A4EAD23053D8A4E7D284A405D0AB
:1016D000755303E15453D8B4818684A205D0765360
:1016E00003E15553D8B48088376B386B000102ECA6
:1016F00000F001017F6B1E0E7E6F00018BEC01F08C
:10170000838C010E01017F6F2C0E7E6F00018BEC2C
:1017100001F022EC02F066EC01F0010165510008D5
:1017200001E252D2452D01D006D04551020803E016
:10173000455103083EE184A402D084B21AD0545328
:1017400007E1755305E184B403D03C5301E0838E77
:10175000555307E1765305E184B203D03D5301E0D0
:101760008180010E7F6F2C0E7E6F00018BEC01F0EB
:101770000101452D1DD0000166EC01F0010165510C
:10178000000801E221D2819680987F6BFA0E7E6F6D
:1017900000018BEC01F08188818A270E01017F6FA7
:1017A000100E7E6F00018BEC01F08198819A01018F
:1017B0000BD12C50CA0806E00001CE532AE1CF53CA
:1017C00028E1010184A4819684A280987F6BFA0E9F
:1017D0007E6F00018BEC01F084A4838E84A2818053
:1017E000010E01017F6F2C0E7E6F00018BEC01F06A
:1017F0000101545305E1755303E13C53D8A481869C
:10180000555305E1765303E13D53D8A48088ADD10B
:10181000000184B402D084A230D00101545307E106
:10182000755305E184A403D03C53D8A48196555345
:1018300007E1765305E184A203D03D53D8A48098F4
:101840007F6BFA0E7E6F00018BEC01F001015453A7
:1018500005E1755303E13C53D8A48188555305E154
:10186000765303E13D53D8A4818A270E7F6F100E73
:101870007E6F00018BEC01F028D00101545307E189
:10188000755305E184A403D03C53D8A481965553E5
:1018900007E1765305E184A203D03D53D8A4809894
:1018A0007F6BFA0E7E6F00018BEC01F00101545347
:1018B00005E1755303E13C53D8A48188555305E1F4
:1018C000765303E13D53D8A4818A0101545305E1C5
:1018D000755303E13C53D8A4838E555305E17653E9
:1018E00003E13D53D8A48180010E7F6F2C0E7E6FE3
:1018F00000018BEC01F0CFEC02F00101F36B81965B
:101900008098CFC0F5F1CEC0F4F1090EF76FD90E73
:10191000F66F0001D1EC02F002C07FF101C07EF150
:101920008BEC01F00101545305E1755303E13C5385
:10193000D8A48188555305E1765303E13D53D8A4DB
:10194000818ACFC0F5F1CEC0F4F1020EF76F300EF0
:10195000F66F0001D1EC02F002C07FF101C07EF110
:101960004750320803E18BEC01F002D0F4EC02F0B6
:101970008198819A66EC01F001016551000801E24D
:1019800023D1545305E1755303E13C53D8A4818618
:10199000555305E1765303E13D53D8A480887F6B0E
:1019A000370E7E6F00018BEC01F00101F32B4750E5
:1019B000320803E1F3512708A2E247503C0803E153
:1019C000F3512F089CE2D1D0000166EC01F0010137
:1019D0006551000801E2F8D0545305E1755303E165
:1019E0003C53D8A48186555305E1765303E13D531A
:1019F000D8A480882C50CA0806E13A5304E13B532E
:101A000002E1656BB2D0030E7F6FE80E7E6F0001BE
:101A10008BEC01F0CFEC02F0CE5305E1CF5303E1A4
:101A20000101A3D0000166EC01F00101655100083D
:101A300001E2CAD0CFC0F5F1CEC0F4F1F76B570E7A
:101A4000F66F0001D1EC02F002C07FF101C07EF11F
:101A50004750320803E18BEC01F002D0F4EC02F0C5
:101A60000101F36B819680988188818A7F6B0A0ED1
:101A70007E6F00018BEC01F08198819A66EC01F099
:101A800001016551000801E29FD0545305E17553EF
:101A900003E13C53D8A48188555305E1765303E113
:101AA0003D53D8A4818ACFC0F5F1CEC0F4F1010E28
:101AB000F76F180EF66F0001D1EC02F002C07FF153
:101AC00001C07EF18BEC01F08198819A01017F6B5E
:101AD000140E7E6F00018BEC01F00101545305E1FF
:101AE000755303E13C53D8A48186555305E17653E1
:101AF00003E13D53D8A48088CFC0F5F1CEC0F4F106
:101B0000F76B870EF66F0001D1EC02F002C07FF197
:101B100001C07EF14750320803E18BEC01F002D0A6
:101B2000F4EC02F00101F32BF32D01D09BD7F3511C
:101B3000030898E0CFC0F5F1CEC0F4F1F76B7E0E4C
:101B4000F66F0001D1EC02F002C07FF101C07EF11E
:101B50008BEC01F0F4EC02F0F4EC02F0F4EC02F0A7
:101B60000101F3510208D8B47DD70F0E7F6FA00E8C
:101B70007E6F00018BEC01F0010165530AE15453C3
:101B800008E1755306E13C5304E000010AEC03F060
:101B9000010165530AE1555308E1765306E13D53CF
:101BA00004E000012AEC06F00101862D03D0872D08
:101BB00001D003D02351B90802E1050E5B6F372D28
:101BC00001D002D0382D2DD0545308E1755306E1D1
:101BD000372D04D081960001C86B0101555305E1F2
:101BE000765303E1382D01D080987F6B640E7E6FB1
:101BF00000018BEC01F00101545306E1755304E13F
:101C0000372D02D0839E8392555306E1765304E12B
:101C1000382D02D081908296372D03D0382D01D0F7
:101C20005B6B2C50CA0808E12C50CA0810E13A2D11
:101C300001D002D03B2D0BD0839C010E7F6F2C0E68
:101C40007E6F00018BEC01F0819680980101655355
:101C500011E154530FE175530DE137530BE13C5340
:101C600009E0010E2E6F0001CE5303E1CF53D8B42B
:101C700083900101655311E155530FE176530DE156
:101C800038530BE13D5309E0010E2F6F0001CE5395
:101C900003E1CF53D8B4829001010001CFEC02F0F0
:101CA000010E0101306F2351B90808E1010E476FA1
:101CB000375302E0385302E1050E5B6F496B4A6B04
:101CC0004B6B4C6B4D6B416B426B345316E12351A4
:101CD000F90807E00001FD2D01D002D001010DD06F
:101CE000010183530AE1060E5B6F130E7F6F880EAE
:101CF0007E6F00018BEC01F00101346B486A00013A
:101D0000000C010181B909D0010E416F436F83803E
:101D10002F2D03D0422D01D082800001000C010143
:101D200081B909D0010E426F446F82802E2D03D0FD
:101D3000412D01D083800001000C01013D53D8B436
:101D4000E5D130B0E3D130B2E1D13253D8A4DED105
:101D50003653D8A4DBD12F2DCED1010E486E9D90E5
:101D6000A0928198819A838082802C50CA080CE1CD
:101D70003A530AE13B5308E13D51020805E15E2D6B
:101D800003D02C2D01D0A9D184B481862C50CA084F
:101D900004E10001B5EC05F001018088000102ECCE
:101DA00000F001017F6B1E0E7E6F00018BEC01F0D5
:101DB000838C010E01017F6F2C0E7E6F00018BEC76
:101DC00001F022EC02F066EC01F00101655100081F
:101DD00001E23AD14551030805E12C2D03D05E2DD7
:101DE00001D06ED080987F6BFA0E7E6F00018BEC75
:101DF00001F0818A2C50CA0802E1B5EC05F0050E0D
:101E000001017F6FDC0E7E6F00018BEC01F02C5026
:101E1000CA0802E1B5EC05F0050E01017F6FDC0E8A
:101E20007E6F00018BEC01F02C50CA0802E1B5EC8A
:101E300005F0050E01017F6FDC0E7E6F00018BEC5B
:101E400001F02C50CA0802E1B5EC05F0050E0101C5
:101E50007F6FDC0E7E6F00018BEC01F02C50CA0806
:101E600002E1B5EC05F0050E01017F6FDC0E7E6F1F
:101E700000018BEC01F02C50CA0802E1B5EC05F032
:101E8000030E01017F6FE80E7E6F00018BEC01F005
:101E9000819A01017F6B140E7E6F00018BEC01F0C3
:101EA00066EC01F001016551000801E2CDD03D5121
:101EB000020805E12C2D03D05E2D01D08088C4D00E
:101EC0002C50CA080FE12B2D0DD037530BE1000128
:101ED000B5EC05F0040E01017F6F7E0E7E6F0001F0
:101EE0008BEC01F0000166EC01F0CE5304E1CF531E
:101EF00002E10101A9D0CFC0F5F1CEC0F4F1010E8D
:101F00000101F76F180EF66F0001D1EC02F002C06C
:101F10007FF101C07EF14750320803E18BEC01F004
:101F200002D0F4EC02F00101F36B8098818A7F6BA0
:101F30000A0E7E6F00018BEC01F0819A66EC01F0D5
:101F400001016551000801E27FD0818ACFC0F5F11F
:101F5000CEC0F4F1010EF76F180EF66F0001D1EC50
:101F600002F002C07FF101C07EF18BEC01F0819A9A
:101F700001017F6B140E7E6F00018BEC01F00101FB
:101F80002C2D01D08088CFC0F5F1CEC0F4F1F76BD5
:101F9000580EF66F0001D1EC02F002C07FF101C0D3
:101FA0007EF14750320803E18BEC01F002D0F4ECF3
:101FB00002F00101F32BF32D01D0B7D7F351030841
:101FC000B4E02C50CA081AE12B2D18D0375316E173
:101FD0000001B5EC05F04750320806E1040E01019E
:101FE0007F6F7E0E7E6F05D0040E01017F6F780E2D
:101FF0007E6F00018BEC01F017D00101CFC0F5F12D
:10200000CEC0F4F1F76B7E0EF66F0001D1EC02F05A
:1020100002C07FF101C07EF1F4EC02F0F4EC02F0BA
:10202000F4EC02F0F4EC02F00101F3510208D8B430
:102030007CD73D51020808E080987F6BFA0E7E6FD6
:1020400000018BEC01F001013D51020802E15E53F9
:10205000D8B42C6B2C53D8B481907F6BC80E7E6F94
:1020600000018BEC01F02C50CA080FE12C50CA087B
:1020700023E101013A2D03D0000107D001013B2DDE
:1020800001D002D0000118D00001839C01017F6BB8
:10209000C80E7E6F00018BEC01F02C50CA080CE1D9
:1020A00001013A2D01D005D03B2D01D002D0000115
:1020B00003D081968098000101013D51020802E1A0
:1020C0005E53D8B480983C51020803E02E53D8B434
:1020D00081960001CFEC02F001012F6B306B2C2DAB
:1020E00001D082902C50CA0806E100012CEC03F0CC
:1020F000010EC56F01012E5308E12F5306E1305345
:1021000004E15B510608D8A45B6B486A0001000C2F
:1021100001013C53D8B4DBD130B0D9D130B2D7D1E2
:102120003153D8A4D4D13653D8A4D1D12E2DC4D173
:10213000010E486E9D90A0928198819A8380828042
:102140002C50CA080CE13A530AE13B5308E13C51D8
:10215000020805E15E2D03D02B2D01D09FD184B262
:1021600080882C50CA0804E10001A1EC01F00101B3
:102170008186000102EC00F001017F6B1E0E7E6F74
:1021800000018BEC01F0838C010E01017F6F2C0E9E
:102190007E6F00018BEC01F022EC02F066EC01F0A6
:1021A00001016551000801E230D14551030805E104
:1021B0002B2D03D05E2D01D06ED081967F6BFA0E51
:1021C0007E6F00018BEC01F081882C50CA0802E17F
:1021D000A1EC01F0050E01017F6FDC0E7E6F0001A6
:1021E0008BEC01F02C50CA0802E1A1EC01F0050EC5
:1021F00001017F6FDC0E7E6F00018BEC01F02C5033
:10220000CA0802E1A1EC01F0050E01017F6FDC0EAE
:102210007E6F00018BEC01F02C50CA0802E1A1ECAA
:1022200001F0050E01017F6FDC0E7E6F00018BEC6B
:1022300001F02C50CA0802E1A1EC01F0050E0101E9
:102240007F6FDC0E7E6F00018BEC01F02C50CA0812
:1022500002E1A1EC01F0030E01017F6FE80E7E6F39
:1022600000018BEC01F0819801017F6B140E7E6FF1
:1022700000018BEC01F066EC01F0010165510008F2
:1022800001E2C3D03C51020805E12B2D03D05E2DA5
:1022900001D08186BAD02C50CA080FE12C2D0DD068
:1022A00038530BE10001A1EC01F0040E01017F6F36
:1022B0007E0E7E6F00018BEC01F0000166EC01F0F8
:1022C000CE5304E1CF5302E101019FD0CFC0F5F11D
:1022D000CEC0F4F1010E0101F76F180EF66F000188
:1022E000D1EC02F002C07FF101C07EF1475032080C
:1022F00003E18BEC01F002D0F4EC02F00101F36B8E
:10230000819681887F6B0A0E7E6F00018BEC01F055
:10231000819866EC01F001016551000801E275D079
:102320008188CFC0F5F1CEC0F4F1010EF76F180E21
:10233000F66F0001D1EC02F002C07FF101C07EF126
:102340008BEC01F0819801017F6B140E7E6F000110
:102350008BEC01F001012B2D01D08186CFC0F5F16E
:10236000CEC0F4F1F76B580EF66F0001D1EC02F01D
:1023700002C07FF101C07EF14750320803E18BECCF
:1023800001F002D0F4EC02F00101F32BF32D01D0A7
:10239000B7D7F3510308B4E02C50CA0811E12C2D33
:1023A0000FD038530DE10001A1EC01F0040E010142
:1023B0007F6F7E0E7E6F00018BEC01F017D0010164
:1023C000CFC0F5F1CEC0F4F1F76B7E0EF66F0001D1
:1023D000D1EC02F002C07FF101C07EF1F4EC02F01A
:1023E000F4EC02F0F4EC02F0F4EC02F00101F35131
:1023F000020886E03C51020808E081967F6BFA0EE5
:102400007E6F00018BEC01F001013C51020802E1FA
:102410005E53D8B42B6B2B53D8B4839E7F6BC80EFE
:102420007E6F00018BEC01F02C50CA080FE12C509C
:10243000CA0823E101013A2D03D0000107D00101B0
:102440003B2D01D002D0000118D00001839C010176
:102450007F6BC80E7E6F00018BEC01F02C50CA0818
:102460000CE101013A2D01D005D03B2D01D002D065
:10247000000103D081968098000101013C510208BF
:1024800002E15E53D8B481963D51020803E02F5318
:10249000D8B480980001CFEC02F001012E6B306BB4
:1024A0002B2D01D083902C50CA0806E100012CECA2
:1024B00003F0010EC56F01012E5308E12F5306E111
:1024C000305304E15B510608D8A45B6B486A0001F5
:1024D000000C01013C5303E13D53D8B4B6D130B0F8
:1024E000B4D130B2B2D13153D8A4AFD13253D8A481
:1024F000ACD13353D8A4A9D13553D8A4A6D13653DF
:10250000D8A4A3D1302D01D004D02E2D8FD12F2DC2
:102510008DD130A004D0000110DC87D1010130A2A0
:1025200004D00001F5DD81D1010130A005D030A239
:1025300003D000017AD101012C50CA0810E12B53BD
:1025400003E12C5301E10BD02B5303E10001E0DD4B
:1025500001012C5304E100019DEC0EF00101010E7C
:10256000486E9D90A0928198819A83808280545376
:1025700004E1755302E184B48186555304E1765336
:1025800002E184B28088000102EC00F001017F6B5F
:102590001E0E7E6F00018BEC01F0838C010E010199
:1025A0007F6F2C0E7E6F00018BEC01F022EC02F0AD
:1025B00066EC01F001016551000801E200D14551CE
:1025C000030806E12B2D01D002D02C2D01D043D0E1
:1025D000819680987F6BFA0E7E6F00018BEC01F084
:1025E0000101545305E1755303E13C53D8A481889C
:1025F000555305E1765303E13D53D8A4818A270E54
:102600007F6F100E7E6F00018BEC01F08198819A34
:1026100001017F6B140E7E6F00018BEC01F066EC04
:1026200001F001016551000801E2C9D0545308E1ED
:10263000755306E13C51020803E12B2D01D0818640
:10264000555308E1765306E13D51020803E12C2D74
:1026500001D08088B4D02C50CA0806E00001CE53C7
:1026600004E1CF5302E10101AAD0CFC0F5F1CEC001
:10267000F4F1010E0101F76F180EF66F0001D1ECB5
:1026800002F002C07FF101C07EF18BEC01F001018C
:10269000F36B819680988188818A7F6B0A0E7E6FAA
:1026A00000018BEC01F08198819A66EC01F0010148
:1026B0006551000801E283D0545305E1755303E1ED
:1026C0003C53D8A48188555305E1765303E13D532B
:1026D000D8A4818ACFC0F5F1CEC0F4F1010EF76F16
:1026E000180EF66F0001D1EC02F002C07FF101C0BC
:1026F0007EF18BEC01F08198819A01017F6B140EC1
:102700007E6F00018BEC01F00101545307E175531A
:1027100005E13C5303E02B2D01D08186555307E1A1
:10272000765305E13D5303E02C2D01D08088CFC0C6
:10273000F5F1CEC0F4F1F76B580EF66F0001D1EC55
:1027400002F002C07FF101C07EF14750320803E180
:102750008BEC01F002D0F4EC02F00101F32BF32D2D
:1027600001D097D7F351030894E0CFC0F5F1CEC064
:10277000F4F1F76B7E0EF66F0001D1EC02F002C0AF
:102780007FF101C07EF1F4EC02F0F4EC02F0F4EC25
:1027900002F0F4EC02F00101F3510208D8B479D749
:1027A0003C510208D8A481963D510208D8A48098D3
:1027B0007F6BC80E7E6F00018BEC01F001013C5174
:1027C0000208D8A42B6B3D510208D8A42C6B2B53C4
:1027D000D8B4839E2C53D8B481907F6BC80E7E6F83
:1027E00000018BEC01F02C50CA0808E0839C010129
:1027F0007F6BC80E7E6F00018BEC01F001013C5134
:102800000208D8A481963D510208D8A480982E6B66
:102810002F6B306B2B2D01D083902C2D01D082900B
:1028200000012CEC03F0010EC56F01010001CFEC9B
:1028300002F001012E5308E12F5306E1305304E169
:102840005B510608D8A45B6B486A0001000C0101CB
:10285000076B2B2D01D007812C2D01D007832D2D47
:1028600001D00785000180EF14F00101716B7F6BCF
:10287000050E7E6F00018BEC01F00101712B71518F
:10288000F90803E2010E376F03D084A4F0D7376B49
:10289000716B0001000C0101726B7F6B050E7E6F86
:1028A00000018BEC01F00101722B7251F90803E277
:1028B000010E386F03D084A2F0D7386B726B000121
:1028C000000CEF510408D8B08FD101013353D8B4B4
:1028D00002D0000189D13453D8B402D0000184D190
:1028E00030A002D0000180D130A202D000017CD102
:1028F000010E486EA0928198819A5B6B0001A7D768
:102900008380828083828286010E0101346F376B5F
:10291000386B0001C86BC96B0101656B0C6B0B6BED
:102920007F6B0A0E7E6F00018BEC01F001010B2B17
:10293000D8B40C2B0C5303E10B511308D8A065D06D
:1029400082AAEED70C6B0B6B0C6B0B6B7F6B0A0EBA
:102950007E6F00018BEC01F001010B2BD8B40C2B26
:1029600082AA05D00C5303E10B511408EFE284B4A2
:1029700002D084A24AD03C5302E0819881863D5324
:1029800002E0819A8088000102EC00F001017F6B77
:10299000320E7E6F00018BEC01F0838C010E010181
:1029A0007F6FF40E7E6F00018BEC01F0CFEC02F034
:1029B00001013C53D8A481963D53D8A48098010EC0
:1029C0007F6FF40E7E6F00018BEC01F001013C5330
:1029D000D8A481883D53D8A4818A030E7F6FE80E66
:1029E0007E6F00018BEC01F08198819A030E01014A
:1029F0007F6FE80E7E6F00018BEC01F001012E6B02
:102A00002F6B306B2B6B2C6B2D6B675307E1130E09
:102A10007F6F880E7E6F00018BEC01F0000102ECED
:102A200000F001017F6B320E7E6F00018BEC01F034
:102A3000838C81968098030E01017F6FE80E7E6F74
:102A400000018BEC01F08388030E01017F6FE80E1B
:102A50007E6F00018BEC01F0838A030E01017F6F12
:102A6000E80E7E6F00018BEC01F001013C5303E0A6
:102A70006B53D8B4838E3D5303E06C53D8B481803C
:102A8000030E7F6FE80E7E6F00018BEC01F00101F9
:102A90000C6B0B6B7F6B0A0E7E6F00018BEC01F0F1
:102AA00001010B2BD8B40C2B0C5303E10B5118086C
:102AB000D8A006D082AAEED70C6B0B6B82BAFED7D9
:102AC0003C5303E06B53D8B481863D530BE06C5309
:102AD00009E1010E7F6F900E7E6F00018BEC01F01B
:102AE000808801010F0E7F6FA00E7E6F00018BECBE
:102AF00001F0CFEC02F001013C5305E06B5303E120
:102B00000001B3DE01013D5305E06C5303E1000118
:102B1000C2DE0101372D01D002D0382D2DD03C531B
:102B200009E06B5307E1372D05D08196010E0001B6
:102B3000C86F01013D5309E06C5307E1382D05D002
:102B40008098010E0001C96F01017F6B640E7E6FDA
:102B500000018BEC01F001013C5306E06B5304E1F2
:102B6000372D02D0839E83923D5306E06C5304E1DF
:102B7000382D02D081908296839C010E7F6FF40ED7
:102B80007E6F00018BEC01F001013C5307E06B53B9
:102B900005E1375303E1010E316F83903D5307E0A8
:102BA0006C5305E1385303E1010E326F8290010E40
:102BB000336F6D6F2E6B2F6B306B476B416B426BBE
:102BC000436B446B5B6B2B6B2C6B2D6B586B576B98
:102BD0000001C82D03D00101376B0001C92D03D0BE
:102BE0000101386B00010000000CEF510408D8B05F
:102BF0007ED084B47CD001013C53D8A402D0000123
:102C000076D030A002D0000172D030A202D00001F4
:102C10006ED0010E486EA0928198819A84B280880D
:102C2000396B376B0001C86B02EC00F001017F6B60
:102C30001E0E7E6F00018BEC01F0838C81968388E1
:102C4000010E01017F6F2C0E7E6F00018BEC01F0F5
:102C5000838A010E01017F6F2C0E7E6F00018BECC9
:102C600001F0838E010E01017F6F2C0E7E6F00013B
:102C70008BEC01F081860F0E01017F6FA00E7E6F3D
:102C800000018BEC01F0CFEC02F0EFDD0101372DFC
:102C90000CD081967F6B640E7E6F00018BEC01F08F
:102CA000839E8392010EC86F0101839C7F6BC80EC7
:102CB0007E6F00018BEC01F00101375302E1010E40
:102CC000316F0001C82D02D00101376B0101312D98
:102CD0000DD0322D01D007D00001C92D01D002D076
:102CE000010104D00101010E336F6D6F396B0001DA
:102CF00051EF42F02C50CA080BE101013A2D01D0EE
:102D000005D03B2D01D002D0000102D09CD00001A3
:102D1000EF510408D8B098D001015453D8B402D070
:102D2000000192D07553D8B402D000018DD03C512F
:102D30000208D8B402D0000187D030A002D0000130
:102D400083D030A202D000017FD03153D8A47BD0F1
:102D50002B53D8A478D065510208D8B474D0656BD1
:102D60002E2D0AD0376B00010AEC03F00101375316
:102D700002E1010E2B6F67D084B465D0010E486E5E
:102D8000A0928198819A84B28088396B376B000158
:102D900002EC00F001017F6B1E0E7E6F00018BECD8
:102DA00001F0838C010E01017F6F2C0E7E6F0001FC
:102DB0008BEC01F0838E010E01017F6F2C0E7E6F74
:102DC00000018BEC01F066EC01F001016551000897
:102DD00001E20FD081860F0E7F6FA00E7E6F000183
:102DE0008BEC01F0CFEC02F00AEC03F00101372D7F
:102DF00011D081967F6B640E7E6F00018BEC01F029
:102E0000839E01017F6BC80E7E6F00018BEC01F089
:102E1000839201012C50CA080AE0839C7F6BFA0E52
:102E20007E6F00018BEC01F0819680980101375391
:102E300008E1655306E1010E2B6F2C2D02D0010E27
:102E40002D6F396B486A00010000000CEF51040837
:102E5000D8B07ED084B27CD001013D53D8A402D03A
:102E6000000176D030A002D0000172D030A202D092
:102E700000016ED0010E486EA0928198819A84B4B0
:102E80008186396B386B0001C96B02EC00F00101DF
:102E90007F6B1E0E7E6F00018BEC01F0838C80989F
:102EA0008388010E01017F6F2C0E7E6F00018BEC79
:102EB00001F0838A010E01017F6F2C0E7E6F0001ED
:102EC0008BEC01F08180010E01017F6F2C0E7E6F73
:102ED00000018BEC01F080880F0E01017F6FA00EC6
:102EE0007E6F00018BEC01F0CFEC02F0D4DC01012D
:102EF000382D0CD080987F6B640E7E6F00018BECB8
:102F000001F081908296010EC86F0101839C7F6B56
:102F1000C80E7E6F00018BEC01F00101385302E115
:102F2000010E326F0001C92D02D00101386B010181
:102F3000322D0DD0312D01D007D00001C82D01D088
:102F400002D0010104D00101010E336F6D6F396BA6
:102F5000000181EF42F02C50CA080BE101013A2D2B
:102F600001D005D03B2D01D002D0000102D0A0D06D
:102F70000001EF510408D8B09CD001015553D8B4DA
:102F800002D0000196D07653D8B402D0000191D07F
:102F90003D510208D8B402D000018BD030A002D03D
:102FA000000187D030A202D0000183D03253D8A4D0
:102FB0007FD02C53D8A47CD065510208D8B478D0E7
:102FC000656B2F2D0AD0386B00012AEC06F0010149
:102FD000385302E1010E2C6F6BD084B269D0010E20
:102FE000486EA0928198819A84B48186396B386B3F
:102FF000000102EC00F001017F6B1E0E7E6F0001EC
:103000008BEC01F0838C010E01017F6F2C0E7E6F23
:1030100000018BEC01F08180010E01017F6F2C0E0D
:103020007E6F00018BEC01F066EC01F0010165514F
:10303000000801E213D080880F0E7F6FA00E7E6F14
:1030400000018BEC01F0CFEC02F00101655304E1CB
:1030500000012AEC06F00101382D11D080987F6B19
:10306000640E7E6F00018BEC01F0819001017F6B9B
:10307000C80E7E6F00018BEC01F0829601012C508E
:10308000CA080AE0839C7F6BFA0E7E6F00018BEC0E
:1030900001F0809881960101385308E1655306E1FB
:1030A000010E2C6F2B2D02D0010E2D6F396B486A4B
:1030B00000010000000C0101876B322D01D002D00D
:1030C00084A26FD030B06DD030B26BD08098819236
:1030D00084B481947F6B320E7E6F00018BEC01F023
:1030E000839801017F6BC80E7E6F00018BEC01F0AD
:1030F000818201017F6B640E7E6F00018BEC01F019
:10310000818A01017F6BC80E7E6F00018BEC01F09C
:10311000819001017F6BC80E7E6F00018BEC01F086
:10312000819A01017F6BC80E7E6F00018BEC01F06C
:103130000101312D0DD0000102EC00F001017F6B87
:103140001E0E7E6F00018BEC01F0838802D001011E
:10315000839A01017F6BC80E7E6F00018BEC01F03A
:1031600081840101326B2C6B2F6B2B5303E12C53A9
:10317000D8B42D6B2E5303E12F53D8B4306B315399
:103180000BE1325309E1336B839A6D5301E1566BC6
:10319000010E516F2D0E506F0001CFEC02F0486A06
:1031A00001010001000C0101866B312D01D002D01C
:1031B00084A46FD030B06DD030B26BD08196819442
:1031C00084B281927F6B320E7E6F00018BEC01F036
:1031D000839801017F6BC80E7E6F00018BEC01F0BC
:1031E000818401017F6B640E7E6F00018BEC01F026
:1031F000818801017F6BC80E7E6F00018BEC01F0AE
:10320000839E01017F6BC80E7E6F00018BEC01F085
:10321000819801017F6BC80E7E6F00018BEC01F07D
:103220000101322D0DD0000102EC00F001017F6B95
:103230001E0E7E6F00018BEC01F0838802D001012D
:10324000839A01017F6BC80E7E6F00018BEC01F049
:1032500081820101316B2B6B2E6B2B5303E12C53BD
:10326000D8B42D6B2E5303E12F53D8B4306B3153A8
:103270000BE1325309E1336B839A6D5301E1566BD5
:10328000010E516F2D0E506F0001CFEC02F0486A15
:1032900001010001000C0101866B876B332D01D009
:1032A00007D0352D01D004D084B402D084A26ED0D2
:1032B00030B06CD030B26AD030A004D00001FBDE58
:1032C00063D0010130A203D000016DDF5DD00001A9
:1032D00002EC00F0809881968194819201017F6BCD
:1032E000640E7E6F00018BEC01F08398010E0101EA
:1032F0007F6F2C0E7E6F00018BEC01F08184819634
:103300008182809801017F6B640E7E6F00018BECDF
:1033100001F08188818A01017F6BC80E7E6F0001F8
:103320008BEC01F0839E819001017F6BC80E7E6F54
:1033300000018BEC01F0839A01017F6BC80E7E6F58
:1033400000018BEC01F00101316B326B336B2E6BA2
:103350002F6B306B476B6D53D8B4566B050E7F6F78
:10336000140E7E6F00018BEC01F08198819A010EA2
:103370000101516F2D0E506F0001CFEC02F02CECCB
:1033800003F0010EC56F486A000001010001000C46
:1033900001013D51020802E02F5266E030B264D0D4
:1033A0002F5362E1325360E135535EE136535CE105
:1033B0002C2D5AD0010E486EA0928198819A84B427
:1033C00081868088000102EC00F001017F6B1E0EF7
:1033D0007E6F00018BEC01F0838C010E01017F6F89
:1033E0002C0E7E6F00018BEC01F066EC01F08098F2
:1033F00001017F6BFA0E7E6F00018BEC01F0CFECC8
:1034000002F00101655309E1818A070E7F6FD00E3A
:103410007E6F00018BEC01F0010181907F6BFA0E51
:103420007E6F00018BEC01F02C50CA0809E0839CF0
:1034300001017F6BFA0E7E6F00018BEC01F081962B
:1034400001012C6B655308E1030E7F6FE80E7E6F60
:1034500000018BEC01F00101819A00012CEC03F0DA
:10346000010EC56F486A01010001000C01013C51C9
:10347000020802E02F5266E030B064D02E5362E1C1
:10348000315360E135535EE136535CE12B2D5AD068
:10349000010E486EA0928198819A84B280888186BC
:1034A000000102EC00F001017F6B1E0E7E6F000137
:1034B0008BEC01F0838C010E01017F6F2C0E7E6F6F
:1034C00000018BEC01F066EC01F0819601017F6B4D
:1034D000FA0E7E6F00018BEC01F0CFEC02F00101DF
:1034E000655309E18188070E7F6FD00E7E6F000162
:1034F0008BEC01F00101839E7F6BFA0E7E6F000161
:103500008BEC01F02C50CA0809E0839C01017F6B11
:10351000FA0E7E6F00018BEC01F0809801012B6B9D
:10352000655308E1030E7F6FE80E7E6F00018BECA0
:1035300001F00101819800012CEC03F0010EC56F30
:10354000486A01010001000C0101866B876B372D71
:1035500003D00001C86B0101382D03D00001C96BF5
:10356000010184B402D084A2E0D030A005D02F6B3A
:1035700000010EDFDAD0010130A205D02E6B000170
:1035800075DFD3D0010130A005D030A203D00001F7
:10359000CCD001013153D8A4C8D03253D8A4C5D05F
:1035A0003553D8A4C2D03653D8A4BFD02E2D01D0C5
:1035B00005D02F2D01D002D0302D55D0010E486EF0
:1035C000A0928198819A81868088000102EC00F0A7
:1035D00001017F6B1E0E7E6F00018BEC01F0838C6E
:1035E000010E01017F6F2C0E7E6F00018BEC01F04C
:1035F00066EC01F08196809801017F6BFA0E7E6F78
:1036000000018BEC01F0CFEC02F00101655316E1F3
:10361000545305E1755303E13C53D8A481885553B5
:1036200005E1765303E13D53D8A4818A070E7F6FED
:10363000D00E7E6F00018BEC01F00101839E819022
:10364000010E7F6F2C0E7E6F00018BEC01F0839CCE
:103650008198819A01012E6B2F6B306B476B5B6BEE
:10366000000163D0010184B404D084B202D02D6B78
:103670005CD02B2D01D005D02C2D01D002D02D2DCA
:1036800054D0010E486EA0928198819A81868088DC
:10369000000102EC00F001017F6B1E0E7E6F000145
:1036A0008BEC01F0838C010E01017F6F2C0E7E6F7D
:1036B00000018BEC01F066EC01F081968098010E20
:1036C00001017F6F2C0E7E6F00018BEC01F0CFECBF
:1036D00002F0010165530AE18188818A070E7F6F3C
:1036E000D00E7E6F00018BEC01F00101839E819072
:1036F0007F6BFA0E7E6F00018BEC01F0839C010161
:103700007F6BFA0E7E6F00018BEC01F08196809842
:103710000101655308E1030E7F6FE80E7E6F000123
:103720008BEC01F001018198819A01012B6B2C6BCC
:103730002D6B355303E12E6B2F6B306B5D6B486A3D
:103740000001000C0101666B6E6B280E6A6F3D0E66
:10375000006E002EFED7662B6E2B82AA06D06E510D
:10376000130803E2180E6A6F02D0280E6A6F6651C2
:10377000FE0803E36A512808EAE00001000C010199
:10378000251F25512419266F251F00016CEF21F0FC
:103790001DC1ADFFACA2FED7000C01012251B8083B
:1037A0000FE02251C8080CE02251190809E022510B
:1037B000290806E02251180803E02251280802E1F6
:1037C00065EF21F02A0E006E002EFED700D02251A8
:1037D0004A0814E12351F90811E1010E7B6F5B5196
:1037E00005080AE12C50CA0804E13A5305E13B53AD
:1037F00003E15BEF21F002D060EF21F022514A0893
:103800000DE1235108080AE1010E7B6F5B510608A8
:1038100003E15BEF21F002D060EF21F02251B90803
:1038200045E12351080842E1010E7B6FF2CF20F2FF
:10383000F29CF29EAA6AFF0EA96EA69CA69EA68086
:10384000A850020120BDF28C20BFF28E01011D6F35
:103850000001BA6BEF51050803E0EF51030823E1C3
:10386000060EEF6F01015C51F1081CE1702D0AD0CA
:10387000130E7F6F880E7E6F00018BEC01F061EC00
:1038800014F00FD000015EDF01016A5118080AE14F
:10389000130E7F6F880E7E6F00018BEC01F0DFEC62
:1038A00008F00101000168EF21F001012251B9087F
:1038B0001AE12351F90817E1010E7B6FF2CF20F2D4
:1038C000F29CF29EAA6AA96AA69CA69EA680A8500F
:1038D000020120BDF28C20BFF28E01011D6F00019C
:1038E00068EF21F001012251C90808E1010E7B6F48
:1038F0003CC11DF1000168EF21F001016451020893
:103900000BE12251D90808E1010E7B6F3DC11DF189
:10391000000168EF21F001012251890808E1010E40
:103920007B6F80C01DF1000168EF21F00101225181
:10393000790808E1010E7B6F81C01DF1000168EF7D
:1039400021F00101645102080BE12251A90808E1AC
:10395000010E7B6F82C01DF1000168EF21F00101B3
:10396000645102080AE12251990807E1010E7B6FB8
:1039700083C01DF1000168EF21F00001EF5105083F
:1039800043E2010122510A08D8B402D000013CD020
:1039900030AE0BD03D50000805E2FF0A06E13C5076
:1039A0008F0803E32951180822E1010E7B6F612D76
:1039B00006D0280E1D6F000168EF21F001010851AB
:1039C000090807E108C11DF1838082808382828615
:1039D00009D02951180804E183928296020E2A6FB9
:1039E00029C11DF1000168EF21F00ED001013D5009
:1039F000010807E303E13C508F0803E33C2AD8B4F5
:103A00003D2A73EF21F0000101012251E9080AE18A
:103A1000010E7B6F100E1D6F1D3B1D87000168EFAF
:103A200021F001012251F9080AE1010E7B6F270EF6
:103A30001D6F1D3B1D87000168EF21F00101225120
:103A4000390814E12A51020803E1280E296F2A6B74
:103A5000010E7B6F752D01D002D0522D05D030B0F4
:103A600003D05BEF21F002D060EF21F02251490832
:103A70001AE12A51020803E1280E296F2A6B010E70
:103A80007B6F645102080DE1762D01D002D0532DD9
:103A900005D030B203D05BEF21F002D060EF21F00F
:103AA00002D065EF21F022515908D8A40FD2010E9F
:103AB0007B6F8051000807E28051030804E3010E88
:103AC0007D6E080E5D6F280E296F2A6B352D04D090
:103AD000010E0001BB6F0101356B2351080835E170
:103AE00030A006D0D80E1D6F000168EF21F0010153
:103AF000372D01D004D00001C82D06D00101F80EE9
:103B00001D6F000168EF21F001013A2D0AD07553B5
:103B100008E1525306E10A0E1D6F000168EF21F023
:103B20000101822D05D00B0E1D6F000168EF21F001
:103B30000001CB2D07D00B0E01011D6F0001CB6BD7
:103B400068EF21F0010165EF21F0233B239F232D36
:103B50000DD00001F2A105D0010160EF21F006D0E7
:103B60000001010ECB6F01015BEF21F02351020830
:103B70000DE10001F2A305D0010160EF21F006D0B4
:103B80000001010ECB6F01015BEF21F0235103080F
:103B90000DE10001F2A505D0010160EF21F006D092
:103BA0000001010ECB6F01015BEF21F023510408EE
:103BB0000DE10001F2A705D0010160EF21F006D070
:103BC0000001010ECB6F01015BEF21F023510508CD
:103BD0000DE10001F2A905D0010160EF21F006D04E
:103BE0000001010ECB6F01015BEF21F023510608AC
:103BF0000DE10001F2AB05D0010160EF21F006D02C
:103C00000001010ECB6F01015BEF21F0235107088A
:103C10000DE10001F2AD05D0010160EF21F006D009
:103C20000001010ECB6F01015BEF21F02351080869
:103C30000DE10001F2AF05D0010160EF21F006D0E7
:103C40000001010ECB6F01015BEF21F02351090848
:103C50000DE10001F3A105D0010160EF21F006D0D4
:103C60000001010ECB6F01015BEF21F023510A0827
:103C70000DE10001F3A305D0010160EF21F006D0B2
:103C80000001010ECB6F01015BEF21F023510B0806
:103C90000DE10001F3A505D0010160EF21F006D090
:103CA0000001010ECB6F01015BEF21F023510C08E5
:103CB0000DE10001F3A705D0010160EF21F006D06E
:103CC0000001010ECB6F01015BEF21F023510D08C4
:103CD0000DE10001F3A905D0010160EF21F006D04C
:103CE0000001010ECB6F01015BEF21F023510E08A3
:103CF0000DE10001F3AB05D0010160EF21F006D02A
:103D00000001010ECB6F01015BEF21F023510F0881
:103D10000BE10001F3AD04D00101D2D205D00001C6
:103D2000010ECB6F0101C7D2235110080BE1000136
:103D3000F3AF04D00101C4D205D00001010ECB6F56
:103D40000101B9D2235111080BE10001F4A104D003
:103D50000101B6D205D00001010ECB6F0101ABD23B
:103D6000235112080BE10001F4A304D00101A8D2F1
:103D700005D00001010ECB6F01019DD22351130824
:103D80000BE10001F4A504D001019AD205D0000195
:103D9000010ECB6F01018FD2235114080BE10001FA
:103DA000F4A704D001018CD205D00001010ECB6F25
:103DB000010181D2235115080BE10001F4A904D0BF
:103DC00001017ED205D00001010ECB6F010173D23B
:103DD000235116080BE10001F4AB04D0010170D2AD
:103DE00005D00001010ECB6F010165D223511708E8
:103DF0000BE10001F4AD04D0010162D205D0000155
:103E0000010ECB6F010157D2235118080BE10001BD
:103E1000F4AF04D0010154D205D00001010ECB6FE4
:103E2000010149D2235119080BE10001F5A104D089
:103E3000010146D205D00001010ECB6F01013BD23A
:103E400023511A080BE10001F5A304D0010138D277
:103E500005D00001010ECB6F01012DD223511B08AB
:103E60000BE10001F5A504D001012AD205D0000123
:103E7000010ECB6F01011FD223511C080BE1000181
:103E8000F5A704D001011CD205D00001010ECB6FB3
:103E9000010111D223511D080BE10001F5A904D045
:103EA00001010ED205D00001010ECB6F010103D23A
:103EB00023511E080BE10001F5AB04D0010100D233
:103EC00005D00001010ECB6F0101F5D12251690827
:103ED000D8A4F0D1010E7B6F8051000807E2805119
:103EE000030804E3010E7D6E080E5D6F280E296F36
:103EF0002A6B352D04D0010E0001BB6F0101356B1B
:103F0000642D01D0E2D1235108082FE130A205D061
:103F1000D80E1D6F0001DCD10101382D01D004D075
:103F20000001C92D05D00101F80E1D6F0001D0D18F
:103F300001013B2D09D0765307E1535305E10A0EE9
:103F40001D6F0001C5D10101822D04D00B0E1D6F24
:103F50000001BED10001CC2D06D00B0E01011D6F5A
:103F60000001CC6BB5D10101B0D1233B239F232DA0
:103F70000BD00001F6A104D00101A2D105D00001AF
:103F8000010ECC6F010197D1235102080BE1000112
:103F9000F6A304D0010194D105D00001010ECC6F2D
:103FA000010189D1235103080BE10001F6A504D0DA
:103FB000010186D105D00001010ECC6F01017BD13A
:103FC000235104080BE10001F6A704D0010178D1C8
:103FD00005D00001010ECC6F01016DD12351050800
:103FE0000BE10001F6A904D001016AD105D000015E
:103FF000010ECC6F01015FD1235106080BE10001D6
:10400000F6AB04D001015CD105D00001010ECC6FEC
:10401000010151D1235107080BE10001F6AD04D095
:1040200001014ED105D00001010ECC6F010143D139
:10403000235108080BE10001F6AF04D0010140D183
:1040400005D00001010ECC6F010135D123510908C3
:104050000BE10001F7A104D0010132D105D000012C
:10406000010ECC6F010127D123510A080BE1000199
:10407000F7A304D0010124D105D00001010ECC6FBB
:10408000010119D123510B080BE10001F7A504D060
:10409000010116D105D00001010ECC6F01010BD139
:1040A00023510C080BE10001F7A704D0010108D14E
:1040B00005D00001010ECC6F0101FDD023510D0888
:1040C0000BE10001F7A904D00101FAD005D00001ED
:1040D000010ECC6F0101EFD023510E080BE100015E
:1040E000F7AB04D00101ECD005D00001010ECC6F7C
:1040F0000101E1D023510F080BE10001F7AD04D01D
:104100000101DED005D00001010ECC6F0101D3D03A
:10411000235110080BE10001F7AF04D00101D0D00A
:1041200005D00001010ECC6F0101C5D0235111084B
:104130000BE10001F8A104D00101C2D005D00001BB
:10414000010ECC6F0101B7D0235112080BE1000121
:10415000F8A304D00101B4D005D00001010ECC6F4A
:104160000101A9D0235113080BE10001F8A504D0E7
:104170000101A6D005D00001010ECC6F01019BD03A
:10418000235114080BE10001F8A704D0010198D0D5
:1041900005D00001010ECC6F01018DD0235115080F
:1041A0000BE10001F8A904D001018AD005D000017B
:1041B000010ECC6F01017FD0235116080BE10001E5
:1041C000F8AB04D001017CD005D00001010ECC6F0A
:1041D000010171D0235117080BE10001F8AD04D0A3
:1041E00001016ED005D00001010ECC6F010163D03A
:1041F000235118080BE10001F8AF04D0010160D091
:1042000005D00001010ECC6F010155D023511908D2
:104210000BE10001F9A104D0010152D005D0000149
:10422000010ECC6F010147D023511A080BE10001A8
:10423000F9A304D0010144D005D00001010ECC6FD8
:10424000010139D023511B080BE10001F9A504D06D
:10425000010136D005D00001010ECC6F01012BD039
:1042600023511C080BE10001F9A704D0010128D05B
:1042700005D00001010ECC6F01011DD023511D0896
:104280000BE10001F9A904D001011AD005D0000109
:10429000010ECC6F01010FD023511E080BE100016C
:1042A000F9AB04D001010CD005D00001010ECC6F98
:1042B000010101D00AD0180E1D6F000109D00101C3
:1042C000280E1D6F000104D00101080E1D6F0001B2
:1042D0001DC125F1BFEF1BF0C8EC1BF026C11DF17D
:1042E000C8EC1BF00101000000010FEF43F0A092A9
:1042F00001012B2D02D0819881862C2D02D0819A2C
:1043000080888F918F95909190958C6B9F6BAA6A06
:10431000130EA96E9FC1A8FFA69CA69EA684F2CFED
:1043200000F0F29CF29E0F01550EA76EAA0EA76E2A
:10433000A682A6B2FED7A6940050F2120101A06B8D
:10434000AA6A140EA96EA0C1A8FFA69CA69EA68468
:10435000F2CF00F0F29CF29E0F01550EA76EAA0E4E
:10436000A76EA682A6B2FED7A6940050F212010153
:10437000A16BAA6A150EA96EA1C1A8FFA69CA69E54
:10438000A684F2CF00F0F29CF29E0F01550EA76EAC
:10439000AA0EA76EA682A6B2FED7A6940050F2126D
:1043A0000101A26BAA6A160EA96EA2C1A8FFA69C63
:1043B000A69EA684F2CF00F0F29CF29E0F01550E4D
:1043C000A76EAA0EA76EA682A6B2FED7A69400502C
:1043D000F2120101A36BAA6A170EA96EA3C1A8FF6E
:1043E000A69CA69EA684F2CF00F0F29CF29E0F013E
:1043F000550EA76EAA0EA76EA682A6B2FED7A694E9
:104400000050F2120101A46BAA6A180EA96EA4C191
:10441000A8FFA69CA69EA684F2CF00F0F29CF29E76
:104420000F01550EA76EAA0EA76EA682A6B2FED7E2
:10443000A6940050F2120101A56BAA6A230EA96E80
:10444000A5C1A8FFA69CA69EA684F2CF00F0F29C70
:10445000F29E0F01550EA76EAA0EA76EA682A6B2F7
:10446000FED7A6940050F2120101A66BAA6A240E90
:10447000A96EA6C1A8FFA69CA69EA684F2CF00F0B6
:10448000F29CF29E0F01550EA76EAA0EA76EA68291
:10449000A6B2FED7A6940050F2120101A76BAA6A39
:1044A000250EA96EA7C1A8FFA69CA69EA684F2CF42
:1044B00000F0F29CF29E0F01550EA76EAA0EA76E99
:1044C000A682A6B2FED7A6940050F2120101A86BF4
:1044D000AA6A260EA96EA8C1A8FFA69CA69EA684BD
:1044E000F2CF00F0F29CF29E0F01550EA76EAA0EBD
:1044F000A76EA682A6B2FED7A6940050F2120101C2
:10450000A96BAA6A270EA96EA9C1A8FFA69CA69EA0
:10451000A684F2CF00F0F29CF29E0F01550EA76E1A
:10452000AA0EA76EA682A6B2FED7A6940050F212DB
:104530000101AA6BAA6A280EA96EAAC1A8FFA69CAF
:10454000A69EA684F2CF00F0F29CF29E0F01550EBB
:10455000A76EAA0EA76EA682A6B2FED7A69400509A
:10456000F2120101B76BB86BB96BBA6BBB6BBC6B6A
:10457000CF6BD06BD16BD26BD36BD46B846B866BF0
:10458000886B8A6B0001C693AA6A330EA96EA86A6B
:10459000A69CA69EA684F2CF00F0F29CF29E0F018C
:1045A000550EA76EAA0EA76EA682A6B2FED7A69437
:1045B0000050F212AA6A340EA96EA86AA69CA69EA2
:1045C000A684F2CF00F0F29CF29E550EA76EAA0EC2
:1045D000A76EA682A6B2FED7A6940050F212AA6ACF
:1045E000350EA96EA86AA69CA69EA684F2CF00F0FE
:1045F000F29CF29E550EA76EAA0EA76EA682A6B2D8
:10460000FED7A6940050F212AA6A360EA96EA86AC6
:10461000A69CA69EA684F2CF00F0F29CF29E550EB8
:10462000A76EAA0EA76EA682A6B2FED7A6940050C9
:10463000F212AA6A370EA96EA86AA69CA69EA68444
:10464000F2CF00F0F29CF29E550EA76EAA0EA76E56
:10465000A682A6B2FED7A6940050F212AA6A380E1D
:10466000A96EA86AA69CA69EA684F2CF00F0F29C32
:10467000F29E550EA76EAA0EA76EA682A6B2FED710
:10468000A6940050F2120101A9EF50F0A09201018E
:104690002B2D02D0819881862C2D02D0819A808882
:1046A0008F938F97909390998D6BAB6BAA6A1A0E2C
:1046B000A96EABC1A8FFA69CA69EA684F2CF00F06F
:1046C000F29CF29E0F01550EA76EAA0EA76EA6824F
:1046D000A6B2FED7A6940050F2120101AC6BAA6AF2
:1046E0001B0EA96EACC1A8FFA69CA69EA684F2CF05
:1046F00000F0F29CF29E0F01550EA76EAA0EA76E57
:10470000A682A6B2FED7A6940050F2120101AD6BAC
:10471000AA6A1C0EA96EADC1A8FFA69CA69EA6847F
:10472000F2CF00F0F29CF29E0F01550EA76EAA0E7A
:10473000A76EA682A6B2FED7A6940050F21201017F
:10474000AE6BAA6A1D0EA96EAEC1A8FFA69CA69E5E
:10475000A684F2CF00F0F29CF29E0F01550EA76ED8
:10476000AA0EA76EA682A6B2FED7A6940050F21299
:104770000101AF6BAA6A1E0EA96EAFC1A8FFA69C6D
:10478000A69EA684F2CF00F0F29CF29E0F01550E79
:10479000A76EAA0EA76EA682A6B2FED7A694005058
:1047A000F2120101B06BAA6A1F0EA96EB0C1A8FF78
:1047B000A69CA69EA684F2CF00F0F29CF29E0F016A
:1047C000550EA76EAA0EA76EA682A6B2FED7A69415
:1047D0000050F2120101B16BAA6A2A0EA96EB1C192
:1047E000A8FFA69CA69EA684F2CF00F0F29CF29EA3
:1047F0000F01550EA76EAA0EA76EA682A6B2FED70F
:10480000A6940050F2120101B26BAA6A2B0EA96E97
:10481000B2C1A8FFA69CA69EA684F2CF00F0F29C8F
:10482000F29E0F01550EA76EAA0EA76EA682A6B223
:10483000FED7A6940050F2120101B36BAA6A2C0EA7
:10484000A96EB3C1A8FFA69CA69EA684F2CF00F0D5
:10485000F29CF29E0F01550EA76EAA0EA76EA682BD
:10486000A6B2FED7A6940050F2120101B46BAA6A58
:104870002D0EA96EB4C1A8FFA69CA69EA684F2CF59
:1048800000F0F29CF29E0F01550EA76EAA0EA76EC5
:10489000A682A6B2FED7A6940050F2120101B56B13
:1048A000AA6A2E0EA96EB5C1A8FFA69CA69EA684D4
:1048B000F2CF00F0F29CF29E0F01550EA76EAA0EE9
:1048C000A76EA682A6B2FED7A6940050F2120101EE
:1048D000B66BAA6A2F0EA96EB6C1A8FFA69CA69EAB
:1048E000A684F2CF00F0F29CF29E0F01550EA76E47
:1048F000AA0EA76EA682A6B2FED7A6940050F21208
:104900000101BD6BBE6BBF6BC06BC16BC26BD56B66
:10491000D66BD76BD86BD96BDA6B856B876B896B72
:104920008B6B0001C695AA6A3A0EA96EA86AA69C6E
:10493000A69EA684F2CF00F0F29CF29E0F01550EC7
:10494000A76EAA0EA76EA682A6B2FED7A6940050A6
:10495000F212AA6A3B0EA96EA86AA69CA69EA6841D
:10496000F2CF00F0F29CF29E550EA76EAA0EA76E33
:10497000A682A6B2FED7A6940050F212AA6A3C0EF6
:10498000A96EA86AA69CA69EA684F2CF00F0F29C0F
:10499000F29E550EA76EAA0EA76EA682A6B2FED7ED
:1049A000A6940050F212AA6A3D0EA96EA86AA69CAF
:1049B000A69EA684F2CF00F0F29CF29E550EA76E42
:1049C000AA0EA76EA682A6B2FED7A6940050F21237
:1049D000AA6A3E0EA96EA86AA69CA69EA684F2CFDD
:1049E00000F0F29CF29E550EA76EAA0EA76EA6824C
:1049F000A6B2FED7A6940050F212AA6A3F0EA96E84
:104A0000A86AA69CA69EA684F2CF00F0F29CF29E15
:104A1000550EA76EAA0EA76EA682A6B2FED7A694C2
:104A20000050F2120101A9EF50F0F16BF051010AB0
:104A30001FE0170A22E0010A25E0370A28E0010AF0
:104A40002BE0170A2EE0010A31E0770A34E0010A70
:104A500037E0170A3AE0010A3DE0370A40E0010A70
:104A600043E0170A46E0010A49E0F70A4CE050D05B
:104A700086B102D0010EF16F4BD086B302D0010E89
:104A8000F16F46D086B502D0010EF16F41D086B7E6
:104A900002D0010EF16F3CD086B902D0010EF16F49
:104AA00037D086BB02D0010EF16F32D086BD02D066
:104AB000010EF16F2DD086BF02D0010EF16F28D00C
:104AC00087B102D0010EF16F23D087B302D0010E5F
:104AD000F16F1ED087B502D0010EF16F19D087B7E4
:104AE00002D0010EF16F14D087B902D0010EF16F20
:104AF0000FD087BB02D0010EF16F0AD087BD02D064
:104B0000010EF16F05D087BF02D0010EF16F00D00A
:104B1000000CA09201012B2D02D0819881862C2DB2
:104B200002D0819A80882351070B926F922D03D077
:104B3000010E926F29D09251020803E1020E926F8A
:104B400023D09251030803E1040E926F1DD09251BD
:104B5000040803E1080E926F17D09251050803E193
:104B6000100E926F11D09251060803E1200E926F41
:104B70000BD09251070803E1400E926F05D092537B
:104B800003E1800E926F00D0233B23510F0B916FF6
:104B9000912D03D0010E916F59D09151020803E17C
:104BA000160E916F53D09151030803E1170E916FC8
:104BB0004DD09151040803E1200E916F47D09151DF
:104BC000050803E1210E916F41D09151060803E1E0
:104BD000360E916F3BD09151070803E1370E916F6C
:104BE00035D09151080803E1400E916F2FD09151BB
:104BF000090803E1410E916F29D091510A0803E1A0
:104C0000560E916F23D091510B0803E1570E916F0F
:104C10001DD091510C0803E1600E916F17D0915196
:104C20000D0803E1610E916F11D091510E0803E15F
:104C3000760E916F0BD091510F0803E1770E916FB3
:104C400005D0915303E1800E916F00D08C2B0001B1
:104C5000C683010E01018C5DFA0FD8B0B8EF2AF0BF
:104C6000060F0001EEEF2AF091C1F0F0DEDEF12D2B
:104C700004D00101B8EF2AF0000191C19FF192C167
:104C8000A5F101018FAB1AD0010ECF6FAA6A330EC6
:104C9000A96ECFC1A8FFA69CA69EA684F2CF00F065
:104CA000F29CF29E0F01550EA76EAA0EA76EA68269
:104CB000A6B2FED7A6940050F21201018FAD1AD011
:104CC000020ECF6FAA6A330EA96ECFC1A8FFA69CB1
:104CD000A69EA684F2CF00F0F29CF29E0F01550E24
:104CE000A76EAA0EA76EA682A6B2FED7A694005003
:104CF000F21201018FAF1AD0030ECF6FAA6A330EE2
:104D0000A96ECFC1A8FFA69CA69EA684F2CF00F0F4
:104D1000F29CF29E0F01550EA76EAA0EA76EA682F8
:104D2000A6B2FED7A6940050F212010190A71AD0A5
:104D3000040ECF6FAA6A330EA96ECFC1A8FFA69C3E
:104D4000A69EA684F2CF00F0F29CF29E0F01550EB3
:104D5000A76EAA0EA76EA682A6B2FED7A694005092
:104D6000F2120101AA6A130EA96E9FC1A8FFA69CA8
:104D7000A69EA684F2CF00F0F29CF29E0F01550E83
:104D8000A76EAA0EA76EA682A6B2FED7A694005062
:104D9000F212AA6A230EA96EA5C1A8FFA69CA69E20
:104DA000A684F2CF00F0F29CF29E550EA76EAA0EDA
:104DB000A76EA682A6B2FED7A6940050F2120101F9
:104DC000B8EF2AF091C1F0F030DEF12D03D00101EF
:104DD000B8EF2AF0010191519F5D06E19251A55D66
:104DE00003E18C07B5EF2AF091C1A0F192C1A6F1C1
:104DF0008FAB1AD0010ED06FAA6A340EA96ED0C143
:104E0000A8FFA69CA69EA684F2CF00F0F29CF29E7C
:104E10000F01550EA76EAA0EA76EA682A6B2FED7E8
:104E2000A6940050F21201018FAD1AD0020ED06F7D
:104E3000AA6A340EA96ED0C1A8FFA69CA69EA6841D
:104E4000F2CF00F0F29CF29E0F01550EA76EAA0E53
:104E5000A76EA682A6B2FED7A6940050F212010158
:104E60008FAF1AD0030ED06FAA6A340EA96ED0C1CC
:104E7000A8FFA69CA69EA684F2CF00F0F29CF29E0C
:104E80000F01550EA76EAA0EA76EA682A6B2FED778
:104E9000A6940050F212010190A71AD0040ED06F10
:104EA000AA6A340EA96ED0C1A8FFA69CA69EA684AD
:104EB000F2CF00F0F29CF29E0F01550EA76EAA0EE3
:104EC000A76EA682A6B2FED7A6940050F2120101E8
:104ED000AA6A140EA96EA0C1A8FFA69CA69EA684CD
:104EE000F2CF00F0F29CF29E0F01550EA76EAA0EB3
:104EF000A76EA682A6B2FED7A6940050F212AA6AA6
:104F0000240EA96EA6C1A8FFA69CA69EA684F2CFD9
:104F100000F0F29CF29E550EA76EAA0EA76EA68216
:104F2000A6B2FED7A6940050F212010121D391C17E
:104F3000F0F07BDDF12D02D001011AD30101915176
:104F40009F5D05E19251A55D02E18C070ED3915161
:104F5000A05D05E19251A65D02E18C0706D391C1E7
:104F6000A1F192C1A7F18FAB1AD0010ED16FAA6A3D
:104F7000350EA96ED1C1A8FFA69CA69EA684F2CF2D
:104F800000F0F29CF29E0F01550EA76EAA0EA76EBE
:104F9000A682A6B2FED7A6940050F21201018FADF0
:104FA0001AD0020ED16FAA6A350EA96ED1C1A8FF20
:104FB000A69CA69EA684F2CF00F0F29CF29E0F0162
:104FC000550EA76EAA0EA76EA682A6B2FED7A6940D
:104FD0000050F21201018FAF1AD0030ED16FAA6AEE
:104FE000350EA96ED1C1A8FFA69CA69EA684F2CFBD
:104FF00000F0F29CF29E0F01550EA76EAA0EA76E4E
:10500000A682A6B2FED7A6940050F212010190A784
:105010001AD0040ED16FAA6A350EA96ED1C1A8FFAD
:10502000A69CA69EA684F2CF00F0F29CF29E0F01F1
:10503000550EA76EAA0EA76EA682A6B2FED7A6949C
:105040000050F2120101AA6A150EA96EA1C1A8FFB3
:10505000A69CA69EA684F2CF00F0F29CF29E0F01C1
:10506000550EA76EAA0EA76EA682A6B2FED7A6946C
:105070000050F212AA6A250EA96EA7C1A8FFA69C2D
:10508000A69EA684F2CF00F0F29CF29E550EA76E6B
:10509000AA0EA76EA682A6B2FED7A6940050F21260
:1050A000010166D291C1F0F0C0DCF12D02D0010106
:1050B0005FD2010191519F5D05E19251A55D02E131
:1050C0008C0753D29151A05D05E19251A65D02E19A
:1050D0008C074BD29151A15D05E19251A75D02E190
:1050E0008C0743D291C1A2F192C1A8F18FAB1AD023
:1050F000010ED26FAA6A360EA96ED2C1A8FFA69C75
:10510000A69EA684F2CF00F0F29CF29E0F01550EEF
:10511000A76EAA0EA76EA682A6B2FED7A6940050CE
:10512000F21201018FAD1AD0020ED26FAA6A360EAA
:10513000A96ED2C1A8FFA69CA69EA684F2CF00F0BD
:10514000F29CF29E0F01550EA76EAA0EA76EA682C4
:10515000A6B2FED7A6940050F21201018FAF1AD06A
:10516000030ED26FAA6A360EA96ED2C1A8FFA69C02
:10517000A69EA684F2CF00F0F29CF29E0F01550E7F
:10518000A76EAA0EA76EA682A6B2FED7A69400505E
:10519000F212010190A71AD0040ED26FAA6A360E3D
:1051A000A96ED2C1A8FFA69CA69EA684F2CF00F04D
:1051B000F29CF29E0F01550EA76EAA0EA76EA68254
:1051C000A6B2FED7A6940050F2120101AA6A160EEA
:1051D000A96EA2C1A8FFA69CA69EA684F2CF00F04D
:1051E000F29CF29E0F01550EA76EAA0EA76EA68224
:1051F000A6B2FED7A6940050F212AA6A260EA96E95
:10520000A8C1A8FFA69CA69EA684F2CF00F0F29C9F
:10521000F29E550EA76EAA0EA76EA682A6B2FED764
:10522000A6940050F2120101A3D191C1F0F015EC47
:1052300025F0F12D02D001019BD1010191519F5D1B
:1052400005E19251A55D02E18C078FD19151A05DDE
:1052500005E19251A65D02E18C0787D19151A15DD4
:1052600005E19251A75D02E18C077FD19151A25DCA
:1052700005E19251A85D02E18C0777D191C1A3F1BC
:1052800092C1A9F18FAB1AD0010ED36FAA6A370E63
:10529000A96ED3C1A8FFA69CA69EA684F2CF00F05B
:1052A000F29CF29E0F01550EA76EAA0EA76EA68263
:1052B000A6B2FED7A6940050F21201018FAD1AD00B
:1052C000020ED36FAA6A370EA96ED3C1A8FFA69C9F
:1052D000A69EA684F2CF00F0F29CF29E0F01550E1E
:1052E000A76EAA0EA76EA682A6B2FED7A6940050FD
:1052F000F21201018FAF1AD0030ED36FAA6A370ED4
:10530000A96ED3C1A8FFA69CA69EA684F2CF00F0EA
:10531000F29CF29E0F01550EA76EAA0EA76EA682F2
:10532000A6B2FED7A6940050F212010190A71AD09F
:10533000040ED36FAA6A370EA96ED3C1A8FFA69C2C
:10534000A69EA684F2CF00F0F29CF29E0F01550EAD
:10535000A76EAA0EA76EA682A6B2FED7A69400508C
:10536000F2120101AA6A170EA96EA3C1A8FFA69C9A
:10537000A69EA684F2CF00F0F29CF29E0F01550E7D
:10538000A76EAA0EA76EA682A6B2FED7A69400505C
:10539000F212AA6A270EA96EA9C1A8FFA69CA69E12
:1053A000A684F2CF00F0F29CF29E550EA76EAA0ED4
:1053B000A76EA682A6B2FED7A6940050F2120101F3
:1053C000D7D091C1F0F015EC25F0F12D02D00101FC
:1053D000CFD0010191519F5D05E19251A55D02E1A0
:1053E0008C07C3D09151A05D05E19251A65D02E109
:1053F0008C07BBD09151A15D05E19251A75D02E1FF
:105400008C07B3D09151A25D05E19251A85D02E1F4
:105410008C07ABD09151A35D05E19251A95D02E1EA
:105420008C07A3D091C1A4F192C1AAF18FAB1AD07D
:10543000010ED46FAA6A380EA96ED4C1A8FFA69C2B
:10544000A69EA684F2CF00F0F29CF29E0F01550EAC
:10545000A76EAA0EA76EA682A6B2FED7A69400508B
:10546000F21201018FAD1AD0020ED46FAA6A380E63
:10547000A96ED4C1A8FFA69CA69EA684F2CF00F078
:10548000F29CF29E0F01550EA76EAA0EA76EA68281
:10549000A6B2FED7A6940050F21201018FAF1AD027
:1054A000030ED46FAA6A380EA96ED4C1A8FFA69CB9
:1054B000A69EA684F2CF00F0F29CF29E0F01550E3C
:1054C000A76EAA0EA76EA682A6B2FED7A69400501B
:1054D000F212010190A71AD0040ED46FAA6A380EF6
:1054E000A96ED4C1A8FFA69CA69EA684F2CF00F008
:1054F000F29CF29E0F01550EA76EAA0EA76EA68211
:10550000A6B2FED7A6940050F2120101AA6A180EA4
:10551000A96EA4C1A8FFA69CA69EA684F2CF00F007
:10552000F29CF29E0F01550EA76EAA0EA76EA682E0
:10553000A6B2FED7A6940050F212AA6A280EA96E4F
:10554000AAC1A8FFA69CA69EA684F2CF00F0F29C5A
:10555000F29E550EA76EAA0EA76EA682A6B2FED721
:10556000A6940050F212010103D00C6B0B6B0101E9
:105570008F9B8F9D8F9F9097AA6A200EA96E8FC1D7
:10558000A8FFA69CA69EA684F2CF00F0F29CF29EF5
:105590000F01550EA76EAA0EA76EA682A6B2FED761
:1055A000A6940050F212AA6A210EA96E90C1A8FF1B
:1055B000A69CA69EA684F2CF00F0F29CF29E550E09
:1055C000A76EAA0EA76EA682A6B2FED7A69400501A
:1055D000F2120101916B926B0001000CE824F76A52
:1055E000F736F70FF66E550EF7220A00F550FA6EF1
:1055F0000800F550F96E684CC44D2E4FA4502A5245
:10560000C25301018F818F8B000189EC25F040EF9F
:1056100043F0A09201012B2D02D0819881862C2D80
:1056200002D0819A80882351070B946F942D03D068
:10563000010E946F29D09451020803E1020E946F79
:1056400023D09451030803E1040E946F1DD09451AC
:10565000040803E1080E946F17D09451050803E184
:10566000100E946F11D09451060803E1200E946F30
:105670000BD09451070803E1400E946F05D094536A
:1056800003E1800E946F00D0233B23510F0B936FE7
:10569000932D03D0010E936F59D09351020803E16B
:1056A000160E936F53D09351030803E1170E936FB7
:1056B0004DD09351040803E1200E936F47D09351CE
:1056C000050803E1210E936F41D09351060803E1D1
:1056D000360E936F3BD09351070803E1370E936F5B
:1056E00035D09351080803E1400E936F2FD09351AA
:1056F000090803E1410E936F29D093510A0803E191
:10570000560E936F23D093510B0803E1570E936FFE
:105710001DD093510C0803E1600E936F17D0935185
:105720000D0803E1610E936F11D093510E0803E150
:10573000760E936F0BD093510F0803E1770E936FA2
:1057400005D0935303E1800E936F00D08D2B0001A1
:10575000C685010E01018D5DFA0FD8B03CEF30F027
:10576000060F000172EF30F093C1F0F015EC25F058
:10577000F12D04D001013CEF30F0000193C1ABF1F9
:1057800094C1B1F101018FAB1AD0010ED56FAA6A95
:105790003A0EA96ED5C1A8FFA69CA69EA684F2CFFC
:1057A00000F0F29CF29E0F01550EA76EAA0EA76E96
:1057B000A682A6B2FED7A6940050F21201018FADC8
:1057C0001AD0020ED56FAA6A3A0EA96ED5C1A8FFEB
:1057D000A69CA69EA684F2CF00F0F29CF29E0F013A
:1057E000550EA76EAA0EA76EA682A6B2FED7A694E5
:1057F0000050F21201018FAF1AD0030ED56FAA6AC2
:105800003A0EA96ED5C1A8FFA69CA69EA684F2CF8B
:1058100000F0F29CF29E0F01550EA76EAA0EA76E25
:10582000A682A6B2FED7A6940050F212010190AB58
:105830001AD0040ED56FAA6A3A0EA96ED5C1A8FF78
:10584000A69CA69EA684F2CF00F0F29CF29E0F01C9
:10585000550EA76EAA0EA76EA682A6B2FED7A69474
:105860000050F2120101AA6A1A0EA96EABC1A8FF7C
:10587000A69CA69EA684F2CF00F0F29CF29E0F0199
:10588000550EA76EAA0EA76EA682A6B2FED7A69444
:105890000050F212AA6A2A0EA96EB1C1A8FFA69CF6
:1058A000A69EA684F2CF00F0F29CF29E550EA76E43
:1058B000AA0EA76EA682A6B2FED7A6940050F21238
:1058C00001013CEF30F093C1F0F015EC25F0F12D23
:1058D00003D001013CEF30F001019351AB5D06E1D3
:1058E0009451B15D03E18D0739EF30F093C1ACF114
:1058F00094C1B2F18FAB1AD0010ED66FAA6A3B0EDB
:10590000A96ED6C1A8FFA69CA69EA684F2CF00F0E1
:10591000F29CF29E0F01550EA76EAA0EA76EA682EC
:10592000A6B2FED7A6940050F21201018FAD1AD094
:10593000020ED66FAA6A3B0EA96ED6C1A8FFA69C1E
:10594000A69EA684F2CF00F0F29CF29E0F01550EA7
:10595000A76EAA0EA76EA682A6B2FED7A694005086
:10596000F21201018FAF1AD0030ED66FAA6A3B0E56
:10597000A96ED6C1A8FFA69CA69EA684F2CF00F071
:10598000F29CF29E0F01550EA76EAA0EA76EA6827C
:10599000A6B2FED7A6940050F212010190AB1AD025
:1059A000040ED66FAA6A3B0EA96ED6C1A8FFA69CAC
:1059B000A69EA684F2CF00F0F29CF29E0F01550E37
:1059C000A76EAA0EA76EA682A6B2FED7A694005016
:1059D000F2120101AA6A1B0EA96EACC1A8FFA69C17
:1059E000A69EA684F2CF00F0F29CF29E0F01550E07
:1059F000A76EAA0EA76EA682A6B2FED7A6940050E6
:105A0000F212AA6A2B0EA96EB2C1A8FFA69CA69E8E
:105A1000A684F2CF00F0F29CF29E550EA76EAA0E5D
:105A2000A76EA682A6B2FED7A6940050F21201017C
:105A300023D393C1F0F015EC25F0F12D02D0010134
:105A40001BD301019351AB5D05E19451B15D02E1BE
:105A50008D070FD39351AC5D05E19451B25D02E126
:105A60008D0707D393C1ADF194C1B3F18FAB1AD0B9
:105A7000010ED76FAA6A3C0EA96ED7C1A8FFA69CDB
:105A8000A69EA684F2CF00F0F29CF29E0F01550E66
:105A9000A76EAA0EA76EA682A6B2FED7A694005045
:105AA000F21201018FAD1AD0020ED76FAA6A3C0E16
:105AB000A96ED7C1A8FFA69CA69EA684F2CF00F02F
:105AC000F29CF29E0F01550EA76EAA0EA76EA6823B
:105AD000A6B2FED7A6940050F21201018FAF1AD0E1
:105AE000030ED76FAA6A3C0EA96ED7C1A8FFA69C69
:105AF000A69EA684F2CF00F0F29CF29E0F01550EF6
:105B0000A76EAA0EA76EA682A6B2FED7A6940050D4
:105B1000F212010190AB1AD0040ED76FAA6A3C0EA4
:105B2000A96ED7C1A8FFA69CA69EA684F2CF00F0BE
:105B3000F29CF29E0F01550EA76EAA0EA76EA682CA
:105B4000A6B2FED7A6940050F2120101AA6A1C0E5A
:105B5000A96EADC1A8FFA69CA69EA684F2CF00F0B8
:105B6000F29CF29E0F01550EA76EAA0EA76EA6829A
:105B7000A6B2FED7A6940050F212AA6A2C0EA96E05
:105B8000B3C1A8FFA69CA69EA684F2CF00F0F29C0B
:105B9000F29E550EA76EAA0EA76EA682A6B2FED7DB
:105BA000A6940050F212010167D293C1F0F015ECF7
:105BB00025F0F12D02D001015FD201019351AB5DBF
:105BC00005E19451B15D02E18D0753D29351AC5D73
:105BD00005E19451B25D02E18D074BD29351AD5D69
:105BE00005E19451B35D02E18D0743D293C1AEF15B
:105BF00094C1B4F18FAB1AD0010ED86FAA6A3D0ED2
:105C0000A96ED8C1A8FFA69CA69EA684F2CF00F0DC
:105C1000F29CF29E0F01550EA76EAA0EA76EA682E9
:105C2000A6B2FED7A6940050F21201018FAD1AD091
:105C3000020ED86FAA6A3D0EA96ED8C1A8FFA69C15
:105C4000A69EA684F2CF00F0F29CF29E0F01550EA4
:105C5000A76EAA0EA76EA682A6B2FED7A694005083
:105C6000F21201018FAF1AD0030ED86FAA6A3D0E4F
:105C7000A96ED8C1A8FFA69CA69EA684F2CF00F06C
:105C8000F29CF29E0F01550EA76EAA0EA76EA68279
:105C9000A6B2FED7A6940050F212010190AB1AD022
:105CA000040ED86FAA6A3D0EA96ED8C1A8FFA69CA3
:105CB000A69EA684F2CF00F0F29CF29E0F01550E34
:105CC000A76EAA0EA76EA682A6B2FED7A694005013
:105CD000F2120101AA6A1D0EA96EAEC1A8FFA69C10
:105CE000A69EA684F2CF00F0F29CF29E0F01550E04
:105CF000A76EAA0EA76EA682A6B2FED7A6940050E3
:105D0000F212AA6A2D0EA96EB4C1A8FFA69CA69E87
:105D1000A684F2CF00F0F29CF29E550EA76EAA0E5A
:105D2000A76EA682A6B2FED7A6940050F212010179
:105D3000A3D193C1F0F015EC25F0F12D02D00101B3
:105D40009BD101019351AB5D05E19451B15D02E13D
:105D50008D078FD19351AC5D05E19451B25D02E1A5
:105D60008D0787D19351AD5D05E19451B35D02E19B
:105D70008D077FD19351AE5D05E19451B45D02E191
:105D80008D0777D193C1AFF194C1B5F18FAB1AD024
:105D9000010ED96FAA6A3E0EA96ED9C1A8FFA69CB2
:105DA000A69EA684F2CF00F0F29CF29E0F01550E43
:105DB000A76EAA0EA76EA682A6B2FED7A694005022
:105DC000F21201018FAD1AD0020ED96FAA6A3E0EEF
:105DD000A96ED9C1A8FFA69CA69EA684F2CF00F00A
:105DE000F29CF29E0F01550EA76EAA0EA76EA68218
:105DF000A6B2FED7A6940050F21201018FAF1AD0BE
:105E0000030ED96FAA6A3E0EA96ED9C1A8FFA69C3F
:105E1000A69EA684F2CF00F0F29CF29E0F01550ED2
:105E2000A76EAA0EA76EA682A6B2FED7A6940050B1
:105E3000F212010190AB1AD0040ED96FAA6A3E0E7D
:105E4000A96ED9C1A8FFA69CA69EA684F2CF00F099
:105E5000F29CF29E0F01550EA76EAA0EA76EA682A7
:105E6000A6B2FED7A6940050F2120101AA6A1E0E35
:105E7000A96EAFC1A8FFA69CA69EA684F2CF00F093
:105E8000F29CF29E0F01550EA76EAA0EA76EA68277
:105E9000A6B2FED7A6940050F212AA6A2E0EA96EE0
:105EA000B5C1A8FFA69CA69EA684F2CF00F0F29CE6
:105EB000F29E550EA76EAA0EA76EA682A6B2FED7B8
:105EC000A6940050F2120101D7D093C1F0F015EC66
:105ED00025F0F12D02D00101CFD001019351AB5D2E
:105EE00005E19451B15D02E18D07C3D09351AC5DE2
:105EF00005E19451B25D02E18D07BBD09351AD5DD8
:105F000005E19451B35D02E18D07B3D09351AE5DCD
:105F100005E19451B45D02E18D07ABD09351AF5DC3
:105F200005E19451B55D02E18D07A3D093C1B0F1B5
:105F300094C1B6F18FAB1AD0010EDA6FAA6A3F0E88
:105F4000A96EDAC1A8FFA69CA69EA684F2CF00F097
:105F5000F29CF29E0F01550EA76EAA0EA76EA682A6
:105F6000A6B2FED7A6940050F21201018FAD1AD04E
:105F7000020EDA6FAA6A3F0EA96EDAC1A8FFA69CCC
:105F8000A69EA684F2CF00F0F29CF29E0F01550E61
:105F9000A76EAA0EA76EA682A6B2FED7A694005040
:105FA000F21201018FAF1AD0030EDA6FAA6A3F0E08
:105FB000A96EDAC1A8FFA69CA69EA684F2CF00F027
:105FC000F29CF29E0F01550EA76EAA0EA76EA68236
:105FD000A6B2FED7A6940050F212010190AB1AD0DF
:105FE000040EDA6FAA6A3F0EA96EDAC1A8FFA69C5A
:105FF000A69EA684F2CF00F0F29CF29E0F01550EF1
:10600000A76EAA0EA76EA682A6B2FED7A6940050CF
:10601000F2120101AA6A1F0EA96EB0C1A8FFA69CC8
:10602000A69EA684F2CF00F0F29CF29E0F01550EC0
:10603000A76EAA0EA76EA682A6B2FED7A69400509F
:10604000F212AA6A2F0EA96EB6C1A8FFA69CA69E40
:10605000A684F2CF00F0F29CF29E550EA76EAA0E17
:10606000A76EA682A6B2FED7A6940050F212010136
:1060700003D00C6B0B6B01018F9B8F9D8F9F909BAF
:10608000AA6A200EA96E8FC1A8FFA69CA69EA68410
:10609000F2CF00F0F29CF29E0F01550EA76EAA0EF1
:1060A000A76EA682A6B2FED7A6940050F212AA6AE4
:1060B000210EA96E90C1A8FFA69CA69EA684F2CF31
:1060C00000F0F29CF29E550EA76EAA0EA76EA68255
:1060D000A6B2FED7A6940050F2120101936B946B06
:1060E0000001000CE824F76AF736FF0FF66E600E29
:1060F000F7220A00F550FA6E0800F550F96E68575D
:10610000C658325AAA5B325DCA5E01018F838F8BFB
:10611000000109EC2BF04AEF43F001018F858F8DD0
:10612000000189EC25F054EF43F001018F878F8D3A
:10613000000109EC2BF05EEF43F02C50CA0806E09A
:10614000010190818F8F000189EC25F068EF43F009
:106150002C50CA080CE0010123510808D8A402D031
:10616000000105D090838F8F000109EC2BF072EFB6
:1061700043F02C50CA0806E0010190859087000189
:1061800089EC25F07CEF43F02C50CA0806E00101B1
:106190009089908B000109EC2BF086EF43F0010110
:1061A0002251FC0826E1233B239F23C190F00001EC
:1061B000916B915303E190512E0803E2916B2E0EE7
:1061C000906FAA6A0A0EA96E90C0A8FFA69CA69E10
:1061D000A684F2CF00F0F29CF29E0F01550EA76E3E
:1061E000AA0EA76EA682A6B2FED7A6940050F212FF
:1061F00001012251FD0826E1233B239F23C192F098
:106200000001936B935303E192512E0803E2936BC9
:106210002E0E926FAA6A0D0EA96E92C0A8FFA69CC0
:10622000A69EA684F2CF00F0F29CF29E0F01550EBE
:10623000A76EAA0EA76EA682A6B2FED7A69400509D
:10624000F21201012251FC0802E00A2D5BD000018C
:10625000915303E190510F0818E2915316E19051C8
:106260002E0813E30E0E905F000E915B91C0F5F1C6
:1062700090C0F4F10101F76B0F0EF66F000111EC05
:1062800002F002C091F001C090F091C0F5F190C011
:10629000F4F10101F76B3C0EF66F000111EC02F016
:1062A00002C091F001C090F0AA6A0B0EA96E91C0D5
:1062B000A8FFA69CA69EA684F2CF00F0F29CF29EB8
:1062C0000F01550EA76EAA0EA76EA682A6B2FED724
:1062D000A6940050F212AA6A0C0EA96E90C0A8FFF4
:1062E000A69CA69EA684F2CF00F0F29CF29E550ECC
:1062F000A76EAA0EA76EA682A6B2FED7A6940050DD
:10630000F21201012251FD0802E00A2D5BD00001CA
:10631000935303E192510F0818E2935316E19251FF
:106320002E0813E30E0E925F000E935B93C0F5F1FF
:1063300092C0F4F10101F76B0F0EF66F000111EC42
:1063400002F002C093F001C092F093C0F5F192C048
:10635000F4F10101F76B3C0EF66F000111EC02F055
:1063600002C093F001C092F0AA6A0E0EA96E93C00B
:10637000A8FFA69CA69EA684F2CF00F0F29CF29EF7
:106380000F01550EA76EAA0EA76EA682A6B2FED763
:10639000A6940050F212AA6A0F0EA96E92C0A8FF2E
:1063A000A69CA69EA684F2CF00F0F29CF29E550E0B
:1063B000A76EAA0EA76EA682A6B2FED7A69400501C
:1063C000F21201010001000C01011B6B83A21B8171
:1063D00082A61B8383A01B8582A01B870001000C63
:1063E00001017F6B820E7E6F00018BEC01F0EE6B82
:1063F000ED6B0101006B0001FF6B0101026B016B92
:10640000046B026B010E016F02510708D8A009D27C
:1064100004E101518208D8A004D20B0E006E002EB8
:10642000FED700D0C282C2B2FED7C4CFEEF00001C8
:10643000C3CFEDF00101045303E1010E046FE7D176
:106440000001FF51ED5D01010B6F00510001EE599C
:1064500001010C6F01E2DBD10B51055D0D6F000EE8
:106460000C550E6F01E209D00B51065D0D6F000E49
:106470000C550E6F01E3CFD1CAD1032DE1D083902B
:106480001251050804E10001F281D3D1010112513A
:10649000060804E10001F283CCD101011251070882
:1064A00004E10001F285C5D101011251080804E19F
:1064B0000001F287BED101011251090804E1000177
:1064C000F289B7D1010112510A0804E10001F28BEF
:1064D000B0D1010112510B0804E10001F28DA9D1E4
:1064E000010112510C0804E10001F28FA2D1010157
:1064F00012510D0804E10001F3819BD101011251F9
:106500000E0804E10001F38394D1010112510F0838
:1065100004E10001F3858DD101011251100804E15D
:106520000001F38786D101011251110804E1000135
:10653000F3897FD101011251120804E10001F38BAC
:1065400078D101011251130804E10001F38D71D1DA
:1065500001011251140804E10001F38F6AD1010115
:106560001251150804E10001F48163D101011251B7
:10657000160804E10001F4835CD1010112511708EF
:1065800004E10001F48555D101011251180804E11C
:106590000001F4874ED101011251190804E10001F4
:1065A000F48947D1010112511A0804E10001F48B6A
:1065B00040D1010112511B0804E10001F48D39D1D1
:1065C000010112511C0804E10001F48F32D10101D4
:1065D00012511D0804E10001F5812BD10101125176
:1065E0001E0804E10001F58324D1010112511F08A6
:1065F00004E10001F5851DD101011251200804E1DB
:106600000001F58716D101011251210804E10001B2
:10661000F5890FD101011251220804E10001F58B27
:1066200008D101011251230804E10001F58D01D1C7
:1066300001011251240804E10001F58FFAD0010193
:106640000353D8A4E1D082901251050804E100015F
:10665000F681EFD001011251060804E10001F68332
:10666000E8D001011251070804E10001F685E1D0EC
:1066700001011251080804E10001F687DAD0010196
:106680001251090804E10001F689D3D00101125129
:106690000A0804E10001F68BCCD0010112510B086D
:1066A00004E10001F68DC5D0010112510C0804E18E
:1066B0000001F68FBED0010112510D0804E1000166
:1066C000F781B7D0010112510E0804E10001F783F0
:1066D000B0D0010112510F0804E10001F785A9D0E3
:1066E00001011251100804E10001F787A2D0010155
:1066F0001251110804E10001F7899BD001011251E8
:10670000120804E10001F78B94D001011251130823
:1067100004E10001F78D8DD001011251140804E14C
:106720000001F78F86D001011251150804E1000124
:10673000F8817FD001011251160804E10001F883AD
:1067400078D001011251170804E10001F88571D0D9
:1067500001011251180804E10001F8876AD0010113
:106760001251190804E10001F88963D001011251A6
:106770001A0804E10001F88B5CD0010112511B08DA
:1067800004E10001F88D55D0010112511C0804E10B
:106790000001F88F4ED0010112511D0804E10001E3
:1067A000F98147D0010112511E0804E10001F9836B
:1067B00040D0010112511F0804E10001F98539D0D0
:1067C00001011251200804E10001F98732D00101D2
:1067D0001251210804E10001F9892BD00101125165
:1067E000220804E10001F98B24D001011251230891
:1067F00004E10001F98D1DD001011251240804E1CA
:106800000001F98F16D00101000113D00101EEC083
:1068100000F1EDC0FFF00C6B0B6B012BD8B4022B19
:10682000F3D5032D02D083908392035302E182902B
:10683000829601010C6B0B6B0001000C01011BB176
:1068400002D0372D02D0839201D083821BB302D0B5
:10685000382D02D0829601D082861BA502D083906B
:1068600001D083801BA702D0829001D082800001DA
:10687000000C0101786B776B772BD8B4782B3D0E29
:10688000006E002EFED782A208D07351F90802E3F1
:10689000732B02D0010E756F02D0756B736B83A4DE
:1068A00008D07451F90802E3742B02D0010E766F00
:1068B00002D0766B746B7851030804E3DDE1775105
:1068C000E808DAE20001000C010107B502D03553F7
:1068D00036E0755311E176530FE1186AF2BC188C5B
:1068E000F29CF2BE188EF29E0001B7EC0AF018BCC2
:1068F000F28C18BEF28E010175530FE1186AF2BCDA
:10690000188CF29CF2BE188EF29E000151EC03F03E
:1069100018BCF28C18BEF28E010176530FE1186A92
:10692000F2BC188CF29CF2BE188EF29E00014CEC68
:1069300006F018BCF28C18BEF28E01010FD0186A56
:10694000F2BC188CF29CF2BE188EF29E0001DFECB5
:1069500008F018BCF28C18BEF28E010107A123D0FA
:10696000755321E1355310E0186AF2BC188CF29C83
:10697000F2BE188EF29E000151EC03F018BCF28CAE
:1069800018BEF28E0FD00101186AF2BC188CF29C6E
:10699000F2BE188EF29E00017AEC16F018BCF28C52
:1069A00018BEF28E010107A323D0765321E135539F
:1069B00010E0186AF2BC188CF29CF2BE188EF29E9F
:1069C00000014CEC06F018BCF28C18BEF28E0FD011
:1069D0000101186AF2BC188CF29CF2BE188EF29E6D
:1069E0000001ABEC17F018BCF28C18BEF28E01015E
:1069F000076B0001E2EF3AF0010E486EA092819819
:106A0000819AF2CFF4F1F29CF29EAA6AFF0EA96E6F
:106A1000A69CA69EA680A8500101F4BDF28CF4BFEE
:106A2000F28E096F83828286010E356F0001CB6B77
:106A3000CC6B0101335308E1316B326B336B346B38
:106A4000000161EC14F0010130B0A3EF3AF030B274
:106A5000A3EF3AF00C6B0B6B146B136B156B1853A5
:106A600005E14E0E176F200E166F04D0270E176F1C
:106A7000100E166F0001FC5309E001011551310899
:106A800002E3152B03D0156B8B708C7001017F6BAB
:106A90000A0E7E6F00018BEC01F00101132BD8B4BC
:106AA000142B000E82BA010E82BA09D00C5306E1F3
:106AB0000B51130803E30B2BD8B40C2B02D00C6B37
:106AC0000B6B0C5303E10B51130802E2A3EF3AF0F6
:106AD0001451175D04E3CEE11651135DCBE30001C1
:106AE000FC5318E00101372D01D004D00001C82D5E
:106AF00004D00101838003D0000183900101382D6F
:106B000001D004D00001C92D04D00101828003D03E
:106B1000000182900101156B000102EC00F0CB0E28
:106B2000926EC150C00B1D09C16EC050C00B080948
:106B3000C06EC08EC28001013C53D8A481943D53E5
:106B4000D8A481927F6B640E7E6F00018BEC01F004
:106B5000839801010C6B0B6B146B136B7F6B0A0E2C
:106B60007E6F00018BEC01F00101132BD8B4142BC4
:106B7000000E82BA010E82BA09D00C5306E10B5105
:106B8000130803E30B2BD8B40C2B02D00C6B0B6B4C
:106B90000C5303E10B51130802E2A3EF3AF0145334
:106BA00003E11351C708DAE23C530CE0372D01D062
:106BB00009D00001C82D03D0010104D0000130A08C
:106BC00003D00101C4D00001040E016EC250C30BFA
:106BD0000110C26E0B0E006E002EFED700D0816B2E
:106BE000806B806B816B010E0101126F12511008D6
:106BF00018E37F6B0A0E7E6F00018BEC01F0C282FE
:106C0000C2B2FED7C4CF0EF10101C3CF0DF10D51B9
:106C10000001802701010E51000181230101122B87
:106C2000E5D781C085F080C084F0000185338433CE
:106C30008533843385338433853384330F0E85174E
:106C400001010951CA080EE10001855303E1845195
:106C5000900805E2010E01013A6F839203D0010111
:106C60003A6B83820951380803E00951190811E190
:106C70000001855100080AE2FF0A03E184518008FF
:106C800005E2010E01013A6F839203D001013A6BD4
:106C900083820951580803E00951290811E10001D4
:106CA000855100080AE2FF0A03E18451F80805E271
:106CB000010E01013A6F839203D001013A6B838286
:106CC0000951480803E00951390811E100018551D3
:106CD00002080AE2FF0A03E184511A0805E2010EE4
:106CE00001013A6F839203D001013A6B8382000164
:106CF00081338033813380333F0E8117D8908037C2
:106D0000813780A302D0808101D0809180A502D0FC
:106D1000808301D0809380A702D0808501D08095A8
:106D2000808781AD02D0818F01D0819F81AB02D05D
:106D3000818D01D0819D81A902D0818B01D0819B61
:106D400081A702D0818901D08199818701013D53BA
:106D50000CE0382D01D009D00001C92D03D001016C
:106D600004D0000130A203D00101BAD00001000E0E
:106D7000016EC250C30B0110C26E1E0E006E002EBB
:106D8000FED70000836B826B826B836B010E010167
:106D9000126F1251100818E37F6B0A0E7E6F00010C
:106DA0008BEC01F0C282C2B2FED7C4CF0EF101015A
:106DB000C3CF0DF10D510001822701010E510001D9
:106DC00083230101122BE5D783C085F082C084F0B4
:106DD00000018533843385338433853384338533AD
:106DE00084330F0E851701010951CA080EE1000115
:106DF000855303E18451900805E2010E01013B6FC8
:106E0000829603D001013B6B82860951380811E15B
:106E10000001855100080AE2FF0A03E1845180085D
:106E200005E2010E01013B6F829603D001013B6B2D
:106E300082860951580811E10001855100080AE2D3
:106E4000FF0A03E18451F80805E2010E01013B6FDE
:106E5000829603D001013B6B82860951480811E1FB
:106E60000001855102080AE2FF0A03E184511A0871
:106E700005E2010E01013B6F829603D001013B6BDD
:106E80008286000183338233833382333F0E83173C
:106E9000D8908237833782A302D0828101D0829139
:106EA00082A502D0828301D0829382A702D08285FC
:106EB00001D08295828783AD02D0838F01D0839FDA
:106EC00083AB02D0838D01D0839D83A902D0838BB5
:106ED00001D0839B83A702D0838901D083998387C4
:106EE0000001E4EC31F001017F6BC80E7E6F000100
:106EF0008BEC01F0C150C00B0D09C16E01010C6B90
:106F00000B6B146B136B7F6B0A0E7E6F00018BECA7
:106F100001F00101132BD8B4142B000E82BA010E1C
:106F200082BA09D00C5306E10B51130803E30B2B73
:106F3000D8B40C2B02D00C6B0B6B0C5303E10B5130
:106F4000130801E200D3145303E113516308DBE299
:106F50003C530EE0372D01D00BD00001C82D02D0DC
:106F6000010106D001013A2D01D002D030A001D09C
:106F700009D1838283800C6B0B6B146B136B1853DA
:106F800005E1010E176F2C0E166F04D0010E176F5E
:106F9000F40E166F7F6B0A0E7E6F00018BEC01F012
:106FA0000101132BD8B4142B000E82BA010E82BA41
:106FB00009D00C5306E10B51130803E30B2BD8B493
:106FC0000C2B02D00C6B0B6B0C5303E10B51130811
:106FD00001E2B9D21451175D04E3DCE11651135DEF
:106FE000D9E3010E126F125111081DE38184990E2D
:106FF000006E002EFED781887F6B0E0E7E6F000123
:107000008BEC01F08198050E006E002EFED700D0AB
:10701000819401017F6B3F0E7E6F00018BEC01F0CC
:107020000101122BE0D70C6B0B6B146B136B7F6B96
:107030000A0E7E6F00018BEC01F00101132BD8B416
:10704000142B000E82BA010E82BA09D00C5306E14D
:107050000B51130803E30B2BD8B40C2B02D00C6B91
:107060000B6B0C5303E10B51130801E26CD214516A
:10707000020804E3DCE113515708D9E20001F56B83
:10708000F46BF36BF26B040E016EC250C30B011074
:10709000C26E0B0E006E002EFED700D0050EFE6FE6
:1070A000FEC012F18184990E006E002EFED78188F9
:1070B00001017F6B0E0E7E6F00018BEC01F0819859
:1070C000050E006E002EFED700D0819401017F6B6B
:1070D0003F0E7E6F00018BEC01F0FE07FE5101E0D8
:1070E000E1D7010E0101036F0001F0EC31F0010165
:1070F000122B12C1FEF0010E7F6F900E7E6F000109
:107100008BEC01F08382838001010C6B0B6B146BA1
:10711000136B185304E1176B640E166F04D0010E45
:10712000176F5E0E166F7F6B0A0E7E6F00018BEC81
:1071300001F00101132BD8B4142B000E82BA010EFA
:1071400082BA09D00C5306E10B51130803E30B2B51
:10715000D8B40C2B02D00C6B0B6B0C5303E10B510E
:10716000130801E2F0D11451175D04E3DCE116517C
:10717000135DD9E30001FE51180801E393D71EEC1B
:1071800034F001013D530EE0382D01D00BD0000149
:10719000C92D02D0010106D001013B2D01D002D042
:1071A00030A201D02DD10C6B0B6B146B136B7F6B6A
:1071B0000A0E7E6F00018BEC01F00101132BD8B495
:1071C000142B000E82BA010E82BA09D00C5306E1CC
:1071D0000B51130803E30B2BD8B40C2B02D00C6B10
:1071E0000B6B0C5303E10B51130801E2ACD11453A8
:1071F00003E11351C708DBE2828682800C6B0B6BC4
:10720000146B136B185304E1176BC80E166F04D080
:10721000030E176F200E166F7F6B0A0E7E6F000134
:107220008BEC01F00101132BD8B4142B000E82BAA1
:10723000010E82BA09D00C5306E10B51130803E387
:107240000B2BD8B40C2B02D00C6B0B6B0C5303E143
:107250000B51130801E277D11451175D04E3DCE10F
:107260001651135DD9E3010E126F125111081DE37F
:107270008182990E006E002EFED7818A7F6B0E0EE2
:107280007E6F00018BEC01F0819A050E006E002EDE
:10729000FED700D0819201017F6B3F0E7E6F00010F
:1072A0008BEC01F00101122BE0D70C6B0B6B146B14
:1072B000136B7F6B0A0E7E6F00018BEC01F00101F6
:1072C000132BD8B4142B000E82BA010E82BA09D047
:1072D0000C5306E10B51130803E30B2BD8B40C2B12
:1072E00002D00C6B0B6B0C5303E10B51130801E242
:1072F0002AD11451020804E3DCE113515708D9E202
:107300000001F96BF86BF76BF66B000E016EC25063
:10731000C30B0110C26E0B0E006E002EFED700D004
:10732000050EFE6FFEC012F18182990E006E002ED6
:10733000FED7818A01017F6B0E0E7E6F00018BEC00
:1073400001F0819A050E006E002EFED700D08192CA
:1073500001017F6B3F0E7E6F00018BEC01F0FE0799
:10736000FE5101E0E1D70101036B0001F0EC31F0C7
:107370000101122B12C1FEF0010E7F6F900E7E6F85
:1073800000018BEC01F08286828001010C6B0B6B9B
:10739000146B136B185304E1176B640E166F04D053
:1073A000010E176F5E0E166F7F6B0A0E7E6F000167
:1073B0008BEC01F00101132BD8B4142B000E82BA10
:1073C000010E82BA09D00C5306E10B51130803E3F6
:1073D0000B2BD8B40C2B02D00C6B0B6B0C5303E1B2
:1073E0000B51130801E2AFD01451175D04E3DCE147
:1073F0001651135DD9E30001FE51180801E394D73B
:1074000000011EEC34F0838801017F6BC80E7E6F93
:1074100000018BEC01F08184818201010C6B0B6B0C
:10742000146B136B185305E1010E176FF40E166FF2
:1074300004D0050E176FDC0E166F7F6B0A0E7E6F81
:1074400000018BEC01F00101132BD8B4142B000EBA
:1074500082BA010E82BA09D00C5306E10B5113080F
:1074600003E30B2BD8B40C2B02D00C6B0B6B0C531F
:1074700003E10B51130801E266D01451175D04E3D8
:10748000DCE11651135DD9E30C6B0B6B146B136BC2
:107490007F6B0A0E7E6F00018BEC01F00101132B54
:1074A000D8B4142B000E82BA010E82BA09D00C5344
:1074B00006E10B51130803E30B2BD8B40C2B02D0BD
:1074C0000C6B0B6B0C5303E10B51130801E23BD027
:1074D0001451010804E3DCE11351F308D9E20C6B09
:1074E0000B6B7F6B0A0E7E6F00018BEC01F0000EC0
:1074F00082BA010E0101F46F0B2BD8B40C2B0B5187
:10750000140803E10C53D8B41ED082AAEAD70001B4
:107510004BEC19F0CFEC02F00101525302E053534F
:1075200012E1030E7F6FE80E7E6F00018BEC01F01D
:1075300039EC34F00101752D02D0010E526F762D19
:1075400002D0010E536F0C5303E10B5113080AE2F2
:1075500083887F6BC80E7E6F00018BEC01F0818405
:1075600081820101346B0C6B0B6BC80E926E896AC1
:10757000010E7F6FF40E7E6F00018BEC01F00101B4
:10758000522D01D002D0532D16D0522D03D0010E12
:10759000756F8392532D03D0010E766F8296070E7E
:1075A0007F6FD00E7E6F00018BEC01F0010108515E
:1075B0000908D8B4086B0001FC5304E166EC01F043
:1075C00064EF34F00101076B352D04D00851090830
:1075D000D8B4356B0001FC5314E00101356B000198
:1075E000FC6B01016D6B2E6B2F6B306B476B416B2E
:1075F000426B436B446B5B6B2B6B2C6B2D6B586B33
:10760000576B0001000C010E486E69EC12F001018D
:107610005C51F10810E15E2D0ED070530CE1465321
:107620000AE1270E7F6F100E7E6F00018BEC01F0D8
:10763000DFEC08F00101486A0101A9EF50F0EA53BC
:10764000D8A406EF43F0EF510508D8B006EF43F099
:107650002C50CA080DE101013A53D8B403D00001FF
:1076600006EF43F03B53D8B403D0000106EF43F0DC
:1076700001016153D8B403D0000106EF43F083B693
:1076800003D0000106EF43F04653D8B403D0000105
:1076900006EF43F04753D8B403D0000106EF43F0A0
:1076A0005B510608D8A403D0000106EF43F0355320
:1076B000D8B403D0000106EF43F03653D8B403D05A
:1076C000000106EF43F02151F708D8A406EF43F07C
:1076D00022510B08D8A406EF43F023510A08D8A47E
:1076E00006EF43F08E2D03D08E6BA9EF50F08E5134
:1076F000180802E1A9EF50F03C53D8B45DD08FA533
:107700005BD06D53D8A458D0000134EC01F00101D6
:10771000CF51020803E1B71FA551B717D051020896
:1077200003E1B81FA651B817D151020803E1B91FF0
:10773000A751B917D251020803E1BA1FA851BA17CD
:10774000D351020803E1BB1FA951BB17D451020852
:1077500003E1BC1FAA51BC17CF51020803E1A55198
:10776000B75D1EE0D051020803E1A651B85D18E0F4
:10777000D151020803E1A751B95D12E0D2510208CC
:1077800003E1A851BA5D0CE0D351020803E1A9510D
:10779000BB5D06E0D45102080BE1AA51BC5D08E1D3
:1077A000972B972D04D0010E866F956B976B04D0A5
:1077B0002E2D01D0866B976B3D53D8B45DD08FA72B
:1077C0005BD06D53D8A458D0000141EC01F0010109
:1077D000D551020803E1BD1FB151BD17D6510208B2
:1077E00003E1BE1FB251BE17D751020803E1BF1F0C
:1077F000B351BF17D851020803E1C01FB451C017DD
:10780000D951020803E1C11FB551C117DA5102086D
:1078100003E1C21FB651C217D551020803E1B151AD
:10782000BD5D1EE0D651020803E1B251BE5D18E015
:10783000D751020803E1B351BF5D12E0D8510208ED
:1078400003E1B451C05D0CE0D951020803E1B55128
:10785000C15D06E0DA5102080BE1B651C25D08E1F4
:10786000982B982D04D0010E876F966B986B04D0DF
:107870002F2D01D0876B986B2C50CA0801E199D14C
:107880003C53D8B455D090A153D06D5351E1000171
:1078900034EC01F00101CF51030802E1A551B71703
:1078A000D051030802E1A651B817D151030802E1F3
:1078B000A751B917D251030802E1A851BA17D35101
:1078C000030802E1A951BB17D451030802E1AA51F0
:1078D000BC17CF51030803E1A551B75D1EE0D0519D
:1078E000030803E1A651B85D18E0D151030803E194
:1078F000A751B95D12E0D251030803E1A851BA5D66
:107900000CE0D351030803E1A951BB5D06E0D4515B
:1079100003080AE1AA51BC5D07E1992B992D03D018
:10792000010E886F996B04D02E2D01D0886B996B56
:107930003D53D8B455D090A353D06D5351E10001BD
:1079400041EC01F00101D551030802E1B151BD172D
:10795000D651030802E1B251BE17D751030802E124
:10796000B351BF17D851030802E1B451C017D95120
:10797000030802E1B551C117DA51030802E1B6511B
:10798000C217D551030803E1B151BD5D1EE0D651C8
:10799000030803E1B251BE5D18E0D751030803E1CB
:1079A000B351BF5D12E0D851030803E1B451C05D8B
:1079B0000CE0D951030803E1B551C15D06E0DA518D
:1079C00003080AE1B651C25D07E19A2B9A2D03D054
:1079D000010E896F9A6B04D02F2D01D0896B9A6BA1
:1079E0005E530BE0462D01D008D0975302E02E5392
:1079F00004E0985304E02F5302E159EF40F02C507B
:107A0000CA0801E1D6D03C53D8B468D090A566D05E
:107A1000000134EC01F00101CF51040802E1A5514D
:107A2000B717D051040802E1A651B817D151040884
:107A300002E1A751B917D251040802E1A851BA17BF
:107A4000D351040802E1A951BB17D451040802E143
:107A5000AA51BC17CF51040803E1A551B75D1EE040
:107A6000D051040803E1A651B85D18E0D1510408D3
:107A700003E1A751B95D12E0D251040803E1A85116
:107A8000BA5D0CE0D351040803E1A951BB5D06E0E7
:107A9000D451040817E1AA51BC5D14E12B5308E04E
:107AA0006D2D02D0315304E0842D0BD08A5309E1AF
:107AB0009D2B9D2D06D0010E8A6F9D6B6D2D01D0E3
:107AC000846B0CD02B2D01D007D02E2D01D004D0EB
:107AD0006D2D03D0312D01D08A6B9D6B3D53D8B4F1
:107AE00068D090A966D0000141EC01F00101D551A8
:107AF000040802E1B151BD17D651040802E1B251A8
:107B0000BE17D751040802E1B351BF17D85104087A
:107B100002E1B451C017D951040802E1B551C117AF
:107B2000DA51040802E1B651C217D551040803E145
:107B3000B151BD5D1EE0D651040803E1B251BE5DF6
:107B400018E0D751040803E1B351BF5D12E0D851EA
:107B5000040803E1B451C05D0CE0D951040803E10D
:107B6000B551C15D06E0DA51040817E1B651C25DB6
:107B700014E12C5308E06D2D02D0325304E0852D22
:107B80000BD08B5309E19E2B9E2D06D0010E8B6FDF
:107B90009E6B6D2D01D0856B0CD02C2D01D007D0A4
:107BA0002F2D01D004D06D2D03D0322D01D08B6B41
:107BB0009E6B3C510208D8A43CD18FA13AD16D53A1
:107BC000D8A437D1000134EC01F00101CF2D02D04F
:107BD000A551B717D02D02D0A651B817D12D02D07C
:107BE000A751B917D22D02D0A851BA17D32D02D060
:107BF000A951BB17D42D02D0AA51BC17CF2D03D049
:107C0000A551B75D1AE0D02D03D0A651B85D15E09F
:107C1000D12D03D0A751B95D10E0D22D03D0A851CA
:107C2000BA5D0BE0D32D03D0A951BB5D06E0D42D86
:107C3000E6D0AA51BC5DD8A4E2D02C50CA08D8A482
:107C4000D1D02B2DCED0010E846FCF2D0AD0B753BB
:107C500008E10001B7B102D0010103D053EC01F0FB
:107C60000101D02D0AD0B85308E10001B7B302D00A
:107C7000010103D053EC01F00101D12D0AD0B95319
:107C800008E10001B7B502D0010103D053EC01F0C7
:107C90000101D22D0AD0BA5308E10001B7B702D0D2
:107CA000010103D053EC01F00101D32D0AD0BB53E5
:107CB00008E10001B7B902D0010103D053EC01F093
:107CC0000101D42D0AD0BC5308E10001B7BB02D09A
:107CD000010103D053EC01F00101CF2D14D0A551C7
:107CE000B75D11E10001B7A102D001010CD04EEC4B
:107CF00001F0365051123750521238505312395049
:107D00005412B7810101D02D14D0A651B85D11E1F4
:107D10000001B7A302D001010CD04EEC01F042509B
:107D20005112435052124450531245505412B783CB
:107D30000101D12D14D0A751B95D11E10001B7A502
:107D400002D001010CD04EEC01F05D5051125E509A
:107D500052125F50531260505412B7850101D22D58
:107D600014D0A851BA5D11E10001B7A702D00101FA
:107D70000CD04EEC01F0615051126250521263501F
:107D8000531264505412B7870101D32D14D0A95156
:107D9000BB5D11E10001B7A902D001010CD04EEC8E
:107DA00001F06550511266505212675053126850DC
:107DB0005412B7890101D42D14D0AA51BC5D11E130
:107DC0000001B7AB02D001010CD04EEC01F06950BC
:107DD00051126A5052126B5053126C505412B78B9E
:107DE00001010CD02B5304E08A2D08D0845306E106
:107DF0009B2B9B2D03D0010E846F9B6B1AD02C50B4
:107E0000CA0810E1842D0DD03E504D163F504E163D
:107E100040504F1641505016846B000153EC01F056
:107E2000010107D02B2D01D002D02E2D01D0846B63
:107E30009B6B3D510208D8A43CD18FA33AD16D531E
:107E4000D8A437D1000141EC01F00101D52D02D0B9
:107E5000B151BD17D62D02D0B251BE17D72D02D0C9
:107E6000B351BF17D82D02D0B451C017D92D02D0AD
:107E7000B551C117DA2D02D0B651C217D52D03D096
:107E8000B151BD5D1AE0D62D03D0B251BE5D15E0F3
:107E9000D72D03D0B351BF5D10E0D82D03D0B4511E
:107EA000C05D0BE0D92D03D0B551C15D06E0DA2DE0
:107EB000E6D0B651C25DD8A4E2D02C50CA08D8A4EE
:107EC000D1D02C2DCED0010E856FD52D0AD0BD532B
:107ED00008E10001B7BD02D0010103D05DEC01F063
:107EE0000101D62D0AD0BE5308E10001B7BF02D070
:107EF000010103D05DEC01F00101D72D0AD0BF5381
:107F000008E10001B8B102D0010103D05DEC01F03D
:107F10000101D82D0AD0C05308E10001B8B302D046
:107F2000010103D05DEC01F00101D92D0AD0C1534C
:107F300008E10001B8B502D0010103D05DEC01F009
:107F40000101DA2D0AD0C25308E10001B8B702D00E
:107F5000010103D05DEC01F00101D52D14D0B15128
:107F6000BD5D11E10001B7AD02D001010CD04EECB6
:107F700001F09451751295517612965177129751DE
:107F80007812B78D0101D62D14D0B251BE5D11E12A
:107F90000001B7AF02D001010CD04EEC01F09851B6
:107FA0007512995176129A5177129B517812B78FA8
:107FB0000101D72D14D0B351BF5D11E10001B8A16B
:107FC00002D001010CD04EEC01F09C5175129D5174
:107FD00076129E5177129F517812B8810101D82DE7
:107FE00014D0B451C05D11E10001B8A302D0010169
:107FF0000CD04EEC01F0A0517512A1517612A25195
:108000007712A3517812B8830101D92D14D0B5513C
:10801000C15D11E10001B8A502D001010CD04EEC08
:1080200001F0A4517512A5517612A6517712A751ED
:108030007812B8850101DA2D14D0B651C25D11E174
:108040000001B8A702D001010CD04EEC01F0A851FC
:108050007512A9517612AA517712AB517812B887CE
:1080600001010CD02C5304E08B2D08D0855306E180
:108070009C2B9C2D03D0010E856F9C6B1AD02C502D
:10808000CA0810E1852D0DD071506D1672506E1614
:1080900073506F1674507016856B00015DEC01F023
:1080A000010107D02C2D01D002D02F2D01D0856BDE
:1080B0009C6B6D2D01D002D0702D01D085D137532E
:1080C00002E0385327E1862D25D0872D23D02E536B
:1080D00021E12F531FE13C531DE03D531BE0416B59
:1080E0004C6B4A6B426B4D6B4B6B050E5B6F3053A9
:1080F00010E1010E836F000166EC01F00101655192
:10810000000802E27FD204D00001B7EC0AF00101BE
:10811000836B38D08FA51AD0375318E1862D16D02F
:108120003C5314E0416B4C6B4A6B050E5B6F2E5356
:108130000DE1000166EC01F001016551000802E269
:1081400061D204D0000151EC03F001018FA71AD0D5
:10815000385318E1872D16D03D5314E0426B4D6B18
:108160004B6B050E5B6F2F530DE1000166EC01F0C8
:1081700001016551000802E245D204D000014CEC37
:1081800006F001018FA52DD08FA72BD0865329E1B2
:10819000875327E1955325E1965323E1302D21D0D4
:1081A00041531FE142531DE13C5308E0755306E182
:1081B000842D04D05E2D02D0010E2B6F000181ECC6
:1081C0000EF001013D5308E0765306E1852D04D001
:1081D0005E2D02D0010E2C6F00018FEC0EF030D01E
:1081E00001018FA516D0865314E1955312E12E2D6F
:1081F00010D041530EE13C5308E0755306E1842D45
:1082000004D05E2D02D0010E2B6F000181EC0EF028
:1082100001018FA716D0875314E1965312E12F2D39
:1082200010D042530EE13D5308E0765306E1852D10
:1082300004D05E2D02D0010E2C6F00018FEC0EF0E9
:1082400001012C50CA0801E1DDD1375302E0385357
:108250002AE190A128D090A326D0865324E1882D2E
:1082600022D0875320E1892D1ED02E531CE12F539D
:108270001AE13C5318E03D5316E0010E956F966FDE
:10828000305310E1010E836F000166EC01F0010133
:108290006551000802E2B6D104D00001B7EC0AF043
:1082A0000101836B36D090A119D0375317E1882D87
:1082B00015D0865313E13C5311E0010E956F2E53F8
:1082C0000DE1000166EC01F001016551000802E2D8
:1082D00099D104D0000151EC03F0010190A319D011
:1082E000385317E1892D15D0875313E13D5311E021
:1082F000010E966F2F530DE1000166EC01F00101B4
:108300006551000802E27ED104D000014CEC06F079
:10831000010190A129D090A327D0885325E189534A
:1083200023E1865321E187531FE1302D1DD04153B6
:108330001BE1425319E13C5308E0755306E1842DDB
:1083400004D05E2D02D0010E2B6F3D5308E0765312
:1083500006E1852D04D05E2D02D0010E2C6F0001A8
:1083600069EC12F0010130D090A116D0885314E1CD
:10837000865312E12E2D10D041530EE13C5308E0FC
:10838000755306E1842D04D05E2D02D0010E2B6FB3
:10839000000188EC10F0010190A316D0895314E17C
:1083A000875312E12F2D10D042530EE13D5308E0C8
:1083B000765306E1852D04D05E2D02D0010E2C6F80
:1083C00000019DEC0EF001018FA107D08FA305D015
:1083D000842D03D0852D01D008D090A545D08A2DBD
:1083E00043D090A941D08B2D3FD0375302E0385372
:1083F0003BE12E5339E12F5337E13C5335E03D53F8
:1084000033E06D2D1FD090A51DD090A91BD0312D2C
:1084100001D002D0322D01D027D0335312E1000118
:10842000FA53D8B402D001010CD0FB53D8B402D017
:10843000010107D00101346B000161EC14F001016E
:10844000E1D012D02D5310E1000166EC01F00101E2
:108450006551000802E2D6D006D05E2D04D000019E
:10846000DFEC08F00101CED08FA103D0842D01D024
:1084700004D090A529D08A2D27D0375325E12E533B
:1084800023E13C5321E06D2D0ED090A50CD031534B
:1084900009E10001FA53D8B402D0010103D0F5EF8D
:1084A00015F0010111D02B530FE1000166EC01F032
:1084B00001016551000802E2A5D006D05E2D04D06E
:1084C00000017AEC16F001018FA303D0852D01D0B5
:1084D00004D090A929D08B2D27D0385325E12F53D4
:1084E00023E13D5321E06D2D0ED090A90CD03253E5
:1084F00009E10001FB53D8B402D0010103D026EFFB
:1085000017F0010111D02C530FE1000166EC01F0CE
:1085100001016551000802E275D006D05E2D04D03D
:108520000001ABEC17F001018FA102D08FB304D092
:1085300090A528D090A926D0845324E1855322E128
:108540008A5320E18B531EE16D2D0CD090A50AD0EB
:1085500090A908D0332D05D000014BEC19F0010192
:1085600051D010D02D2D0ED070530CE12E5307E1B9
:108570002F5305E10001A4EC1AF002D001012D6B8C
:10858000010140D08FB102D090A51BD0845319E1D6
:108590008A5317E16D2D09D090A507D0312D04D055
:1085A0000001D3EC18F001010CD02B2D0AD0705330
:1085B00008E12E5305E1000136EC1AF003D0010169
:1085C0002B6B000101018FB302D090A91BD0855302
:1085D00019E18B5317E16D2D09D090A907D0322DE9
:1085E00004D000015BEC18F001010CD02C2D0AD056
:1085F000705308E12F5305E10001C8EC19F003D0D6
:1086000001012C6B00010101A9EF50F0010128517B
:10861000215D02E0A9EF50F00001CDEF1BF0EF511A
:10862000050808E20101612D03D0000103D001011A
:108630007B2D03D00101A9EF50F022511A0809E166
:108640002351080806E1010E0001FC6F7BEF50F09A
:10865000010122514B0805E10001BA8377EF21F0B7
:1086600001012251BB0805E10001BA8546EF23F064
:1086700001012251FA0807E10001BA8301EF2BF052
:108680000101A9EF50F022512C0807E10001BA8541
:1086900085EF30F00101A9EF50F022512B0807E1DE
:1086A0000001BA838DEF30F00101A9EF50F02251A3
:1086B0003B0807E10001BA8595EF30F00101A9EF11
:1086C00050F022515A0807E10001BA839DEF30F0C3
:1086D0000101A9EF50F022511A0807E10001BA8503
:1086E000A8EF30F00101A9EF50F022511D0807E179
:1086F0000001BA83B9EF30F00101A9EF50F0225127
:108700002D0807E10001BA85C4EF30F00101A9EF9F
:1087100050F02C50CA0802E018EF4DF022510D081D
:10872000D8A4C1D0A0928198819A0001BA83010196
:108730002351070B0001B96FB951FB0FD8B076D0A8
:10874000050FACEF50F0010123A902D04D8E01D0EE
:108750004D9E23AB02D04D8C01D04D9C23AD02D059
:108760004D8A01D04D9A23AF02D04D8801D04D984B
:1087700000015CD0010123A902D04D8601D04D96A5
:1087800023AB02D04D8401D04D9423AD02D04D8255
:1087900001D04D9223AF02D04D8001D04D90000109
:1087A00045D0010123A902D04E8E01D04E9E23ABAD
:1087B00002D04E8C01D04E9C23AD02D04E8A01D007
:1087C0004E9A23AF02D04E8801D04E9800012ED091
:1087D000010123A902D04E8601D04E9623AB02D0D0
:1087E0004E8401D04E9423AD02D04E8201D04E92E1
:1087F00023AF02D04E8001D04E90000117D001016E
:1088000023A902D04F8E01D04F9E23AB02D04F8CB4
:1088100001D04F9C23AD02D04F8A01D04F9A23AF95
:1088200002D04F8801D04F98000100D0F00E4F16B3
:10883000506A50C041F04FC040F04EC03FF04DC0B4
:108840003EF03E5036163F503716405038164150D5
:1088500039163E5042163F50431640504416415080
:1088600045163E505D163F505E1640505F16415013
:1088700060163E5061163F506216405063164150DC
:1088800064163E5065163F506616405067164150BC
:1088900068163E5069163F506A1640506B1641509C
:1088A0006C16C683010122510E08D8A4C1D0A09233
:1088B0008198819A0001BA8501012351070B0001BB
:1088C000B96FB951FB0FD8B076D0050FBEEF50F09D
:1088D000010123A902D06D8E01D06D9E23AB02D081
:1088E0006D8C01D06D9C23AD02D06D8A01D06D9A44
:1088F00023AF02D06D8801D06D9800015CD00101DA
:1089000023A902D06D8601D06D9623AB02D06D8471
:1089100001D06D9423AD02D06D8201D06D9223AF52
:1089200002D06D8001D06D90000145D0010123A9D6
:1089300002D06E8E01D06E9E23AB02D06E8C01D021
:108940006E9C23AD02D06E8A01D06E9A23AF02D006
:108950006E8801D06E9800012ED0010123A902D0AB
:108960006E8601D06E9623AB02D06E8401D06E94D9
:1089700023AD02D06E8201D06E9223AF02D06E8002
:1089800001D06E90000117D0010123A902D06F8E93
:1089900001D06F9E23AB02D06F8C01D06F9C23ADB2
:1089A00002D06F8A01D06F9A23AF02D06F8801D0B6
:1089B0006F98000100D0F00E6F16706A70C074F0EE
:1089C0006FC073F06EC072F06DC071F0715094178B
:1089D00072509517735096177450971771509817D7
:1089E0007250991773509A1774509B1771509C17B7
:1089F00072509D1773509E1774509F177150A01797
:108A00007250A1177350A2177450A3177150A41776
:108A10007250A5177350A6177450A7177150A81756
:108A20007250A9177350AA177450AB17C68501016D
:108A30002251AD08D8A48DD0A0928198819A0001CE
:108A4000BA8301012351070B0001B96FB951FB0F24
:108A5000D8B076D0050FD0EF50F0010123A902D095
:108A6000368E01D0369E23AB02D0368C01D0369C98
:108A700023AD02D0368A01D0369A23AF02D0368891
:108A800001D0369800015CD0010123A902D03686BE
:108A900001D0369623AB02D0368401D0369423AD74
:108AA00002D0368201D0369223AF02D0368001D078
:108AB0003690000145D0010123A902D0378E01D0A4
:108AC000379E23AB02D0378C01D0379C23AD02D028
:108AD000378A01D0379A23AF02D0378801D0379830
:108AE00000012ED0010123A902D0378601D037968C
:108AF00023AB02D0378401D0379423AD02D0378224
:108B000001D0379223AF02D0378001D037900001D7
:108B100017D0010123A902D0388E01D0389E23AB93
:108B200002D0388C01D0389C23AD02D0388A01D0D5
:108B3000389A23AF02D0388801D03898000100D08D
:108B40003E5036163F5037164050381641503916B1
:108B500001012251BD08D8A48DD0A0928198819A9C
:108B60000001BA8301012351070B0001B96FB9510C
:108B7000FB0FD8B076D0050FE2EF50F0010123A92A
:108B800002D0428E01D0429E23AB02D0428C01D053
:108B9000429C23AD02D0428A01D0429A23AF02D038
:108BA000428801D0429800015CD0010123A902D083
:108BB000428601D0429623AB02D0428401D0429437
:108BC00023AD02D0428201D0429223AF02D0428034
:108BD00001D04290000145D0010123A902D0438E6B
:108BE00001D0439E23AB02D0438C01D0439C23ADE4
:108BF00002D0438A01D0439A23AF02D0438801D0E8
:108C0000439800012ED0010123A902D0438601D050
:108C1000439623AB02D0438401D0439423AD02D0CA
:108C2000438201D0439223AF02D0438001D04390CE
:108C3000000117D0010123A902D0448E01D0449E27
:108C400023AB02D0448C01D0449C23AD02D0448A93
:108C500001D0449A23AF02D0448801D04498000147
:108C600000D03E5042163F504316405044164150EB
:108C7000451601012251CD08D8A48DD0A09281982B
:108C8000819A0001BA8301012351070B0001B96FDA
:108C9000B951FB0FD8B076D0050FF4EF50F00101B9
:108CA00023A902D05D8E01D05D9E23AB02D05D8CE6
:108CB00001D05D9C23AD02D05D8A01D05D9A23AFC7
:108CC00002D05D8801D05D9800015CD0010123A92C
:108CD00002D05D8601D05D9623AB02D05D8401D0C9
:108CE0005D9423AD02D05D8201D05D9223AF02D0AE
:108CF0005D8001D05D90000145D0010123A902D023
:108D00005E8E01D05E9E23AB02D05E8C01D05E9C55
:108D100023AD02D05E8A01D05E9A23AF02D05E8876
:108D200001D05E9800012ED0010123A902D05E86F9
:108D300001D05E9623AB02D05E8401D05E9423AD59
:108D400002D05E8201D05E9223AF02D05E8001D05D
:108D50005E90000117D0010123A902D05F8E01D0DF
:108D60005F9E23AB02D05F8C01D05F9C23AD02D00D
:108D70005F8A01D05F9A23AF02D05F8801D05F98ED
:108D8000000100D03E505D163F505E1640505F1609
:108D90004150601601012251DD08D8A48DD0A09267
:108DA0008198819A0001BA8301012351070B0001C8
:108DB000B96FB951FB0FD8B076D0050F06EF51F05F
:108DC000010123A902D0618E01D0619E23AB02D0A4
:108DD000618C01D0619C23AD02D0618A01D0619A7F
:108DE00023AF02D0618801D0619800015CD00101FD
:108DF00023A902D0618601D0619623AB02D06184A1
:108E000001D0619423AD02D0618201D0619223AF81
:108E100002D0618001D06190000145D0010123A9F9
:108E200002D0628E01D0629E23AB02D0628C01D050
:108E3000629C23AD02D0628A01D0629A23AF02D035
:108E4000628801D0629800012ED0010123A902D0CE
:108E5000628601D0629623AB02D0628401D0629414
:108E600023AD02D0628201D0629223AF02D0628031
:108E700001D06290000117D0010123A902D0638EB6
:108E800001D0639E23AB02D0638C01D0639C23ADE1
:108E900002D0638A01D0639A23AF02D0638801D0E5
:108EA0006398000100D03E5061163F50621640505A
:108EB00063164150641601012251ED08D8A48DD0EB
:108EC000A0928198819A0001BA8301012351070B76
:108ED0000001B96FB951FB0FD8B076D0050F18EF6C
:108EE00051F0010123A902D0658E01D0659E23AB0C
:108EF00002D0658C01D0659C23AD02D0658A01D07B
:108F0000659A23AF02D0658801D0659800015CD0D6
:108F1000010123A902D0658601D0659623AB02D05A
:108F2000658401D0659423AD02D0658201D065923D
:108F300023AF02D0658001D06590000145D00101CA
:108F400023A902D0668E01D0669E23AB02D0668C28
:108F500001D0669C23AD02D0668A01D0669A23AF09
:108F600002D0668801D0669800012ED0010123A9A5
:108F700002D0668601D0669623AB02D0668401D00B
:108F8000669423AD02D0668201D0669223AF02D0F0
:108F9000668001D06690000117D0010123A902D09C
:108FA000678E01D0679E23AB02D0678C01D0679C8F
:108FB00023AD02D0678A01D0679A23AF02D06788B9
:108FC00001D06798000100D03E5065163F506616EC
:108FD0004050671641506816010122511E08D8A45E
:108FE0008DD0A0928198819A0001BA83010123510A
:108FF000070B0001B96FB951FB0FD8B076D0050F40
:109000002AEF51F0010123A902D0698E01D0699E97
:1090100023AB02D0698C01D0699C23AD02D0698A50
:1090200001D0699A23AF02D0698801D06998000104
:109030005CD0010123A902D0698601D0699623ABD7
:1090400002D0698401D0699423AD02D0698201D035
:10905000699223AF02D0698001D06990000145D0A8
:10906000010123A902D06A8E01D06A9E23AB02D0EF
:109070006A8C01D06A9C23AD02D06A8A01D06A9AB8
:1090800023AF02D06A8801D06A9800012ED0010176
:1090900023A902D06A8601D06A9623AB02D06A84E3
:1090A00001D06A9423AD02D06A8201D06A9223AFC4
:1090B00002D06A8001D06A90000117D0010123A973
:1090C00002D06B8E01D06B9E23AB02D06B8C01D093
:1090D0006B9C23AD02D06B8A01D06B9A23AF02D078
:1090E0006B8801D06B98000100D03E5069163F504C
:1090F0006A1640506B1641506C1601012251AE08A1
:10910000D8A4BFD0A0928198819A0001BA850101AC
:109110002351070B0001B96FB951FB0FD8B0A8D08C
:10912000050F3CEF51F0010123A903D00001948FFA
:1091300002D00001949F010123AB03D00001948D64
:1091400002D00001949D010123AD03D00001948B56
:1091500002D00001949B010123AF03D00001948948
:1091600002D00001949984D0010123A903D0000109
:10917000948702D000019497010123AB03D0000132
:10918000948502D000019495010123AD03D0000124
:10919000948302D000019493010123AF03D0000116
:1091A000948102D00001949163D0010123A903D0DE
:1091B0000001958F02D00001959F010123AB03D0E0
:1091C0000001958D02D00001959D010123AD03D0D2
:1091D0000001958B02D00001959B010123AF03D0C4
:1091E0000001958902D00001959942D0010123A97F
:1091F00003D00001958702D000019597010123ABB0
:1092000003D00001958502D000019595010123ADA1
:1092100003D00001958302D000019593010123AF93
:1092200003D00001958102D00001959121D0010168
:1092300023A903D00001968F02D00001969F01015F
:1092400023AB03D00001968D02D00001969D010151
:1092500023AD03D00001968B02D00001969B010143
:1092600023AF03D00001968902D00001969900D067
:109270007150941772509517735096177450971732
:1092800001012251BE08D8A4BFD0A0928198819A32
:109290000001BA8501012351070B0001B96FB951D3
:1092A000FB0FD8B0A8D0050F4EEF51F0010123A954
:1092B00003D00001988F02D00001989F010123ABD9
:1092C00003D00001988D02D00001989D010123ADCB
:1092D00003D00001988B02D00001989B010123AFBD
:1092E00003D00001988902D00001989984D001012F
:1092F00023A903D00001988702D0000198970101AB
:1093000023AB03D00001988502D00001989501019C
:1093100023AD03D00001988302D00001989301018E
:1093200023AF03D00001988102D00001989163D04F
:10933000010123A903D00001998F02D00001999F58
:10934000010123AB03D00001998D02D00001999D4A
:10935000010123AD03D00001998B02D00001999B3C
:10936000010123AF03D00001998902D0000199992E
:1093700042D0010123A903D00001998702D0000146
:109380009997010123AB03D00001998502D0000118
:109390009995010123AD03D00001998302D000010A
:1093A0009993010123AF03D00001998102D00001FC
:1093B000999121D0010123A903D000019A8F02D0F5
:1093C00000019A9F010123AB03D000019A8D02D0C6
:1093D00000019A9D010123AD03D000019A8B02D0B8
:1093E00000019A9B010123AF03D000019A8902D0AA
:1093F00000019A9900D071509817725099177350C4
:109400009A1774509B1701012251CE08D8A4BFD0DF
:10941000A0928198819A0001BA8501012351070B1E
:109420000001B96FB951FB0FD8B0A8D0050F60EF9C
:1094300051F0010123A903D000019C8F02D000014B
:109440009C9F010123AB03D000019C8D02D0000141
:109450009C9D010123AD03D000019C8B02D0000133
:109460009C9B010123AF03D000019C8902D0000125
:109470009C9984D0010123A903D000019C8702D0CC
:1094800000019C97010123AB03D000019C8502D011
:1094900000019C95010123AD03D000019C8302D003
:1094A00000019C93010123AF03D000019C8102D0F5
:1094B00000019C9163D0010123A903D000019D8F7D
:1094C00002D000019D9F010123AB03D000019D8DBF
:1094D00002D000019D9D010123AD03D000019D8BB1
:1094E00002D000019D9B010123AF03D000019D89A3
:1094F00002D000019D9942D0010123A903D00001AF
:109500009D8702D000019D97010123AB03D000018C
:109510009D8502D000019D95010123AD03D000017E
:109520009D8302D000019D93010123AF03D0000170
:109530009D8102D000019D9121D0010123A903D07A
:1095400000019E8F02D000019E9F010123AB03D03A
:1095500000019E8D02D000019E9D010123AD03D02C
:1095600000019E8B02D000019E9B010123AF03D01E
:1095700000019E8902D000019E9900D071509C1775
:1095800072509D1773509E1774509F1701012251FE
:10959000DE08D8A4BFD0A0928198819A0001BA8534
:1095A00001012351070B0001B96FB951FB0FD8B06E
:1095B000A8D0050F72EF51F0010123A903D00001DB
:1095C000A08F02D00001A09F010123AB03D00001B6
:1095D000A08D02D00001A09D010123AD03D00001A8
:1095E000A08B02D00001A09B010123AF03D000019A
:1095F000A08902D00001A09984D0010123A903D041
:109600000001A08702D00001A097010123AB03D085
:109610000001A08502D00001A095010123AD03D077
:109620000001A08302D00001A093010123AF03D069
:109630000001A08102D00001A09163D0010123A903
:1096400003D00001A18F02D00001A19F010123AB33
:1096500003D00001A18D02D00001A19D010123AD25
:1096600003D00001A18B02D00001A19B010123AF17
:1096700003D00001A18902D00001A19942D00101CB
:1096800023A903D00001A18702D00001A197010105
:1096900023AB03D00001A18502D00001A1950101F7
:1096A00023AD03D00001A18302D00001A1930101E9
:1096B00023AF03D00001A18102D00001A19121D0EC
:1096C000010123A903D00001A28F02D00001A29FB3
:1096D000010123AB03D00001A28D02D00001A29DA5
:1096E000010123AD03D00001A28B02D00001A29B97
:1096F000010123AF03D00001A28902D00001A29989
:1097000000D07150A0177250A1177350A217745057
:10971000A31701012251EE08D8A4BFD0A0928198CE
:10972000819A0001BA8501012351070B0001B96F2D
:10973000B951FB0FD8B0A8D0050F84EF51F001014B
:1097400023A903D00001A48F02D00001A49F01012E
:1097500023AB03D00001A48D02D00001A49D010120
:1097600023AD03D00001A48B02D00001A49B010112
:1097700023AF03D00001A48902D00001A49984D0B2
:10978000010123A903D00001A48702D00001A497FE
:10979000010123AB03D00001A48502D00001A495F0
:1097A000010123AD03D00001A48302D00001A493E2
:1097B000010123AF03D00001A48102D00001A491D4
:1097C00063D0010123A903D00001A58F02D00001BD
:1097D000A59F010123AB03D00001A58D02D000019C
:1097E000A59D010123AD03D00001A58B02D000018E
:1097F000A59B010123AF03D00001A58902D0000180
:10980000A59942D0010123A903D00001A58702D068
:109810000001A597010123AB03D00001A58502D06B
:109820000001A595010123AD03D00001A58302D05D
:109830000001A593010123AF03D00001A58102D04F
:109840000001A59121D0010123A903D00001A68F19
:1098500002D00001A69F010123AB03D00001A68D19
:1098600002D00001A69D010123AD03D00001A68B0B
:1098700002D00001A69B010123AF03D00001A689FD
:1098800002D00001A69900D07150A4177250A517FC
:109890007350A6177450A717010122512E08D8A49F
:1098A000BED0A0928198819A0001BA85010123510E
:1098B000070B0001B96FB951FB0FD8B0A8D0050F45
:1098C00096EF51F0010123A903D00001A88F02D027
:1098D0000001A89F010123AB03D00001A88D02D095
:1098E0000001A89D010123AD03D00001A88B02D087
:1098F0000001A89B010123AF03D00001A88902D079
:109900000001A89984D0010123A903D00001A887F0
:1099100002D00001A897010123AB03D00001A88564
:1099200002D00001A895010123AD03D00001A88356
:1099300002D00001A893010123AF03D00001A88148
:1099400002D00001A89163D0010123A903D0000136
:10995000A98F02D00001A99F010123AB03D0000110
:10996000A98D02D00001A99D010123AD03D0000102
:10997000A98B02D00001A99B010123AF03D00001F4
:10998000A98902D00001A99942D0010123A903D0DD
:109990000001A98702D00001A997010123AB03D0E0
:1099A0000001A98502D00001A995010123AD03D0D2
:1099B0000001A98302D00001A993010123AF03D0C4
:1099C0000001A98102D00001A99121D0010123A9A0
:1099D00003D00001AA8F02D00001AA9F010123AB8E
:1099E00003D00001AA8D02D00001AA9D010123AD80
:1099F00003D00001AA8B02D00001AA9B010123AF72
:109A000003D00001AA8902D00001AA9900D07150A8
:109A1000A8177250A9177350AA177450AB170001FA
:109A2000BA5305E0E92D03D0A0928198819A0101F3
:109A30002251D80818E1000166EC01F001016551DE
:109A4000000808E32B2D01D005D05C51F00802E09E
:109A50005E5303E1A9EF50F004D000017AEC16F058
:109A60000101A9EF50F02251E80808E1000136ECAD
:109A70001AF0060E01015D6FA9EF50F02251F808AF
:109A800018E1000166EC01F001016551000808E3EE
:109A90002C2D01D005D05C51F00802E05E5303E1AB
:109AA000A9EF50F004D00001ABEC17F00101A9EFD1
:109AB00050F02251090808E10001C8EC19F0060E27
:109AC00001015D6FA9EF50F0225119082EE12351D9
:109AD000B90802E1010E5E6F336A000166EC01F025
:109AE00001013A2D01D002D03B2D0DD0302D04D0F4
:109AF000060E5D6F2ED306D0B90E236F0001B7ECB2
:109B00000AF0010111D06551000808E32D2D01D0A4
:109B100005D05C51F00802E05E5302E11AD304D094
:109B20000001DFEC08F0010114D3225129080CE1F7
:109B30002351B90801E15E6B335205E10001A4EC49
:109B40001AF00101819F05D32251780811E100012B
:109B500066EC01F001016551000802E32E2D02D0F0
:109B6000F8D204D0000151EC03F00101416BF1D2B5
:109B70002251880805E1000181EC0EF00101E9D2D3
:109B80002251980811E1000166EC01F001016551D4
:109B9000000802E32F2D02D0DCD204D000014CECEF
:109BA00006F00101426BD5D22251A80805E100015F
:109BB0008FEC0EF00101CDD22251B80826E13553C9
:109BC00024E1475304E12351B908D8B4306B302D58
:109BD00001D00BD0752D01D002D0762D0AD02351A3
:109BE000F90807E10851090804E1060E5D6FB1D2DA
:109BF00009D0000166EC01F0B7EC0AF0336A326A72
:109C0000316A0101416B426BA4D22251C8082CE198
:109C1000302D29D02C50CA0804E13A5322E13B539D
:109C200020E13C51020808E1755306E18FB104D0F0
:109C30005E2D02D0010E2B6F3D51020808E17653D4
:109C400006E18FB304D05E2D02D0010E2C6F476B5E
:109C5000000181EC0EF08FEC0EF00101306B060E6E
:109C60005D6F050E5B6F75D2335313E122511808F7
:109C700010E16D5304E06B5302E06C530AE1342DA4
:109C800005D0346B000161EC14F00101010E346F5A
:109C900060D22251280829E10001A2EC1BF0010149
:109CA0006D2D09D06A51180806E16D6B566B6B6B10
:109CB0006C6B696B686B352D06D06A51280803E11F
:109CC000010E826F46D2332D01D005D0312D01D047
:109CD00002D0322D05D0010E336F00014BEC19F08C
:109CE0000001FA6BFB6B010134D222516A0803E0D8
:109CF00022517A0837E1A0928198819A010E0001E1
:109D0000BA6F020E01013C6FF2CF20F2F29CF29E7C
:109D1000AA6A010EA96EA69CA69EA680A850020162
:109D200020BDF28C20BFF28E01013E6F3E513C5DA2
:109D300018E0AA6A010EA96E3CC1A8FFA69CA69EC7
:109D4000A684F250006EF29CF29E0F01550EA76E93
:109D5000AA0EA76EA682A6B2FED7A6940050F21253
:109D60000101F7D122518A0803E022519A0838E113
:109D7000A0928198819A010E0001BA6F2F80080E7F
:109D800001013C6FF2CF20F2F29CF29EAA6A010E12
:109D9000A96EA69CA69EA680A850020120BDF28CAA
:109DA00020BFF28E01013E6F3E513C5D18E0AA6A71
:109DB000010EA96E3CC1A8FFA69CA69EA684F250E7
:109DC000006EF29CF29E0F01550EA76EAA0EA76EB2
:109DD000A682A6B2FED7A6940050F2120101B9D114
:109DE0002251AA0803E02251BA083AE1A0928198D0
:109DF000819A010E0001BA6F01016451020830E13D
:109E0000020E3D6FF2CF20F2F29CF29EAA6A020E81
:109E1000A96EA69CA69EA680A850020120BDF28C29
:109E200020BFF28E01013E6F3E513D5D18E0AA6AEF
:109E3000020EA96E3DC1A8FFA69CA69EA684F25064
:109E4000006EF29CF29E0F01550EA76EAA0EA76E31
:109E5000A682A6B2FED7A6940050F212010179D1D3
:109E60002251CA0803E02251DA083BE1A09281980E
:109E7000819A010E0001BA6F2F820101645102081C
:109E800030E1080E3D6FF2CF20F2F29CF29EAA6AFA
:109E9000020EA96EA69CA69EA680A850020120BD17
:109EA000F28C20BFF28E01013E6F3E513D5D18E005
:109EB000AA6A020EA96E3DC1A8FFA69CA69EA68412
:109EC000F250006EF29CF29E0F01550EA76EAA0E84
:109ED000A76EA682A6B2FED7A6940050F212010188
:109EE00038D122512A0836E1A0928198819A010E38
:109EF0000001BA6F01013C6BF2CF20F2F29CF29E9E
:109F0000AA6A010EA96EA69CA69EA680A850020170
:109F100020BDF28C20BFF28E01013E6F3E513C5DB0
:109F200018E0AA6A010EA96E3CC1A8FFA69CA69ED5
:109F3000A684F250006EF29CF29E0F01550EA76EA1
:109F4000AA0EA76EA682A6B2FED7A6940050F21261
:109F50000101FFD022511B0839E1A0928198819A1A
:109F6000010E0001BA6F0101645102082FE13D6B3F
:109F7000F2CF20F2F29CF29EAA6A020EA96EA69C73
:109F8000A69EA680A850020120BDF28C20BFF28EB2
:109F900001013E6F3E513D5D18E0AA6A020EA96EB6
:109FA0003DC1A8FFA69CA69EA684F250006EF29C1E
:109FB000F29E0F01550EA76EAA0EA76EA682A6B23C
:109FC000FED7A6940050F2120101C3D022515808C6
:109FD0003EE1A0928198819A010E0001BA6F0101C1
:109FE000233B23510F0B3F6FF2CF20F2F29CF29EE6
:109FF000AA6A080EA96EA69CA69EA680A850020179
:10A0000020BDF28C20BFF28E0101096F092D05D011
:10A010003F51020802E3030E3F6FAA6A060EA96EC3
:10A020003FC1A8FFA69CA69EA684F2CF00F0F29C9A
:10A03000F29E0F01550EA76EAA0EA76EA682A6B2BB
:10A04000FED7A6940050F2120101086B82D0645131
:10A05000020841E1225168083EE1A0928198819A6C
:10A06000010E0001BA6F0101233B23510F0B406F1A
:10A07000F2CF20F2F29CF29EAA6A080EA96EA69C6C
:10A08000A69EA680A850020120BDF28C20BFF28EB1
:10A090000101096F092D05D04051020802E3030EAA
:10A0A000406FAA6A070EA96E40C1A8FFA69CA69E93
:10A0B000A684F2CF00F0F29CF29E0F01550EA76E1F
:10A0C000AA0EA76EA682A6B2FED7A6940050F212E0
:10A0D0000101086B3ED02251FC0803E02251FD082B
:10A0E0000AE1A0928198819A010E0001BA6FCFEC2B
:10A0F00030F001012ED001012251380803E1235133
:10A10000080804E00001FC2D0BD00101A092819809
:10A11000819A010E0001BA6FFCEC34F0010119D0F4
:10A1200001018051000815E28051030812E32C5010
:10A13000CA080FE0225148080CE12351080809E140
:10A14000A0928198819A010E0001BA6F03EF3BF053
:10A1500001017B6B0001000CE824F76AF736730FEE
:10A16000F66EA10EF7220A00F550FA6E0800F550BF
:10A17000F96E46877487A287D087FE87E824F76A3E
:10A18000F736970FF66EA10EF7220A00F550FA6E19
:10A190000800F550F96ED088FE882C895A89888984
:10A1A000E824F76AF736BB0FF66EA10EF7220A0015
:10A1B000F550FA6E0800F550F96E5A8A888AB68A08
:10A1C000E48A128BE824F76AF736DF0FF66EA10EE9
:10A1D000F7220A00F550FA6E0800F550F96E7C8BF4
:10A1E000AA8BD88B068C348CE824F76AF736030FD9
:10A1F000F66EA20EF7220A00F550FA6E0800F5502E
:10A20000F96E9E8CCC8CFA8C288D568DE824F76ADA
:10A21000F736270FF66EA20EF7220A00F550FA6EF7
:10A220000800F550F96EC08DEE8D1C8E4A8E788E2A
:10A23000E824F76AF7364B0FF66EA20EF7220A00F3
:10A24000F550FA6E0800F550F96EE28E108F3E8FD1
:10A250006C8F9A8FE824F76AF7366F0FF66EA20EAE
:10A26000F7220A00F550FA6E0800F550F96E0490D6
:10A27000329060908E90BC90E824F76AF736930F86
:10A28000F66EA20EF7220A00F550FA6E0800F5509D
:10A29000F96E26916891AA91EC912E92E824F76AC2
:10A2A000F736B70FF66EA20EF7220A00F550FA6ED7
:10A2B0000800F550F96EAC92EE9230937293B4931D
:10A2C000E824F76AF736DB0FF66EA20EF7220A00D3
:10A2D000F550FA6E0800F550F96E32947494B69405
:10A2E000F8943A95E824F76AF736FF0FF66EA20E57
:10A2F000F7220A00F550FA6E0800F550F96EB8958D
:10A30000FA953C967E96C096E824F76AF736230FB6
:10A31000F66EA30EF7220A00F550FA6E0800F5500B
:10A32000F96E3E978097C29704984698E824F76A9A
:10A33000F736470FF66EA30EF7220A00F550FA6EB5
:10A340000800F550F96EC498069948998A99CC99F5
:10A35000AA6A530EA96E87C0A8FFA69CA69EA684D3
:10A36000F2CF00F0F29CF29E0F01550EA76EAA0EDE
:10A37000A76EA682A6B2FED7A6940050F212AA6AD1
:10A38000540EA96E86C0A8FFA69CA69EA684F2CFF6
:10A3900000F0F29CF29E550EA76EAA0EA76EA68242
:10A3A000A6B2FED7A6940050F212000150EF54F06E
:10A3B00001011F2B00001F511B0802E2010E1E6F3E
:10A3C0000001000C0101251F25512419276F251FAD
:10A3D000000121EF52F001011F6B1E6B256B000184
:10A3E000E7DF01011E2D01D005D00001EA51000870
:10A3F00003E2010131D000019EAAF2D701011C6BDA
:10A400000001AEEC00F01CC125F101011F6B1E6BB9
:10A41000266B0001CDDF01011E2D01D005D000010A
:10A42000EA51000803E2010117D000019EAAF2D709
:10A43000FF0E01011C6F0001AEEC00F01CC126F103
:10A44000C1D701012751265D05E10001EA5100084D
:10A4500004E20101010E1E6F000101011F6B0001EA
:10A46000000CAB98050E006E002EFED700D0AB8816
:10A47000B2DF01011E53D8A44AD02151010A0001C4
:10A480001FE0170A1FE0010A1FE0370A1FE0010A58
:10A490001FE0170A1FE0010A1FE0770A1FE0010A08
:10A4A0001FE0170A1FE0010A1FE0370A1FE0010A38
:10A4B0001FE0170A1FE0010A1FE0F70A1FE025D07E
:10A4C000868123D0868321D086851FD086871DD0A4
:10A4D00086891BD0868B19D0868D17D0868F15D094
:10A4E000878113D0878311D087850FD087870DD0C0
:10A4F00087890BD0878B09D0878D07D0878FEF5145
:10A50000020802E1030EEF6F00D00DD001012151CE
:10A5100080080AE10001EF510208D8B402D001011D
:10A5200003D0030EEF6F0101010141EF56F001016D
:10A530002251FE0824E123A103D0000186810101FC
:10A5400023A303D000018683010123A503D00001CA
:10A550008685010123A903D000018687010123AB71
:10A5600003D000018689010123AD03D00001868B51
:10A57000010123AF03D00001868D010133D0223DBC
:10A5800024D023A103D00001868F010123A303D08F
:10A5900000018781010123A503D000018783010108
:10A5A00023A903D000018785010123AB03D000015B
:10A5B0008787010123AD03D000018789010123AF03
:10A5C00003D00001878B01010DD02251FD080AE163
:10A5D00023A103D00001878D010123A303D0000133
:10A5E000878F01012251FD080EE10001EF5105089E
:10A5F000D8B002D0010107D0050EEF6F83808280B2
:10A60000839282960101010141EF56F001019F51B1
:10A61000215D22E0A051215D1FE0A151215D1CE0E0
:10A62000A251215D19E0A351215D16E0A451215DE5
:10A6300013E0AB51215D10E0AC51215D0DE0AD5157
:10A64000215D0AE0AE51215D07E0AF51215D04E0DC
:10A65000B051215DD8A4DBD00001BDDEEA51000875
:10A6600004E301011E2D03D00001D2D001019F514E
:10A67000215D0EE12551DB5D02E1E72B03D025C111
:10A68000DBF1E76BE751020803E125C1C3F1E707FE
:10A69000A051215D0EE12551DC5D02E1E82B03D0E4
:10A6A00025C1DCF1E86BE851020803E125C1C4F1E2
:10A6B000E807A151215D0EE12551DD5D02E1E92BA5
:10A6C00003D025C1DDF1E96BE951020803E125C1A1
:10A6D000C5F1E907A251215D0EE12551DE5D02E1E0
:10A6E000EA2B03D025C1DEF1EA6BEA51020803E14F
:10A6F00025C1C6F1EA07A351215D0EE12551DF5DB9
:10A7000002E1EB2B03D025C1DFF1EB6BEB5102082B
:10A7100003E125C1C7F1EB07A451215D0EE12551ED
:10A72000E05D02E1EC2B03D025C1E0F1EC6BEC51D4
:10A73000020803E125C1C8F1EC07AB51215D0EE130
:10A740002551E15D02E1ED2B03D025C1E1F1ED6B77
:10A75000ED51020803E125C1C9F1ED07AC51215DBE
:10A760000EE12551E25D02E1EE2B03D025C1E2F1BD
:10A77000EE6BEE51020803E125C1CAF1EE07AD51BF
:10A78000215D0EE12551E35D02E1EF2B03D025C1F0
:10A79000E3F1EF6BEF51020803E125C1CBF1EF07C5
:10A7A000AE51215D0EE12551E45D02E1F02B03D0B5
:10A7B00025C1E4F1F06BF051020803E125C1CCF1B1
:10A7C000F007AF51215D0EE12551E55D02E1F12B6E
:10A7D00003D025C1E5F1F16BF151020803E125C178
:10A7E000CDF1F107B051215D0EE12551E65D02E1A9
:10A7F000F22B03D025C1E6F1F26BF251020803E11E
:10A8000025C1CEF1F2078E6B0001EA6B010106D083
:10A81000010E01018E6F0001EA6B01011E6B8A9E21
:10A82000000102EF56F09EBA02D0ABA212D0AB9854
:10A830000000AB88000001010C6BAECF0BF19EBA9B
:10A84000FBD70000AB980000AB8800000C6BAECFCC
:10A850000BF10001000CCBEF00F001015A2D01D0EB
:10A8600010D20001EF5104083DE301012851215DA0
:10A8700005E100011FEC3BF0010103D22151F70873
:10A8800003E122510B0804E00001EF51030812E13B
:10A890000001EF2D01D003D0EF51030806E158D598
:10A8A000050EEF6F0101EDD10001010EEF6F010107
:10A8B000E8D10001EF2D01D003D0EF51020812E1E1
:10A8C000010122510B08D8B402D000010BD0235152
:10A8D0000A0806E023511A08D8B402D0000102D0B9
:10A8E0000001BFD501012151D7080BE12251FE081B
:10A8F00006E0223D01D003D02251FD0802E1000113
:10A9000016D60001EF51040803E30101BAD100019A
:10A91000326A316A01012151960811E122512A0857
:10A920000EE123A90CD030520AE03D50000807E2A6
:10A93000FF0A03E13C508F0802E23D6A3C6A215164
:10A94000D7080AE122513E0807E123C181F181A520
:10A950006F6B3553D8B4826B6153D8A489D1285119
:10A96000215DD8B485D12151810824E122518C0880
:10A9700021E12F521FE02FA00DD02B2D0BD02E53F5
:10A9800009E1315307E13C51080804E1000136ECCC
:10A990001AF001012FA20DD02C2D0BD02F5309E15D
:10A9A000325307E13D51080804E10001C8EC19F0F9
:10A9B00001012F6A805346E12151810843E1225170
:10A9C000E90840E1235108083DE1010E486EA092DC
:10A9D0008198819A0001FFDC01011E5332E18390CE
:10A9E000839282968290253B259F25C180F18051DC
:10A9F00000081BE28051030818E3090E7F6FC40EA4
:10AA00007E6F00018BEC01F08380839282968280BE
:10AA1000090E01017F6FC40E7E6F00018BEC01F007
:10AA200083908382828682900101130E7F6F880E4D
:10AA30007E6F00018BEC01F08380838282868280AE
:10AA400001011FD12151E108D8A494D02351080855
:10AA5000D8A490D022AF27D0F10E5C6F0001CA536A
:10AA60001EE1C82D01D002D0C92D19D00101336BD0
:10AA7000346B000161EC14F0030E01017F6FE80EEE
:10AA80007E6F00018BEC01F04BEC19F001016D6B56
:10AA9000130E7F6F880E7E6F00018BEC01F0030EAA
:10AAA000CA6F07D00101F00E5C6F0001CA53D8A431
:10AAB000CA07010122A507D0010E6F6F0001FA6BD2
:10AAC000FB6B02D001016F6B010122AB07D0010EBD
:10AAD000706F6551020801E1656B01D0706B22ADAA
:10AAE0000FD0010E466F2C50CA0809E15C51F108E5
:10AAF00006E130B004D030B202D0050E5B6F04D056
:10AB0000466B0001CD6B01018051000806E28051C7
:10AB1000030803E3010E5E6F09D05C51F10805E103
:10AB200022A103D0010E5E6F01D05E6B22A30BD079
:10AB3000010E0001FD6F0101305304E10001B7EC8B
:10AB40000AF0010109D00001FD6B010181B904D0B7
:10AB50005B51060801E15B6B5C51F0080AE1462D90
:10AB600008D00001CD53D8B402D0010102D0CD2BC2
:10AB7000010187D00001865302E1875306E00101FD
:10AB80008F530CE190530AE10001010EC76F2C5066
:10AB9000CA0803E1BB5301E0BB6B010122510B0862
:10ABA00041E123510A0803E023511A083BE18F5386
:10ABB00002E190532BE0010E0001EC6F01012151E5
:10ABC000F70818E123510A0815E10001BA53D8B477
:10ABD00002D001010FD001018E530BE100011FECE7
:10ABE0003BF0010EC76FEC6BBB51020801E1BB6B80
:10ABF000010147D0AB98030E006E002EFED7AB8844
:10AC0000000104D5EC6B01013CD00CD02C50CA08DB
:10AC100009E10001BB510208D8B402D0010102D001
:10AC2000BB6B01015C51F10816E12151E10813E011
:10AC300022510C0810E1235108080DE133530AE1B9
:10AC40006D5308E1A092346B000161EC14F0FA6BD3
:10AC5000FB6B010116D06B2D01D002D06C2D08D0FA
:10AC60002251CB0805E1696B686B6B6B6C6B09D08B
:10AC7000180E8E6F2851215D04E100011FEC3BF09E
:10AC800001010001D0DD9E9A40EF00F030B002D00B
:10AC900030A221D0462A30A007D0462C03D0839082
:10ACA000839202D08380838230A207D0462C03D0C7
:10ACB0008290829602D0828082860101756B766BCB
:10ACC000526B536B46500108D8A0466A8F0ECF6E68
:10ACD0007F0ECE6E1BD101016F2D11D084B48C700C
:10ACE00084B28B708F0ECF6E7F0ECE6E00018E53AE
:10ACF00004E1010E8E6FD2D001D08E6B02D0000124
:10AD00008E6B0101482B6B2D05D0482D02D083900E
:10AD100001D083806C2D05D0482D02D0829001D0C7
:10AD20008280312D01D002D0322D21D0485104082B
:10AD30001EE169510001915D06E310E101016851D6
:10AD40000001905D0BE2010169510001935D10E388
:10AD500005E1010168510001925D0AE301016F53B1
:10AD6000D8B402D0000104D0682BD8B4692B0001FC
:10AD7000010181A90CD0412D01D002D0422D07D074
:10AD8000496B4A6B4B6B4C6B4D6B416B426B335356
:10AD900042E12E2D40D0325005083DE303E1315011
:10ADA000DB0839E3542D01D002D0552D1BD0595169
:10ADB000040818E1412D02D08C7013D048510408CA
:10ADC00009E10001CE5305E1CF53D8A402D001011F
:10ADD00001D08C700001CE5303E1CF5301E1839089
:10ADE000010119D0412D04D0050E5B6F8C7013D07A
:10ADF0004851040809E10001CE5305E1CF53D8A41E
:10AE000002D0010101D08C700001CE5303E1CF5379
:10AE100001E183900101335342E12F2D40D03250A4
:10AE200005083DE303E13150DB0839E3542D01D03F
:10AE300002D0552D1BD05951040818E1422D02D0E3
:10AE40008B7013D04851040809E10001CE5305E18D
:10AE5000CF53D8A402D0010101D08B700001CE5392
:10AE600003E1CF5301E18290010119D0422D04D0BA
:10AE7000050E5B6F8B7013D04851040809E1000187
:10AE8000CE5305E1CF53D8A402D0010101D08B707D
:10AE90000001CE5303E1CF5301E1829001013C5305
:10AEA0000AE0545308E1752D01D002D0522D03D091
:10AEB000010E526F8C723D530AE0555308E1762D16
:10AEC00001D002D0532D03D0010E536F8B76542D39
:10AED00001D002D0552D1AD0592B482D17D03C53F4
:10AEE00005E0542D03D0010E526F8C723D5305E0E6
:10AEF000552D03D0010E536F8B76486BC30ECF6E6A
:10AF0000500ECE6E59510508D8B4596B48510308FC
:10AF100006E2040E496F486B5D5301E05D07545330
:10AF200008E1555306E16F5304E11E0ECF6EFF0E8C
:10AF3000CE6E9E90000140EF00F03250050811E304
:10AF400003E13150DB080DE3312AD8B4322A325004
:10AF5000040807E2FF0A03E13150DB0802E2010EB8
:10AF6000336E2D2A010ECC6E9E9240EF00F002014E
:10AF7000086B076B08530EE10651075D0BE20451A5
:10AF80000725E96E05510821EA6EEF6A072BD8B450
:10AF9000082BF0D7000135EF5BF00201196B163179
:10AFA0001A6F1A331A331F0E1A171A51080DF3505D
:10AFB000165D02E001E31A2B19511A5D49E3036A99
:10AFC00019511325E96E14510320EA6EEFCF1BF2DD
:10AFD000080ED8801755016EFF0E006E015204E076
:10AFE000D8900032012EFCD700501B15186F036A51
:10AFF00019511325016E1451032201C01BF203C025
:10B000001CF2036A19511325E96E14510320EA6EEC
:10B01000EFCF1EF21751016E04E0D8901E33012EBF
:10B02000FCD7080ED8801755016E1551006E0152DD
:10B0300004E0D8900036012EFCD700501E111CC22F
:10B04000EAFF1BC2E9FFEF6E18C215F2192BB4D745
:10B0500017511625016E0001000C02010737073752
:10B060000737F80E071705C209F204C208F209C231
:10B0700003F00851082BD8B4092BE96E03C0EAFF8E
:10B08000EFCF0AF20B6B010E065D0B5D4AE20C6B13
:10B090000C51070841E30ABF1ED0D8900A3709C2F5
:10B0A00003F008C2E9FF09C2EAFFEFCF0DF2070E75
:10B0B000D8800C550E6F0DC200F00E51016E04E0E9
:10B0C000D8900032012EFCD700A003D00A810A518B
:10B0D00001D00A911FD0D8900A3709C203F008C2E4
:10B0E000E9FF09C2EAFFEFCF0DF2070ED8800C5539
:10B0F0000E6F0DC200F00E51016E04E0D8900032C8
:10B10000012EFCD700A003D00A810A5101D00A9178
:10B1100007510A1B0C2BBCD7082BD8B4092B0B2BBF
:10B12000B2D70C6B0C5107080BE30ABF03D0D890C1
:10B130000A3704D0D8900A3707510A1B0C2BF2D7D4
:10B140000A31006E003200321F0E001600C001F0FE
:10B1500000018BEF5BF00201086B0631096F0933C8
:10B1600009331F0E09170951080DF350065D02E05F
:10B1700001E3092B0851095D6DE3036A08510425B9
:10B18000016E0551032201C00AF203C00BF2036AEB
:10B1900008510425E96E05510320EA6EEFCF00F057
:10B1A0000751016E04E0D8900036012EFCD7005004
:10B1B0000BC2EAFF0AC2E9FFEF6E036A08510425D9
:10B1C000016E0551032201C00AF203C00BF2036AAB
:10B1D00008510425E96E05510320EA6EEFCF0CF209
:10B1E000FF0E006E0751016E04E0D8900036012E6C
:10B1F000FCD700500C150D6F010E0825036A0425BD
:10B20000E96E05510320EA6EEFCF0FF2080ED880E9
:10B210000755016EFF0E006E015204E0D890003613
:10B22000012EFCD700500F15106F080ED88007555F
:10B23000016E1051006E015204E0D8900032012ED0
:10B24000FCD700500D110BC2EAFF0AC2E9FFEF6EF6
:10B25000082B90D70751065D016E000198EF5BF057
:10B260000201076B086B04C2E9FF05C2EAFFEFCFDA
:10B270000AF2036A07510425016E0551032203C037
:10B280000CF203C0EAFF01C0E9FFEFCF0DF2036A41
:10B2900007510425E96E05510320EA6ED890EF307E
:10B2A0000D190CC2EAFF01C0E9FFEF6E072B080E73
:10B2B00008270651085D32E2036A07510425E96E4A
:10B2C00005510320EA6EEFCF09F2036A0751042506
:10B2D000016E0551032203C00CF203C0EAFF01C056
:10B2E000E9FFEFCF0DF2036A07510425E96E05511E
:10B2F0000320EA6ED890EF300F6F006A0AB1008E1B
:10B3000000500F110D190CC2EAFF01C0E9FFEF6EEA
:10B3100009C20AF2072B080E0827CBD70651085F8F
:10B32000085314E0010E075D036A0425E96E055118
:10B330000320EA6EFF0E006E0851016E04E0D89003
:10B340000036012EFCD70050EF14EF6E0001DCEF49
:10B350005BF00201076B086B096B0A6B0B6B0C6BE4
:10B3600006310D6F0D330D331F0E0D170D51080DE6
:10B37000F350065D02E001E30D2B0D51075DD8B0DF
:10B380002AD1080E086F0853D8B4EAD00807036A18
:10B3900007510425E96E05510320EA6EEFCF0FF245
:10B3A000010E006E0851016E04E0D8900036012EA7
:10B3B000FCD700500F1503E0092B0A6B02D00A2BB3
:10B3C000096B0951020857E1085353E0036A07511A
:10B3D0000425E96E05510320EA6EEF50010B006E63
:10B3E0000B51016E04E0D8900036012EFCD70050BE
:10B3F0000C13036A07510425016E0551032201C095
:10B400000FF203C010F2036A07510425E96E0551DB
:10B410000320EA6EEFCF11F2FF0E006E0851016EAD
:10B4200004E0D8900036012EFCD700501115126FA1
:10B43000036A07510425E96E05510320EA6EEFCF38
:10B4400013F2080ED8800855016EFF0E006E0152EF
:10B4500004E0D8900032012EFCD700501315006E86
:10B46000D89000320050121110C2EAFF0FC2E9FF5B
:10B47000EF6E0B2B74D00A510A08D8A470D0085371
:10B4800062E0036A07510425E96E05510320EA6E64
:10B49000EF50010B006E0B51016E04E0D8900036A6
:10B4A000012EFCD700500C13036A07510425016ECE
:10B4B0000551032201C00FF203C010F2036A0751C5
:10B4C0000425E96E05510320EA6EEFCF11F2FF0E5D
:10B4D000006E0851016E04E0D8900036012EFCD7B2
:10B4E00000501115126F036A07510425E96E0551CA
:10B4F0000320EA6EEFCF13F2080ED8800855016ED4
:10B50000FF0E006E015204E0D8900032012EFCD7ED
:10B5100000501315006ED890003200501211156FB4
:10B52000010E085D016E010E006E015204E0D8901C
:10B530000036012EFCD70050151110C2EAFF0FC2D1
:10B54000E9FFEF6E0BD0010E006E0B51016E04E0AF
:10B55000D8900036012EFCD700500C130B2B13D7BC
:10B560000751080DF350065D07E006E30751080D8B
:10B57000F350065D0E6F02D006C20EF20B5329E0A7
:10B58000075104250F6F000E0521106F010E0F25C6
:10B59000116F000E1021126F146F11C213F20CC242
:10B5A00015F20EC216F20BC217F20001F6DC020110
:10B5B0000B51062706310D6F0D330D331F0E0D177E
:10B5C0000D51080DF350065D02E001E30D2B0B6BEE
:10B5D0000C6B072BD2D606C201F0000132EF5CF0F3
:10B5E000080E0201076F086B096B0A6B0B6B0651A3
:10B5F000095D20E20707036A08510425E96E055139
:10B600000320EA6EEFCF0DF2010E006E0751016EBE
:10B6100004E0D8900036012EFCD700500D1502E052
:10B620000B2B01D00A2B075303E1080E076F082BE1
:10B63000092BDDD70B510A5D04E2D8900B350C6F56
:10B6400002D006C20CF20CC201F0000153EF5CF014
:10B65000080E0201006F016B026B036BF8C105F26B
:10B66000F7C104F2066F000182D4F5C1E9FFF6C10B
:10B67000EAFFEFCF06F20201F8C1EAFFF7C1E9FFE6
:10B6800006C2EFFF010E0101F725016E000EF82141
:10B69000036E010E0101F525E96E000EF621EA6E3A
:10B6A000EFCF06F2020103C0EAFF01C0E9FF06C2C4
:10B6B000EFFF020E0101F725016E000EF821036E67
:10B6C000020E0101F525E96E000EF621EA6EEFCFBC
:10B6D00006F2020103C0EAFF01C0E9FF06C2EFFF64
:10B6E0000101F451010B0201046FF8C114F2F7C11A
:10B6F00013F2156F140E166F040E176F00014DDC58
:10B70000F8C105F2F7C104F2030E0201066FF9C198
:10B7100007F20001A2D401C0FBF1F8C105F2F7C1A4
:10B7200004F2180E0201066F020E076F000113D516
:10B73000020E0101F725E96E000EF821EA6EFB31D9
:10B74000006E003200321F0E00160050EF10EF6E38
:10B75000030EF725E96E000EF821EA6EFB39006E44
:10B760000036E00E001600C0EFFFF7C1E9FFF8C198
:10B77000EAFFEFCFFCF1010EF725E96E000EF8218C
:10B78000EA6EEFCFFDF1020EF725E96E000EF8210B
:10B79000EA6EEFCFFEF1030EF725E96E000EF821F9
:10B7A000EA6EEFCFFFF1F8C105F2F7C104F21B0E0C
:10B7B0000201066F000154D5020103511B0820E36A
:10B7C0000007036A01510101F725E96EF8510320D2
:10B7D000EA6EEFCF04F2010E006E02010051016E1D
:10B7E00004E0D8900036012EFCD70050041501E08B
:10B7F000022B005303E1080E006F012B032BDDD752
:10B800000251110827E20101F7C1E9FFF8C1EAFF7F
:10B81000FCC1EFFF010EF725E96E000EF821EA6E7C
:10B82000FDC1EFFF020EF725E96E000EF821EA6E6A
:10B83000FEC1EFFF030EF725E96E000EF821EA6E58
:10B84000FFC1EFFFF7C1E9FFF8C1EAFFEF50800940
:10B85000EF6E0201F8C105F2F7C104F21B0E066F8C
:10B86000000177D501C0FAF1F8C114F2F7C113F263
:10B870000201156BFAC116F2050E176F0001CDEC2F
:10B8800057F001C0FAF10101F7C1E9FFF8C1EAFF81
:10B89000EF507009EF6EF8C105F2F7C104F2FAC17A
:10B8A00006F200019DD601C0FAF10101FAC101F0D2
:10B8B0000001000C54C058F053C057F052C056F06D
:10B8C00051C055F04D505110596E4E5052105A6E95
:10B8D0004F5053105B6E505054105C6E5CC04CF077
:10B8E0005BC04BF05AC04AF059C049F00101F46BFB
:10B8F000F66B490EF56FF86BD10EF76F050EF96F09
:10B900000001A6DE01C0BCF0D1C0D9F0D2C0DAF08F
:10B91000D3C0DBF0D4C0DCF0D5C0DDF0D6C0DEF0A3
:10B92000BCC0BEF0000CAD6BB06B080EAE6FAF6B61
:10B93000D9C0ACF08F6BC551010803E2020EC06F95
:10B9400002D0030EC06F020EE86FC26B000CB36B27
:10B95000B66B080EB46FB56BDFC0B2F0B16BC551FA
:10B96000010803E2020EC16F02D0030EC16F000C8A
:10B9700078C07CF077C07BF076C07AF075C079F043
:10B980006D5075108A6F6E5076108B6F6F507710F8
:10B990008C6F705078108D6F8DC04CF08CC04BF058
:10B9A0008BC04AF08AC049F00101F46BF66B490E76
:10B9B000F56FF86BD10EF76F050EF96F000148DED9
:10B9C00001C0BDF0D1C0DFF0D2C0E0F0D3C0E1F0E3
:10B9D000D4C0E2F0D5C0E3F0D6C0E4F0BDC0BFF003
:10B9E000000C66EC01F001017F6B500E7E6F0001D0
:10B9F0008BEC01F001012B2D04D02E5302E1819636
:10BA000081882C2D04D02F5302E18098818A666BA7
:10BA1000656B000E82BA010E0201256F0101663DC1
:10BA200002D0010E656F3D0E006E002EFED7662B14
:10BA300082BA02D06553EDE02B2D03D02E53D8B43B
:10BA400081982C2D03D02F53D8B4819A655311E1DE
:10BA50007F6B140E7E6F00018BEC01F001012B2D2A
:10BA600003D02E53D8B481862C2D03D02F53D8B4B5
:10BA70008088000131EF5FF0E851010802E2010E19
:10BA8000EA6FE85302E0E82D48D0E62BD8B4E72B64
:10BA900082BA06D0E85304E1010EE86FA6EF60F029
:10BAA00082AA3BD0E82D39D0A092020EE86FE7C001
:10BAB000F5F1E6C0F4F10101F76B850EF66F0001B8
:10BAC00011EC02F002C089F001C088F089C0F5F1E4
:10BAD00088C0F4F10101F76B640EF66F0001D1EC40
:10BAE00002F002C089F001C088F088C0EBF089C084
:10BAF000F5F188C0F4F10101F76B3D0EF66F00011E
:10BB000011EC02F002C089F001C088F0FF0ED8806D
:10BB100088578957EA6BA6EF60F0E8510208D8A46D
:10BB200062D101012E53D8A4AED00001AE53D8A4E7
:10BB300002D00101A8D0AE5108080DE1AD530BE1D0
:10BB4000B05309E1010EB06FAF6BD890D890AC370D
:10BB5000D8B0AF8306D08F5304E1D890AF37030E2F
:10BB6000AF178F5306E1D890D890AC3701E3AF817F
:10BB7000AE0701012E5354E12B2D52D05150555C8C
:10BB800009E15250565C06E15350575C03E15450B2
:10BB9000585C46E08198819A2B2D01D081862C2D0E
:10BBA00001D08088000186DEBEDED1DE01012F5388
:10BBB0000FE12C2D0DD07550795C09E176507A5C3F
:10BBC00006E177507B5C03E178507C5C01E083D038
:10BBD0000001E56B82BA13D0000E82BA010E020199
:10BBE000256F3D0E006E002EFED70001E52BE53DD2
:10BBF00001D0ACD282BA02D00201F3D710D0000E2D
:10BC000082BA010E0201256F3D0E006E002EFED796
:10BC10000001E52BE53D01D095D282BAF0D77DD762
:10BC200000018F532FE1AE51010A03E0010A20E029
:10BC300029D0AD2BAD2D02D0DAC0ACF0AD51020849
:10BC400002E1DBC0ACF0AD51030802E1DCC0ACF0B6
:10BC5000AD51040802E1DDC0ACF0AD51050802E1D0
:10BC6000DEC0ACF0AD51060802E1D9C0ACF00AD09C
:10BC7000AD51060806E3080EAE6FAD51060801E1AE
:10BC8000AD6B00D001012F53D8A4AED00001B45346
:10BC9000D8A402D00101A8D0B45108080DE1B353D3
:10BCA0000BE1B65309E1010EB66FB56BD890D89091
:10BCB000B237D8B0B58306D0B15304E1D890B537C8
:10BCC000030EB517B15306E1D890D890B23701E30F
:10BCD000B581B40701012F5354E12C2D52D075507A
:10BCE000795C09E176507A5C06E177507B5C03E190
:10BCF00078507C5C46E08198819A2B2D01D081861A
:10BD00002C2D01D08088000133DE0DDE20DE010104
:10BD10002E530FE12B2D0DD05150555C09E152509F
:10BD2000565C06E15350575C03E15450585C01E007
:10BD300021D70001E56B82BA13D0000E82BA010E42
:10BD40000201256F3D0E006E002EFED70001E52B8F
:10BD5000E53D01D0FBD182BA02D00201F3D710D069
:10BD6000000E82BA010E0201256F3D0E006E002EFC
:10BD7000FED70001E52BE53D01D0E4D182BAF0D732
:10BD8000CCD60001B1532FE1B451010A03E0010AFE
:10BD900020E029D0B32BB32D02D0E0C0B2F0B351D4
:10BDA000020802E1E1C0B2F0B351030802E1E2C0CF
:10BDB000B2F0B351040802E1E3C0B2F0B351050898
:10BDC00002E1E4C0B2F0B351060802E1DFC0B2F014
:10BDD0000AD0B351060806E3080EB46FB351060843
:10BDE00001E1B36B00D001010001E8510108D8B0B6
:10BDF0005DD001012E2D01D005D03C5303E03C5114
:10BE0000080803E10001C06B01012F2D01D005D00E
:10BE10003D5303E03D51080803E10001C16B0101FE
:10BE20000001C05343E1C15341E1C25101081AE28C
:10BE3000C26BC32BC551C35D13E3C55101080AE2B0
:10BE4000C45305E1010EC46F030EC35F02D0C36B80
:10BE5000C46B01D0C36B2CEC03F0AB0EC56F01D0EB
:10BE6000C0D501D0C22BC0530DE101012B2D01D053
:10BE700002D0000107D02E53D8B402D0000102D066
:10BE800081860001C1530DE101012C2D01D002D0AA
:10BE9000000107D02F53D8B402D0000102D080880F
:10BEA00000014E0E896F200E886F50D1E8510208B4
:10BEB0003AE101012E5309E10001AFA302D00101D3
:10BEC00004D001012B2D01D081862F5309E10001FF
:10BED000B5A302D0010104D001012C2D01D080882E
:10BEE000030E0001E86F896BEBC088F082AA10D0C6
:10BEF00089C0F5F188C0F4F10101F76B030EF66F0C
:10BF0000000111EC02F002C089F001C088F006D0F7
:10BF10008837893788378937FC0E8817FF0ED88015
:10BF20008857895713D1E851030845E18198819AD0
:10BF300001012E5309E10001AFB302D0010104D089
:10BF400001012B2D01D081862F5309E10001B5B3EA
:10BF500002D0010104D001012C2D01D08088040EF3
:10BF60000001E86F896BEBC088F082AA10D089C00D
:10BF7000F5F188C0F4F10101F76B0E0EF66F0001C8
:10BF800011EC02F002C089F001C088F00FD089C026
:10BF9000F5F188C0F4F10101F76B0F0EF66F0001A7
:10BFA00011EC02F002C089F001C088F0FF0ED880C9
:10BFB00088578957CBD0E85104082DE1050EE86F6A
:10BFC000896BEBC088F001012E5310E10001AFB185
:10BFD00002D001010BD0AFB304D0AFB308D08F2D86
:10BFE00006D001012B2D02D081968188000101012C
:10BFF0002F5310E10001B5B102D001010BD0B5B350
:10C0000004D0B5B308D0B12D06D001012C2D02D03B
:10C010008098818A0001E8510508D8A492D0E56B88
:10C0200001012E5307E10001AFA102D0010102D0AE
:10C03000819801012F5307E10001B5A102D0010150
:10C0400002D0819A010182BA15D0000E82BA010E87
:10C050000201256F050E006E002EFED700D00001F4
:10C06000E52BE53D01D06ED082BA02D00101EDD7BB
:10C0700014D00101000E82BA010E0201256F050ED7
:10C08000006E002EFED700D00001E52BE53D01D06B
:10C0900059D082AA02D00101EDD7020EE86F819833
:10C0A000819AAFB306D08F5303E1010E8F6F01D099
:10C0B0008F6BB5B306D0B15303E1010EB16F01D060
:10C0C000B16B01012E531DE10001AFB109D0AFA347
:10C0D00002D0010116D08F53D8B402D0010111D083
:10C0E000BE5302E0BE070CD0BCC0BEF0AD6BB06B5F
:10C0F000080EAE6FAF6BD9C0ACF0C05301E0C00703
:10C1000001012F531CE10001B5B109D0B5A302D044
:10C11000010115D0B153D8B402D0010110D0BF53E2
:10C1200002E0BF070CD0BDC0BFF0B36BB66B080E0A
:10C13000B46FB56BDFC0B2F0C15301E0C1070001BD
:10C14000ECD404D08198819AE56BA092E85302E088
:10C15000E82D04D0FF0EB36EDC0EB26EE85101087C
:10C1600004E289C0B3FF88C0B2FFEC53D8B4EA6BD5
:10C17000ABA202D013EC54F0A1928BEF00F0F2CFFF
:10C18000F4F1F29CF29EAA6AFF0EA96EA69CA69EEE
:10C19000A680A8500101F4BDF28CF4BFF28E076FA7
:10C1A0000751380821E0075158081EE00751480898
:10C1B0001BE00751CA0818E0AA6AFF0EA96E2CC03E
:10C1C000A8FFA69CA69EA684F2CF00F0F29CF29E49
:10C1D0000F01550EA76EAA0EA76EA682A6B2FED7B5
:10C1E000A6940050F2120101076BF2CFF4F1F29C19
:10C1F000F29EAA6AA96AA69CA69EA680A850F4BD33
:10C20000F28CF4BFF28E456F455103081FE22C50AB
:10C21000CA0803E1030E456F02D0020E456FAA6AF9
:10C22000A96A45C1A8FFA69CA69EA684F2CF00F0ED
:10C23000F29CF29E0F01550EA76EAA0EA76EA68263
:10C24000A6B2FED7A6940050F2120101F2CFF4F18B
:10C25000F29CF29EAA6A010EA96EA69CA69EA680DA
:10C26000A850F4BDF28CF4BFF28E3C6F3C51020832
:10C2700001E11AD0020E3C6FAA6A010EA96E3CC100
:10C28000A8FFA69CA69EA684F2CF00F0F29CF29E88
:10C290000F01550EA76EAA0EA76EA682A6B2FED7F4
:10C2A000A6940050F2120101F2CFF4F1F29CF29E3A
:10C2B000AA6A020EA96EA69CA69EA680A850F4BDEE
:10C2C000F28CF4BFF28E3D6F3D51020801E119D0AE
:10C2D000020E3D6FAA6AA96E3DC1A8FFA69CA69E4C
:10C2E000A684F2CF00F0F29CF29E0F01550EA76ECD
:10C2F000AA0EA76EA682A6B2FED7A6940050F2128E
:10C300000101F2CFF4F1F29CF29EAA6A060EA96E28
:10C31000A69CA69EA680A850F4BDF28CF4BFF28E17
:10C320003F6F3F510F081AE2010E3F6FAA6A060ED7
:10C33000A96E3FC1A8FFA69CA69EA684F2CF00F0DE
:10C34000F29CF29E0F01550EA76EAA0EA76EA68252
:10C35000A6B2FED7A6940050F2120101F2CFF4F17A
:10C36000F29CF29EAA6A070EA96EA69CA69EA680C3
:10C37000A850F4BDF28CF4BFF28E406F40510F080C
:10C380001AE2010E406FAA6A070EA96E40C1A8FF0B
:10C39000A69CA69EA684F2CF00F0F29CF29E0F010E
:10C3A000550EA76EAA0EA76EA682A6B2FED7A694B9
:10C3B0000050F2120101F2CFF4F1F29CF29EAA6A4F
:10C3C000090EA96EA69CA69EA680A850F4BDF28C6C
:10C3D000F4BFF28E646F2C50CA08D8B47ED0F2CF6E
:10C3E000F4F1F29CF29EAA6AFF0EA96EA69CA69E8C
:10C3F000A680A850F4BDF28CF4BFF28E096F642DB4
:10C4000041D00951380802E1190E096F0951580845
:10C4100002E1290E096F0951480802E1390E096F3E
:10C42000AA6AFF0EA96E09C1A8FFA69CA69EA684B3
:10C43000F2CF00F0F29CF29E0F01550EA76EAA0EED
:10C44000A76EA682A6B2FED7A6940050F2120101F2
:10C450003D6BAA6A020EA96E3DC1A8FFA69CA69ECE
:10C46000A684F2CF00F0F29CF29E0F01550EA76E4B
:10C47000AA0EA76EA682A6B2FED7A6940050F2120C
:10C480004DD001016451020828E10951190802E167
:10C49000380E096F0951290802E1580E096F095138
:10C4A000390802E1480E096FAA6AFF0EA96E09C198
:10C4B000A8FFA69CA69EA684F2CF00F0F29CF29E56
:10C4C0000F01550EA76EAA0EA76EA682A6B2FED7C2
:10C4D000A6940050F21222D001016451020805E333
:10C4E000642D1DD02C50CA081AE1020E646FAA6A8E
:10C4F000090EA96E64C1A8FFA69CA69EA684F2CFD1
:10C5000000F0F29CF29E0F01550EA76EAA0EA76EC8
:10C51000A682A6B2FED7A6940050F2120101AA6A22
:10C52000080EA96EA86AA69CA69EA684F2CF00F06B
:10C53000F29CF29E0F01550EA76EAA0EA76EA68260
:10C54000A6B2FED7A6940050F212F2CFF4F1F29CFC
:10C55000F29EAA6A080EA96EA69CA69EA680A85066
:10C560000101F4BDF28CF4BFF28E096F092D0AD0DF
:10C570003F51040802E3050E3F6F4051040802E3F7
:10C58000050E406FF2CFF4F1F29CF29EAA6A100EF3
:10C59000A96EA69CA69EA680A850F4BDF28CF4BFFE
:10C5A000F28E676F6751010819E2676BAA6A100E75
:10C5B000A96E67C1A8FFA69CA69EA684F2CF00F034
:10C5C000F29CF29E0F01550EA76EAA0EA76EA682D0
:10C5D000A6B2FED7A6940050F2120101F2CFF4F1F8
:10C5E000F29CF29EAA6A0A0EA96EA69CA69EA6803E
:10C5F000A850F4BDF28CF4BFF28E0001906FF2CF20
:10C60000F4F1F29CF29EAA6A0D0EA96EA69CA69E5B
:10C61000A680A8500101F4BDF28CF4BFF28E000197
:10C62000926F90512E081AE2916B906BAA6A0A0ED3
:10C63000A96E90C0A8FFA69CA69EA684F2CF00F08B
:10C64000F29CF29E0F01550EA76EAA0EA76EA6824F
:10C65000A6B2FED7A6940050F212000192512E0805
:10C6600019E2936B926BAA6A0D0EA96E92C0A8FF95
:10C67000A69CA69EA684F2CF00F0F29CF29E0F012B
:10C68000550EA76EAA0EA76EA682A6B2FED7A694D6
:10C690000050F212010E01010A6F186AF2BC188CE8
:10C6A000F29CF2BE188EF29E0001CFEC30F018BC66
:10C6B000F28C18BEF28E01010A6BF2CFF4F1F29CFB
:10C6C000F29EAA6A110EA96EA69CA69EA680A850EC
:10C6D000F4BDF28CF4BFF28E186F1851010819E204
:10C6E000186BAA6A110EA96E18C1A8FFA69CA69E77
:10C6F000A684F2CF00F0F29CF29E0F01550EA76EB9
:10C70000AA0EA76EA682A6B2FED7A6940050F21279
:10C710000101000199EF67F0080E016EC250C30BD2
:10C720000110C26E0B0E006E002EFED700D001016C
:10C730000C6B0B6B010E126F1251100816E37F6B1E
:10C740000A0E7E6F00018BEC01F0C282C2B2FED7EE
:10C75000C3CF84F0C4CF85F0845101010B270001C1
:10C76000855101010C23122BE7D70C330B330C330B
:10C770000B330C330B330C330B330F0E0C17000140
:10C78000856B846B01010C5305E10B51640802E3D6
:10C79000020E286F0C5303E10B51640805E20C51A3
:10C7A000000802E3040E286F0C5303E10B51FE084E
:10C7B00005E20C51010802E3060E286F0C51010836
:10C7C00005E20C51020802E3100E286F0C5102081A
:10C7D00009E20C51030806E303E10B51980802E358
:10C7E000120E286F0C51020807E2FF0A03E10B51F9
:10C7F000980802E2140E286F186AF2BC188CF29C9A
:10C80000F2BE188EF29E000113EC54F018BCF28CAC
:10C8100018BEF28EFF0E01011C6F186AF2BC188C54
:10C82000F29CF2BE188EF29E0001AEEC00F018BC35
:10C83000F28C18BEF28E01011C53D8B402D0000154
:10C84000E9D71F6B1E6BFF0E1C6F186AF2BC188CA9
:10C85000F29CF2BE188EF29E0001AEEC00F018BC05
:10C86000F28C18BEF28EB7EC00F001011E2D03D041
:10C870000001D0D701011C53E6E11F6B1E6BFF0EB8
:10C880001C6F186AF2BC188CF29CF2BE188EF29ED5
:10C890000001AEEC00F018BCF28C18BEF28EB7ECC2
:10C8A00000F001011E2D03D00001B4D701011C517D
:10C8B0000F08E5E31CA102D0288101D028911CA318
:10C8C00002D0288B01D0289B1CA502D0288D01D036
:10C8D000289D1CA702D0288F01D0289F106B0F6BBA
:10C8E000FF0E1C6F186AF2BC188CF29CF2BE188EF8
:10C8F000F29E0001AEEC00F018BCF28C18BEF28E75
:10C9000001010F2BD8B4102B0B0E006E002EFED79A
:10C9100000D010514D0806E2FF0A03E10F511F0835
:10C9200001E225D01C53DCE1106B0F6BFF0E1C6F76
:10C93000186AF2BC188CF29CF2BE188EF29E0001AE
:10C94000AEEC00F018BCF28C18BEF28E01010F2B79
:10C95000D8B4102B0000105303E10F51270801E257
:10C9600006D01C53E3E1020E0001EF6F0101106BD2
:10C970000F6BF2CFF4F1F29CF29EAA6AFE0EA96E42
:10C98000A69CA69EA680A850F4BDF28CF4BFF28EA1
:10C99000096F2851095D18E0AA6AFE0EA96E28C128
:10C9A000A8FFA69CA69EA684F2CF00F0F29CF29E61
:10C9B0000F01550EA76EAA0EA76EA682A6B2FED7CD
:10C9C000A6940050F212010100019BEF67F0010EE6
:10C9D000EA6EF50EE96EEF500EE0020E016E006A8F
:10C9E000002EFED7012EFBD7620E006E002EFED762
:10C9F00000D0EF2EF2D7000C82A215D030B013D0A9
:10CA000030B211D001017351FA0805E33D0E006EFA
:10CA1000002EFED7732B82A205D07351F90802E2D3
:10CA2000010E756F03D00101756B736B83A414D075
:10CA300030B012D030B210D07451FA0805E33D0E78
:10CA4000006E002EFED7742B83A405D07451F90814
:10CA500002E2010E766F02D0766B746B0001B8EFC4
:10CA600073F0F86A9F909F92A2829F9AD08E0D8E4B
:10CA7000EA6AE96AB896000EAF6EA20EAC6E900E2E
:10CA8000AB6EC150C00B0F09C16E070EB46E380EED
:10CA90002C6E2D6A2E6A2F6A306A316A326A336AC6
:10CAA000346A356A3A6A3B6A3C6A3D6A466A476A52
:10CAB000486A496A4A6A4B6A4C6A4D6A4E6A4F6ACA
:10CAC000506AFF0E3E6E3F6EF00E406E416A516A34
:10CAD000526A536A546A3E6A3F6A406A416A556ABA
:10CAE000566A576A586A596A5A6A5B6A5C6A366A51
:10CAF000376A386A396A366A376A386A396A426A1E
:10CB0000436A446A456A426A436A446A456A5D6A9E
:10CB10005E6A5F6A606A616A626A636A646A656AB9
:10CB2000666A676A686A696A6A6A6B6A6C6A6D6A69
:10CB30006E6A6F6A706AFF0E716E726EF00E736EBF
:10CB4000746A756A766A776A786A796A7A6A7B6AD9
:10CB50007C6A8A6B8B6B8C6B8D6B946B956B966B15
:10CB6000976B986B996B9A6B9B6B9C6B9D6B9E6B99
:10CB70009F6BA06BA16BA26BA36BA46BA56BA66B49
:10CB8000A76BA86BA96BAA6BAB6B7D6A5B0E7E6E05
:10CB90007F6A8E6B8F6BAC6BAD6BAE6BAF6BB06B3C
:10CBA000B16BB26BB36BB46BB56BB66BB76BB86B89
:10CBB000B96BBA6BBB6BBC6BBD6BBE6BBF6B030E53
:10CBC000C06FC16FC26BC36BC46BC56BC66BC76BE9
:10CBD000C86BC96BCA6BCB6BCC6BCD6BCE6BCF6BA1
:10CBE000D06B886B896B886B896BE56BE66BE76B49
:10CBF000E86BE96BEA6BEB6BEC6BED6BEE6B806BF0
:10CC0000816B826B836B806B816B826B836B846BBC
:10CC1000856B846B856BEF6B866B876BF06BF16B51
:10CC2000866B876BF26BF36BF46BF56BF66BF76BE4
:10CC3000F86BF96B906B916B906B916B926B936B44
:10CC4000926B936BFA6BFB6BFC6BFD6BFE6BFF6B7C
:10CC50000101006B016B026B036B046B500E056FDF
:10CC6000066F076B090E086F0A6B0B6B0C6B0D6B75
:10CC70000E6B0F6B106B116B126B136B146B156BD0
:10CC8000166B176B186B196B1A6B1B6B1C6B1D6B80
:10CC90001E6B1F6B206B216B226B236B246B256B30
:10CCA000266B276B286B296B2A6B2B6B2C6B2D6BE0
:10CCB0002E6B2F6B306B316B326B336B346B356B90
:10CCC000366B376B386B396B3A6B3B6B3E6B416B3A
:10CCD000426B436B446B466B476B486B496B4A6BCB
:10CCE0004B6B4C6B4D6B3C0E4E6F010E4F6F506B90
:10CCF000516B526B536B546B556B566B576B586B38
:10CD0000596B5A6B5B6BF00E5C6F5D6B5E6B5F6BB0
:10CD1000606B616B626B636B656B666B676B686B9B
:10CD2000696B6A6B6B6B6C6B6D6B6E6B6F6B706B47
:10CD3000716B726B736B746B756B766B776B786BF7
:10CD4000796B7A6B7B6B7C6B7D6B7E6B7F6B806BA7
:10CD5000816B826B836B846B856B866B876B886B57
:10CD6000896B8A6B8B6B8C6B8D6B8E6B8F6B906B07
:10CD7000916B926B936B946B956B966B976B986BB7
:10CD8000996B9A6B9B6B9C6B9D6B9E6B9F6BA06B67
:10CD9000A16BA26BA36BA46BA56BA66BA76BA86B17
:10CDA000A96BAA6BAB6BAC6BAD6BAE6BAF6BB06BC7
:10CDB000B16BB26BB36BB46BB56BB66BB76BB86B77
:10CDC000B96BBA6BBB6BBC6BBD6BBE6BBF6BC06B27
:10CDD000C16BC26BC36BC46BC56BC66BC76BC86BD7
:10CDE000C96BCA6BCB6BCC6BCD6BCE6BCF6BD06B87
:10CDF000D16BD26BD36BD46BD56BD66BD76BD86B37
:10CE0000D96BDA6BDB6BDC6BDD6BDE6BDF6BE06BE6
:10CE1000E16BE26BE36BE46BE56BE66BE76BE86B96
:10CE2000E96BEA6BEB6BEC6BED6BEE6BEF6BF06B46
:10CE3000F16BF26BF36BCF0E926E800E936EA20EBF
:10CE4000946E0C0E956E969096829684896A060E64
:10CE50008A6E8B6A8C6A8D90C150C00B0B09C16EB3
:10CE6000C050C00B0809C06EC08EC2800C0E016E8F
:10CE7000C250C30B0110C26EB50ECD6E1E0ECF6E2A
:10CE8000FF0ECE6E780E0609CA6EFB0ECB6E010E3B
:10CE9000CC6EA50EB16EFF0EB36EDC0EB26EC00E80
:10CEA000F212130E7F6F880E7E6F00018BEC01F083
:10CEB00001010C6B0B6B010E126F1251100816E37F
:10CEC0007F6B0A0E7E6F00018BEC01F0C282C2B252
:10CED000FED7C3CF84F0C4CF85F0845101010B2766
:10CEE0000001855101010C23122BE7D70C330B33C2
:10CEF0000C330B330C330B330C330B330F0E0C177B
:10CF00000001856B846B01010C51010805E303E10D
:10CF10000B512B0801E3CDD7C150C00B0C09C16EDA
:10CF2000C050C00B0809C06EC08EC2800001BFEFA8
:10CF300060F08CEF63F0C150C00B0D09C16EC050A2
:10CF4000C00B0809C06EC08EC280C80E926E896A7E
:10CF50002C50CA0820E1E56B1E0E006E002EFED795
:10CF60000000E52BE53D01D016D082BAF5D7E56B80
:10CF70001E0E006E002EFED70000E52BE53D01D011
:10CF80000AD082AAF5D7E56BA082E853FEE0E82D2F
:10CF900001D0FBD7A092186AF2BC188CF29CF2BEAA
:10CFA000188EF29E22EC02F018BCF28C18BEF28EA3
:10CFB00039EC34F00101752D03D0010E546F02D00D
:10CFC000546B526B762D03D0010E556F02D0556B0A
:10CFD000536B83808392829682909D90010E5E6F48
:10CFE000280E296F8D800B0E7F6FB80E7E6F0001AB
:10CFF0008BEC01F084A694D0838083828286828029
:10D00000020E0101F46FFA0EF56F0001E0DC010180
:10D01000F42FF9D78390838282868280640EF56F25
:10D020000001D5DC8380839282868280640E0101B8
:10D03000F56F0001CCDC8380838282968280640E4F
:10D040000101F56F0001C3DC8380838282868290B8
:10D05000640E0101F56F0001BADC84A651D0838013
:10D06000838282968280640E0101F56F0001AFDC3D
:10D070008380839282868280640E0101F56F0001B5
:10D08000A6DC8390838282868280640E0101F56F24
:10D0900000019DDC8380838282868280020E0101F2
:10D0A000F46F960EF56F000192DC0101F42FF9D7B1
:10D0B0008380839282968280020EF46F960EF56FC3
:10D0C000000185DC0101F42FF9D7838083828286F9
:10D0D0008280020EF46F960EF56F000178DC01017C
:10D0E000F42FF9D78380839282968280020EF46FA8
:10D0F000960EF56F00016BDC0101F42FF9D70001EA
:10D100008380838282868280020E0101F46F960EF4
:10D11000F56F00015CDC0101F42FF9D77BD700012A
:10D12000C00EF2129D8AABA20FD083A60DD0186A52
:10D13000F2BC188CF29CF2BE188EF29E13EC54F0E6
:10D1400018BCF28C18BEF28E3250050808E303E1D9
:10D150003150DB0804E3EF510408D8A09D822C5025
:10D16000CA08D8A4CED1010165510208D8A402D0C2
:10D170000001C7D1375305E03853D8B402D00001BD
:10D18000C0D15C51F108D8B402D00001BAD15E2DF3
:10D1900001D002D00001B5D13553D8B402D000017E
:10D1A000B0D15B510608D8A402D00001AAD1000179
:10D1B000BB53D8A4A6D1C72DA4D101013A53D8A4FA
:10D1C00083D13B53D8A480D10001BA53D8B402D044
:10D1D00001017AD1C653D8A402D0010175D1010151
:10D1E0007053D8A471D13353D8A46ED13053D8A47E
:10D1F0006BD12E5305E1315303E12B2D01D008D023
:10D200002F53D8A461D13253D8A45ED12C2D5CD138
:10D210000001E953D8A451D19D9A9D90E56B01017D
:10D220002E5363E1315361E12B2D5FD0546A536A71
:10D23000526A516ACF2D08D03650511237505212CF
:10D240003850531239505412D02D08D04250511238
:10D25000435052124450531245505412D12D08D00D
:10D260005D5051125E5052125F5053126050541272
:10D27000D22D08D061505112625052126350531295
:10D2800064505412D32D08D065505112665052127A
:10D290006750531268505412D42D08D0695051125F
:10D2A0006A5052126B5053126C50541241C050F0DD
:10D2B00040C04FF03FC04EF03EC04DF051504D1AAF
:10D2C00052504E1A53504F1A5450501A186AF2BC0A
:10D2D000188CF29CF2BE188EF29E00015AEC5CF0A3
:10D2E00018BCF28C18BEF28E01012F536EE132533E
:10D2F0006CE12C2D6AD0786A776A766A756AD52DCA
:10D300000AD00001945175129551761296517712F8
:10D31000975178120101D62D0AD00001985175124B
:10D32000995176129A5177129B5178120101D72D9B
:10D330000AD000019C5175129D5176129E517712B0
:10D340009F5178120101D82D0AD00001A051751209
:10D35000A1517612A2517712A35178120101D92D51
:10D360000AD00001A4517512A5517612A651771268
:10D37000A75178120101DA2D0AD00001A8517512C7
:10D38000A9517612AA517712AB517812010174C0DB
:10D3900070F073C06FF072C06EF071C06DF07550B8
:10D3A0006D1A76506E1A77506F1A7850701A186A84
:10D3B000F2BC188CF29CF2BE188EF29E0001B8EC02
:10D3C0005CF018BCF28C18BEF28E010E0001C56F25
:10D3D000E96F93EC5CF00101846B186AF2BC188C65
:10D3E000F29CF2BE188EF29E000153EC01F018BCC4
:10D3F000F28C18BEF28EA7EC5CF00101856B186A06
:10D40000F2BC188CF29CF2BE188EF29E00015DEC0C
:10D4100001F018BCF28C18BEF28E2CEC03F0000E5A
:10D4200082BA010E0101F46F1E0E006E002EFED7AF
:10D4300000000001E52BE53D01D045D082BAEFD7D1
:10D44000E56B000E82BA010E0101F46F1E0E006E34
:10D45000002EFED700000001E52BE53D01D033D0C2
:10D4600082AAEFD7E56B896BEBC088F0186AF2BC33
:10D47000188CF29CF2BE188EF29E89C0F5F188C01D
:10D48000F4F10101F76B3D0EF66F000111EC02F0B3
:10D4900018BCF28C18BEF28E02C089F001C088F070
:10D4A000FF0ED8808857895789C0B3FF88C0B2FF64
:10D4B000C00EF212A082E56B05D0485203E1C00E07
:10D4C000F212A0821BD001010001E92D17D0A09219
:10D4D000E96BEA6B01018FA108D02B2D06D0819852
:10D4E00081860001B86BB76B01018FA308D02C2D8A
:10D4F00006D0819A80880001B86BB76B010102D019
:10D500000001A0920001EF51050801E309D62C505B
:10D51000CA08D8A479D101015E2D5CD06D53D8A47E
:10D5200059D081AF57D081A155D081B553D081BB9F
:10D5300051D081B34FD081B94DD081BD4BD05D5317
:10D5400049E1705347E16551020844E030B042D0F0
:10D5500030B240D084B41ED03C5102081BE13A5393
:10D5600019E1375317E1545315E1755313E1186A64
:10D57000F2BC188CF29CF2BE188EF29E00017AEC7E
:10D5800016F018BCF28C18BEF28E2CEC03F0010ED3
:10D59000C56F010184B21ED03D5102081BE13B530F
:10D5A00019E1385317E1555315E1765313E1186A21
:10D5B000F2BC188CF29CF2BE188EF29E0001ABEC0D
:10D5C00017F018BCF28C18BEF28E2CEC03F0010E92
:10D5D000C56F01016D53D8A4A8D07053D8A4A5D0AD
:10D5E00065510208D8B4A1D081B59FD081BB9DD030
:10D5F00081BD9BD030B099D030B297D0305353E139
:10D6000081B302D081A94FD081A349D081AF47D047
:10D6100081B945D0372D01D002D0382D27D0372DF4
:10D6200011D038530FE1186AF2BC188CF29CF2BE8C
:10D63000188EF29E00014CEC06F018BCF28C18BE5D
:10D64000F28E0101375311E1382D0FD0186AF2BC68
:10D65000188CF29CF2BE188EF29E000151EC03F081
:10D6600018BCF28C18BEF28E010119D0375317E1A5
:10D67000385315E1186AF2BC188CF29CF2BE188E71
:10D68000F29E0001B7EC0AF018BCF28C18BEF28EC4
:10D690000101416B426B010E476F050E5B6F81A963
:10D6A00002D0060E5B6F81B331D081B92FD04653C3
:10D6B0002DE135532BE181AF29D03250050826E307
:10D6C00003E13150DB0822E33A5320E13B531EE1F2
:10D6D0002E2D0DD086530BE1885309E1415307E10C
:10D6E000000181EC0EF0050E01015B6F336A2F2DF6
:10D6F0000DD087530BE1895309E1425307E1000143
:10D700008FEC0EF0050E01015B6F336A3250040896
:10D710000CE2FF0A03E13150DB0807E2496B4A6B78
:10D720004B6B4C6B4D6B416B426B81BB50D081A5F9
:10D730004ED081AF4CD030B04AD030B248D06551D5
:10D740000208D8B4656B84B420D031531EE13C5339
:10D750001CE037531AE10001C853D8B402D00101CC
:10D7600014D00101545311E190B50FD0186AF2BCE6
:10D77000188CF29CF2BE188EF29E000161EC14F03F
:10D7800018BCF28C18BEF28E010184B220D0325344
:10D790001EE13D531CE038531AE10001C953D8B4CF
:10D7A00002D0010114D00101555311E190B90FD0FD
:10D7B000186AF2BC188CF29CF2BE188EF29E000120
:10D7C00061EC14F018BCF28C18BEF28E010181AB32
:10D7D00019D030B017D030B215D084A402D084B2A2
:10D7E00011D035530FE1186AF2BC188CF29CF2BECE
:10D7F000188EF29E0001FCEC34F018BCF28C18BEBE
:10D80000F28E010171D0000101015E2D51D081AF76
:10D810004FD081A14DD081B54BD081BB49D081B3D0
:10D8200047D081B945D05D5343E16551020840E0DE
:10D8300030B03ED030B23CD08FB11CD090B51AD0B1
:10D8400084B418D03C51020815E1375313E1545306
:10D8500011E175530FE1186AF2BC188CF29CF2BE0C
:10D86000188EF29E00017AEC16F018BCF28C18BEED
:10D87000F28E01018FB31CD090B91AD084B218D0A7
:10D880003D51020815E1385313E1555311E1765328
:10D890000FE1186AF2BC188CF29CF2BE188EF29E50
:10D8A0000001ABEC17F018BCF28C18BEF28E01012F
:10D8B000332C1AD03250050817E303E13150DB084E
:10D8C00013E3302D11D081AF0FD041530DE14253FE
:10D8D0000BE1465308E1000181EC0EF08FEC0EF0F5
:10D8E000050E01015B6F336A332C1DD032500508E1
:10D8F0001AE303E13150DB0816E3302D14D081AF79
:10D9000002D05E5310E1336A186AF2BC188CF29CA4
:10D91000F2BE188EF29E0001A4EC1AF018BCF28C34
:10D9200018BEF28E0101805100083EE280510308CA
:10D930003BE37D2C39D05D5337E17D6A356B010EB9
:10D94000486E2E2D01D002D02F2D0FD0186AF2BCB8
:10D95000188CF29CF2BE188EF29E0001A4EC1AF014
:10D9600018BCF28C18BEF28E01015C51F1081BE16B
:10D970005E2D19D0705317E1465315E1270E7F6FC6
:10D98000100E7E6F00018BEC01F0186AF2BC188C4F
:10D99000F29CF2BE188EF29EDFEC08F018BCF28CFE
:10D9A00018BEF28E0101486A332D01D025D06F2DAB
:10D9B00001D022D0542D01D01FD0552D01D01CD024
:10D9C000522D01D019D0532D01D016D0752D01D074
:10D9D00013D0762D01D010D02E2D01D00DD02F2DAB
:10D9E00001D00AD06B2D01D007D06C2D01D004D00E
:10D9F0005D5302E130AE03D0C00EF2129D800001F3
:10DA0000905302E1915342E091510101695DD8B018
:10DA100002D000013BD008E1000190510101685D96
:10DA2000D8B002D0000132D0312D01D002D0000197
:10DA30002DD00001FA532AE101016F53D8B402D06E
:10DA4000000124D09D9A186AF2BC188CF29CF2BE98
:10DA5000188EF29E0001D3EC18F018BCF28C18BEA0
:10DA6000F28E010E01016B6F0001FA6F186AF2BCB1
:10DA7000188CF29CF2BE188EF29E13EC54F018BC77
:10DA8000F28C18BEF28EC00EF2129D8A925302E101
:10DA9000935342E093510101695DD8B002D0000177
:10DAA0003BD008E1000192510101685DD8B002D07D
:10DAB000000132D0322D01D002D000012DD0000162
:10DAC000FB532AE101016F53D8B402D0000124D0E6
:10DAD0009D9A186AF2BC188CF29CF2BE188EF29EC7
:10DAE00000015BEC18F018BCF28C18BEF28E010E2F
:10DAF00001016C6F0001FB6F186AF2BC188CF29C7C
:10DB0000F2BE188EF29E13EC54F018BCF28C18BEC4
:10DB1000F28EC00EF2129D8A83B6B6EF71F0180E27
:10DB200001018E6F0001E4EC31F09D90010E0101C6
:10DB3000616F838083828280828683B69BEF71F0DF
:10DB40006351270815E303E16251100811E383B61E
:10DB500006D0085304E1180E296F010E2A6F622BBC
:10DB6000D8B4632B3D0E006E002EFED79AEF71F0F5
:10DB70005C51F008D8A49AEF71F0116BABA20FD0F2
:10DB8000186AF2BC188CF29CF2BE188EF29E00014C
:10DB900013EC54F018BCF28C18BEF28E0101C00ECA
:10DBA000F2129D8A280E296F2A6B7F6B0A0E7E6FF8
:10DBB00000018BEC01F00101112B1151630801E30D
:10DBC000DDD7116B0D2BD8B40E2B0E5307E10D5181
:10DBD000120804E38C708C728B708B760D511308D5
:10DBE0000EE10E530CE18390839282908296130E85
:10DBF0007F6F880E7E6F00018BEC01F001010D51EB
:10DC0000140803E10E53D8B483800E5304E10D5180
:10DC10001408D8B079D00E53D8A476D00D51270867
:10DC2000D8A072D0C00EF2129D8A83A66DD00E6B62
:10DC30000D6B130E7F6F880E7E6F00018BEC01F071
:10DC40000101455304E18390838282868280452DC1
:10DC500004D083808392828682804551020804E149
:10DC600083808382829682804551030804E1838009
:10DC700083828286829083B61BD02C50CA0818E01B
:10DC8000455303E1010E456F0FD0452D03D0020E21
:10DC9000456F0AD04551020803E1030E456F04D0D9
:10DCA00045510308D8B4456B0E6B0D6B83A6FCD7AA
:10DCB0000D2BD8B40E2B7F6B0A0E7E6F00018BEC00
:10DCC00001F001010D51B8081EE10E510B081BE1D6
:10DCD0000E6B0D6BAA6AA96A45C1A8FFA69CA69EF9
:10DCE000A684F2CF00F0F29CF29E0F01550EA76EB3
:10DCF000AA0EA76EA682A6B2FED7A6940050F21274
:10DD0000D9EF71F001019DD70D51280803E10E53A1
:10DD1000D8B483820E5304E10D512808D8B0EFD057
:10DD20000E53D8A4ECD00D513B08D8A0E8D0C00EBB
:10DD3000F2129D8A83A6E3D00E6B0D6B106B0F6BF6
:10DD4000130E7F6F880E7E6F00018BEC01F0F2CF17
:10DD5000F4F1F29CF29EAA6AFF0EA96EA69CA69E02
:10DD6000A680A8500101F4BDF28CF4BFF28E2C6E97
:10DD7000F2CFF4F1F29CF29EAA6A100EA96EA69C54
:10DD8000A69EA680A850F4BDF28CF4BFF28E676FF9
:10DD9000675302E1828001D082902C50CA0803E0D0
:10DDA0002C5038080CE12C50380803E18390838212
:10DDB00082862C50CA0803E18380839282862C508D
:10DDC000580803E18390839282862C50480803E12F
:10DDD00083808392829683B662D00E6B0D6B0F2B7D
:10DDE000D8B4102B7F6B0A0E7E6F00018BEC01F014
:10DDF00001011051040840E2FF0A03E10F51DB0862
:10DE00003BE20F5140080BE11051060808E10D2BD1
:10DE1000D8B40E2B8B70050E106FDC0E0F6F0D51EA
:10DE200014082AE10E5328E1106B0F6B675302E1CF
:10DE3000828001D082900F2BD8B4102B7F6B0A0EFA
:10DE40007E6F00018BEC01F001010F51DC080BE14A
:10DE50001051050808E1675303E1010E676F01D017
:10DE6000676B106B0F6B83A606D00E6B0D6B106B80
:10DE7000020E0F6F10D0DAD783A6B1D71051020867
:10DE80000AE2FF0A03E10F51E70805E20E6B0D6B92
:10DE9000106B0F6B00D00E6B0D6B83A6FCD70D2B98
:10DEA000D8B40E2B7F6B0A0E7E6F00018BEC01F055
:10DEB00001010D51B80822E10E510B081FE10E6B54
:10DEC0000D6BAA6A100EA96E67C1A8FFA69CA69E3C
:10DED000A684F2CF00F0F29CF29E0F01550EA76EC1
:10DEE000AA0EA76EA682A6B2FED7A6940050F21282
:10DEF0000101106B0F6B0F015CD2010149D70D516D
:10DF00003C0803E10E53D8B482860E5304E10D5150
:10DF10003C08D8B075D00E53D8A472D00D514F081C
:10DF2000D8A06ED0C00EF2129D8A83A669D00E6B67
:10DF30000D6B8390839282868280185303E1010ED9
:10DF4000196F02D0020E196F130E7F6F880E7E6F4D
:10DF500000018BEC01F00101192D04D08390838224
:10DF6000828682801951020804E18380839282862E
:10DF7000828083B60FD0192D03D0020E196F06D000
:10DF80001951020803E1010E196F00D00E6B0D6BE1
:10DF900083A6FCD70D2BD8B40E2B7F6B0A0E7E6F99
:10DFA00000018BEC01F001010E510A0828E2FF0A82
:10DFB00003E10D51B70823E20E6B0D6B192D01D053
:10DFC000186B1951020802E1010E186FAA6A110EAE
:10DFD000A96E18C1A8FFA69CA69EA684F2CF00F049
:10DFE000F29CF29E0F01550EA76EAA0EA76EA68296
:10DFF000A6B2FED7A6940050F212DBD10101ACD735
:10E000000D51500803E10E53D8B482800E5304E141
:10E010000D515008D8B07CD10E53D8A479D10D51F0
:10E020006308D8A075D1C00EF2129D8A83A670D164
:10E030000E6B0D6B130E7F6F880E7E6F00018BECE5
:10E0400001F0F2CFF4F1F29CF29EAA6A080EA96EDA
:10E05000A69CA69EA680A8500101F4BDF28CF4BF38
:10E06000F28E096FF2CFF4F1F29CF29EAA6A090EC9
:10E07000A96EA69CA69EA680A850F4BDF28CF4BF03
:10E08000F28E646F106B640E0F6F095302E1839080
:10E090008382092D02D08380839283B696D08296A4
:10E0A0006451020802E1829001D08280095303E1A9
:10E0B000010E096F03D0092D01D0096B2C50CA083D
:10E0C000D8B47CD00D2BD8B40E2B7F6B0A0E7E6F8C
:10E0D00000018BEC01F001010D51D008D8A46CD0E7
:10E0E0000E510708D8A468D082966451020804E152
:10E0F000090E086F829002D0086B8280270E7F6F16
:10E10000100E7E6F00018BEC01F083B60BD0010185
:10E110006451020803E1010E646F02D0020E646FC5
:10E12000E3D70001F2CFF4F1F29CF29EAA6AFF0E4F
:10E13000A96EA69CA69EA680A8500101F4BDF28CF3
:10E14000F4BFF28E2C6E642D10D02C50380802E1F2
:10E15000190E2C6E2C50580802E1290E2C6E2C50F2
:10E16000480802E1390E2C6E0FD02C50190802E13C
:10E17000380E2C6E2C50290802E1580E2C6E2C50B3
:10E18000390802E1480E2C6EAA6AFF0EA96E2CC057
:10E19000A8FFA69CA69EA684F2CF00F0F29CF29E59
:10E1A0000F01550EA76EAA0EA76EA682A6B2FED7C5
:10E1B000A6940050F212010183A684D783A6FED74D
:10E1C0000E6B0D6B106B640E0F6F0D2BD8B40E2BF6
:10E1D0007F6B0A0E7E6F00018BEC01F001010F5185
:10E1E0000D5D0EE110510E5D0BE1640E0F27000E68
:10E1F00010238B766451020802E18B7001D082807B
:10E200000D51B808D8A483D00E510B08D8A47FD0E4
:10E210000E6B0D6BAA6A080EA96E09C1A8FFA69C19
:10E22000A69EA684F2CF00F0F29CF29E0F01550E3E
:10E23000A76EAA0EA76EA682A6B2FED7A69400501D
:10E24000F212AA6A090EA96E64C1A8FFA69CA69E36
:10E25000A684F2CF00F0F29CF29E550EA76EAA0E95
:10E26000A76EA682A6B2FED7A6940050F2120101B4
:10E27000642D19D03D6BAA6A020EA96E3DC1A8FF9C
:10E28000A69CA69EA684F2CF00F0F29CF29E0F01FF
:10E29000550EA76EAA0EA76EA682A6B2FED7A694AA
:10E2A0000050F2120101496B4A6B4B6B4C6B4D6B8A
:10E2B000F2CFF4F1F29CF29EAA6A060EA96EA69C19
:10E2C000A69EA680A850F4BDF28CF4BFF28E3F6FDC
:10E2D000F2CFF4F1F29CF29EAA6A070EA96EA69CF8
:10E2E000A69EA680A850F4BDF28CF4BFF28E406FBB
:10E2F000092D0AD03F51040802E3050E3F6F40513B
:10E30000040802E3050E406F0F0153D00101BDD692
:10E310000E5303E10D5163080CE2839083928290C7
:10E320008296C00EF2129D8A83A6FBD70F0141D0C0
:10E33000010103D419D0636B626B0E6B0D6B83808C
:10E3400083828280828600011EEC34F0186AF2BC5F
:10E35000188CF29CF2BE188EF29E13EC54F018BC8E
:10E36000F28C18BEF28E010123D000010101636B13
:10E37000626B0E6B0D6B295118081AE1085318E1F6
:10E3800000011EEC34F0186AF2BC188CF29CF2BE4C
:10E39000188EF29E13EC54F018BCF28C18BEF28E5C
:10E3A0000101616B866B876B180E8E6F839282966C
:10E3B00029D00101636B626B0E6B0D6B83808280D1
:10E3C00000011EEC34F00101616B866B876B180E47
:10E3D0008E6F2C50CA0813E19D9A9D90A092000167
:10E3E0002CEC03F0010EC56F030E01017F6FE80EE8
:10E3F0007E6F00018BEC01F0A8EF67F003D0000105
:10E4000090EF68F00001BA5301E0B0D101013C5334
:10E41000D8B496D029512808D8A492D03753D8A47C
:10E420008FD07553D8A48CD05253D8A489D030B093
:10E4300087D02B2D01D005D02E2D01D002D0312D2B
:10E440007FD084B463D0372D01D05FD02C50CA0860
:10E450000CE17151310809E2A0928198819A2B2D2B
:10E4600001D081862C2D01D080887F6B140E7E6FA9
:10E4700000018BEC01F001017151F908D8B0712B4A
:10E4800084B43FD07151F9083CE25F2B2B2D01D0B1
:10E4900002D02E2D04D082AA02D0010E1A6F5F5135
:10E4A000C80801E389D05F6B2B2D01D002D02E2D3F
:10E4B00006D01A5303E06551000801E27DD01A6BC3
:10E4C0008392312D05D0010E0001C86F04D00101E7
:10E4D000010E376F0001839E01012B6B2E6B316B98
:10E4E0002C5301E12D6B2C50CA0803E02F53D8B4F4
:10E4F000306B372D06D0382D01D002D02F53D8B431
:10E500005B6B000190EF68F0010119D03A5315E1FF
:10E510000001CB53D8B402D001010FD0325005080E
:10E52000D8B002D0010109D006E13150DB08D8B0E3
:10E5300002D0010102D083820101376B716B0000B0
:10E540003C5317E0375315E13A2D01D00CD00001B0
:10E55000C82D03D0010107D00001CB2D01D002D07E
:10E56000010107D00101755304E1525302E130A0CB
:10E5700083922951280820E137531EE10001C85336
:10E58000D8B402D0010118D001013A5315E10001BD
:10E59000CB53D8B402D001010FD0010175530CE167
:10E5A00052530AE130B008D03250050805E303E1C8
:10E5B0003150DB08D8B083823D53D8B49AD029516A
:10E5C0002808D8A496D03853D8A493D07653D8A48A
:10E5D00090D05353D8A48DD030B28BD02C2D01D0F5
:10E5E00005D02F2D01D002D0322D83D084B267D038
:10E5F000382D01D063D02C50CA080CE1725131087B
:10E6000009E2A0928198819A2B2D01D081862C2D30
:10E6100001D080887F6B140E7E6F00018BEC01F0BF
:10E6200001017251F908D8B0722B84B243D07251F3
:10E63000F90840E2602B2C2D01D002D02F2D04D000
:10E6400082AA02D0010E1A6F6051C80803E30001CC
:10E650008DD00101606B2C2D01D002D02F2D08D060
:10E660001A5303E06551000803E200017FD0010165
:10E670001A6B8296322D05D0010E0001C96F04D0AD
:10E680000101010E386F0001819001012C6B2F6B8D
:10E69000326B2B5301E12D6B2C50CA0803E02E5333
:10E6A000D8B4306B382D06D0372D01D002D02E5380
:10E6B000D8B45B6B000190EF68F0010119D03B53B7
:10E6C00015E10001CC53D8B402D001010FD0325073
:10E6D0000508D8B002D0010109D006E13150DB08AD
:10E6E000D8B002D0010102D082860101386B726B72
:10E6F00000003D5317E0385315E13B2D01D00CD0FD
:10E700000001C92D03D0010107D00001CC2D01D09B
:10E7100002D0010107D00101765304E1535302E115
:10E7200030A282962951280820E138531EE10001C9
:10E73000C953D8B402D0010118D001013B5315E1EF
:10E740000001CC53D8B402D001010FD0010176539F
:10E750000CE153530AE130B208D03250050805E30A
:10E7600003E13150DB08D8B082860001FCEF64F091
:10E7700083A629D00101752D01D00BD0762D01D0B3
:10E7800008D0542D01D005D0552D01D002D0000164
:10E790001AD0C00EF2129D80752D01D0546B762DCB
:10E7A00001D0556B315305E1755303E15453D8B48F
:10E7B000526B325305E1765303E15553D8B4536B92
:10E7C00048D047D0000101012E5311E12F530FE132
:10E7D00052530DE153530BE130BE09D00001EF510C
:10E7E0000508D8A002D0010102D09D900101522D50
:10E7F00007D0315305E1755303E15453D8B4526B3C
:10E80000532D07D0325305E1765303E15553D8B465
:10E81000536B3C530AE0755302E0525306E183A662
:10E8200004D0372D02D030A083923D530AE07653B6
:10E8300002E0535306E183A604D0382D02D030A263
:10E84000829683A606D0522D01D002D0532D01D03E
:10E85000A0D72951280825E184B423D0375321E1DA
:10E8600075531FE152531DE183A61BD03A5319E1A2
:10E870000001CB53D8B402D0010113D030A002D094
:10E8800001010FD032500508D8B002D0010109D0E3
:10E8900006E13150DB08D8B002D0010102D08382FA
:10E8A00001012951280825E184B223D0385321E100
:10E8B00076531FE153531DE183A61BD03B5319E14F
:10E8C0000001CC53D8B402D0010113D030A202D041
:10E8D00001010FD032500508D8B002D0010109D093
:10E8E00006E13150DB08D8B002D0010102D08286A7
:10E8F0000101502BD8B4512B83A6B5D084B402D0DB
:10E9000084A2B1D02E2D01D002D02F2D34D0C00E34
:10E91000F2129D802E530AE12B5308E184B406D0F5
:10E9200030B004D03753D8B483800CD02B2D01D015
:10E9300002D0312D07D084A405D02E5303E130B08E
:10E9400001D083902F530AE12C5308E184B206D002
:10E9500030B204D03853D8B482800CD02C2D01D0E2
:10E9600002D0322D07D084A205D02F5303E130B25C
:10E9700001D0829064D06F534CE10001EF51050843
:10E98000D8A002D0010145D084A421D00101375381
:10E990001BE10001C853D8B402D0010115D0010118
:10E9A000315312E12E5310E12B530EE1355026085E
:10E9B00008E2FF0A03E134500F0803E23080308E92
:10E9C00003D0342AD8B4352A30A08390000184A221
:10E9D00021D0010138531BE10001C953D8B402D042
:10E9E000010115D00101325312E12F5310E12C53D4
:10E9F0000EE13B50260808E2FF0A03E13A500F08F7
:10EA000003E23082308E03D03A2AD8B43B2A30A2B7
:10EA10008290000183A612D084B407D030A002D027
:10EA2000838083823090356A346A84B207D030A202
:10EA300002D08280828630923B6A3A6A01012E536C
:10EA400011E12F530FE152530DE153530BE130BE4F
:10EA500009D00001EF510508D8A002D0010102D071
:10EA60009D90010129D083A612D084B407D030A094
:10EA700002D0838083823090356A346A84B207D0B2
:10EA800030A202D08280828630923B6A3A6A525328
:10EA900013E1535311E130530FE12E530DE12F5386
:10EAA0000BE130BE09D00001EF510508D8A002D01B
:10EAB000010102D09D900101752D01D005D0522D8C
:10EAC00001D002D0542D02D0308801D03098762D5C
:10EAD00001D005D0532D01D002D0552D02D0308A5F
:10EAE00001D0309A372D01D004D00001C82D05D0B7
:10EAF00001013084308E03D0000130940101382DA3
:10EB000001D004D00001C92D05D001013086308E1E
:10EB100003D000013096010130B00FD030B20DD0DB
:10EB200030B40BD030B609D030B807D030BA05D0E9
:10EB300030BC03D0309E3D6A3C6A83A63ED0515320
:10EB400028E15051C80825E30001EF510508D8A07D
:10EB500002D001011ED084B40CD001016B53D8B493
:10EB600002D0000106D030A002D0000102D0839074
:10EB7000000184B20CD001016C53D8B402D0000162
:10EB800006D030A202D0000102D08290000116D03F
:10EB900001015051100805E15151270802E1516B64
:10EBA000506B84B404D06B5302E130A0838084B2F4
:10EBB00004D06C5302E130A282800001325004087C
:10EBC00043E2FF0A03E13150DB083EE2010130532A
:10EBD00011E1186AF2BC188CF29CF2BE188EF29EFB
:10EBE0000001B7EC0AF018BCF28C18BEF28E010ED0
:10EBF0000101306F2D50280828E22E2A2D6A2E5050
:10EC0000010A000107E0030A0AE0010A0DE0070A11
:10EC100010E015D0839083828286828015D0838015
:10EC200083928286828010D08380838282968280C3
:10EC30000BD083808382828682902E6A05D0838067
:10EC400083828286828000D00101332D01D002D0E0
:10EC5000342D01D002D22E53D8B4416B2F53D8B4E7
:10EC6000426B412D03D02E2D01D004D0422DDED198
:10EC70002F2DDCD149510408D8A4D8D1F2CFF4F11A
:10EC8000F29CF29EAA6A080EA96EA69CA69EA68079
:10EC9000A850F4BDF28CF4BFF28E096F0953D8A4CA
:10ECA000DED03C53D8B46CD0412D6AD04E514A5D71
:10ECB000D8A066D0412D03D02E2D01D04C2B3F5330
:10ECC0005EE03F514C5D5BE39D9A885310E1186A0A
:10ECD000F2BC188CF29CF2BE188EF29E000188ECF9
:10ECE00010F018BCF28C18BEF28E07D00101416BF7
:10ECF000436B83802F2D01D082800101865308E170
:10ED0000875306E1425304E15B510608D8A45B6BCC
:10ED10004A6B4C6B3C5102082DE15C51F1082AE131
:10ED20005E2D28D0705326E12E5323E13A5321E182
:10ED30002F5310E1186AF2BC188CF29CF2BE188EA8
:10ED4000F29E0001DFEC08F018BCF28C18BEF28EC7
:10ED50000FD00101186AF2BC188CF29CF2BE188E1A
:10ED6000F29E00017AEC16F018BCF28C18BEF28EFE
:10ED7000010104D02B6B2C5301E12D6B6ED14A6B3A
:10ED80003D53D8B46CD0422D6AD04E514B5DD8A0C3
:10ED900066D0422D03D02F2D01D04D2B40535EE085
:10EDA00040514D5D5BE39D9A895310E1186AF2BCB6
:10EDB000188CF29CF2BE188EF29E00019DEC0EF0B3
:10EDC00018BCF28C18BEF28E07D00101426B446B66
:10EDD00082802E2D01D083800101865308E1875364
:10EDE00006E1415304E15B510608D8A45B6B4B6B11
:10EDF0004D6B3D5102082DE15C51F1082AE15E2D79
:10EE000028D0705326E12F5323E13B5321E12E53A9
:10EE100010E1186AF2BC188CF29CF2BE188EF29EB9
:10EE20000001DFEC08F018BCF28C18BEF28E0FD097
:10EE30000101186AF2BC188CF29CF2BE188EF29E88
:10EE40000001ABEC17F018BCF28C18BEF28E010179
:10EE500004D02C6B2B5301E12D6BFFD04B6B092D94
:10EE6000DED03C53D8B46CD0412D6AD04F514A5DAE
:10EE7000D8A466D0412D03D02E2D01D04C2B3F536A
:10EE80005EE03F514C5D5BE39D9A885310E1186A48
:10EE9000F2BC188CF29CF2BE188EF29E000188EC37
:10EEA00010F018BCF28C18BEF28E07D00101416B35
:10EEB000436B83802F2D01D082800101865308E1AE
:10EEC000875306E1425304E15B510608D8A45B6B0B
:10EED0004A6B4C6B3C5102082DE15C51F1082AE170
:10EEE0005E2D28D0705326E12E5323E13A5321E1C1
:10EEF0002F5310E1186AF2BC188CF29CF2BE188EE7
:10EF0000F29E0001DFEC08F018BCF28C18BEF28E05
:10EF10000FD00101186AF2BC188CF29CF2BE188E58
:10EF2000F29E00017AEC16F018BCF28C18BEF28E3C
:10EF3000010104D02B6B2C5301E12D6B8ED04A6B59
:10EF40003C53D8B46CD0422D6AD04F514B5DD8A4FD
:10EF500066D0422D03D02F2D01D04D2B40535EE0C3
:10EF600040514D5D5BE39D9A895310E1186AF2BCF4
:10EF7000188CF29CF2BE188EF29E00019DEC0EF0F1
:10EF800018BCF28C18BEF28E07D00101426B446BA4
:10EF900082802E2D01D083800101865308E18753A2
:10EFA00006E1415304E15B510608D8A45B6B4B6B4F
:10EFB0004D6B3D5102082DE15C51F1082AE15E2DB7
:10EFC00028D0705326E12F5323E13B5321E12E53E8
:10EFD00010E1186AF2BC188CF29CF2BE188EF29EF8
:10EFE0000001DFEC08F018BCF28C18BEF28E0FD0D6
:10EFF0000101186AF2BC188CF29CF2BE188EF29EC7
:10F000000001ABEC17F018BCF28C18BEF28E0101B7
:10F0100004D02C6B2B5301E12D6B1FD04B6B496B34
:10F02000412D01D04A2B422D01D04B2B5B5315E0D3
:10F03000372D01D002D03C5310E1382D01D002D041
:10F040003D530BE1306B416B426B436B446B7F6A0A
:10F050007E6A5B510608D8A45B6B000190EF68F0F4
:06F0600090EF68F0FFD7FD
:020000040030CA
:0E0000000002190E000300000FC00FE00F40B9
:00000001FF
